:020000040800F2
:100000000000022091A40008D7A40008D9A4000889
:10001000DBA40008DDA40008DFA400080000000045
:10002000000000000000000000000000E1A4000843
:10003000E3A4000800000000E5A40008011800087F
:10004000EBA40008EDA40008EFA40008F1A4000848
:10005000F3A40008F5A40008F7A40008F9A4000818
:10006000FBA40008FDA40008FFA4000801A50008E7
:1000700003A5000805A5000807A5000821AA000897
:100080000BA500080DA500080FA5000811A5000884
:1000900013A5000815A5000817A5000819A5000854
:1000A0001BA500081DA500081FA5000821A5000824
:1000B0009184000825A5000827A5000829A50008A7
:1000C0002BA500082DA500082FA5000831A50008C4
:1000D00033A5000835A500080183000839A50008EC
:1000E0003BA500083DA500083FA5000841A5000864
:1000F00043A5000845A5000847A5000849A5000834
:100100004BA500084DA500084FA5000851A5000803
:1001100053A5000855A5000857A5000859A50008D3
:100120005BA500085DA500085FA5000861A50008A3
:1001300063A5000865A5000867A5000869A5000873
:100140006BA500086DA500086FA5000871A5000843
:1001500073A5000875A5000877A50008D546000816
:100160007BA500087DA500087FA5000881A50008E3
:1001700083A5000885A5000887A5000889A50008B3
:100180008BA500088DA5000810B5054C237833B960
:10019000044B13B10448AFF300800123237010BD5A
:1001A000B4020020000000007CE4000808B5064B03
:1001B0001BB106480649AFF300800648036813B137
:1001C000054B03B1984708BD000000007CE400081F
:1001D000B8020020B402002000000000154B002BE4
:1001E00008BF134B9D46A3F5803A00218B460F466E
:1001F0001348144A121A0AF030FE0F4B002B00D09D
:1002000098470E4B002B00D0984700200021040097
:100210000D000D48002802D00C48AFF300800AF012
:10022000CFFD2000290008F063FA0AF0B5FD00BFF9
:100230000000080000000220000000000000000094
:10024000B4020020E83E0020000000000000000092
:1002500030B4C3787BB902784FF461435109CEF2D0
:10026000000302F01F022031012000FA02F243F8DD
:10027000212030BC70474FF46D43CEF20003457827
:10028000DA6884780378D243C2F30222C2F104010F
:10029000C9B205FA01F10F2545FA02F2C9B22240AE
:1002A0000A4303F1604303F561431201D2B283F8BC
:1002B000002302784FF461435109CEF2000302F0AB
:1002C0001F02012000FA02F243F82120D1E700BF0B
:1002D000F0B444680B680A7924F0407424F4807404
:1002E000234343EA02234360CD680C6987688A6828
:1002F0004E794FF2FD732C43CCF2FF0322433B4077
:10030000134343EA460383600B7DC26A013B22F438
:100310007002DBB242EA0353C362F0BC704700BF15
:1003200000230360037143718360C3600361012391
:100330000375704770B44FF40C5290E84200C4F259
:10034000010285685468C06843F2E0033143CFF688
:10035000FC732943234001430B43536070BC704737
:100360000023036043608360C3607047836819B9EA
:1003700023F001038360704743F0010383607047FB
:10038000092970B421D901EB41041E3CC668072538
:1003900005FA04F526EA050503FA04F445EA040320
:1003A000062AC36020D90C2A02EB82022BD9413ADB
:1003B000C46A1F2303FA02F324EA030301FA02F1D9
:1003C00043EA0102C26270BC7047066901EB410456
:1003D000072505FA04F526EA050503FA04F445EABB
:1003E0000403062A0361DED8013A02EB8202446B61
:1003F0001F2303FA02F324EA030301FA02F143EA9A
:1004000001024263DFE7233A046B1F2303FA02F37E
:1004100024EA030301FA02F143EA01020263D2E78C
:10042000836843F080438360704700BFC06C80B234
:10043000704700BF036819420CBF002001207047BD
:10044000016846F21002002321F00101C4F2020209
:100450000160036043608360C360036121239042B5
:1004600043616BD046F22803C4F2020398426CD079
:1004700046F24003C4F2020398426ED046F258039B
:10048000C4F20203984270D046F27003C4F2020331
:10049000984272D046F28803C4F20203984275D0A3
:1004A00046F2A003C4F2020398423ED046F2B803DB
:1004B000C4F20203984273D046F21043C4F202031E
:1004C000984275D046F22843C4F20203984276D08F
:1004D00046F24043C4F20203984278D046F25843B1
:1004E000C4F2020398427AD046F27043C4F2020387
:1004F00098427CD046F28843C4F2020398427FD0EF
:1005000046F2A043C4F20203984200F0838046F210
:10051000B843C4F20203984201BF4FF4C843C4F287
:1005200002034FF03D52DA6070474FF4C043C4F20B
:1005300002030022C2F23D02DA6070474FF4C0436A
:10054000C4F202033D229A6070474FF4C043C4F2E4
:1005500002034FF474629A6070474FF4C043C4F2D0
:1005600002034FF474129A6070474FF4C043C4F210
:1005700002034FF074629A6070474FF4C043C4F2B4
:1005800002033D22C2F20002DA6070474FF4C0431A
:10059000C4F202034FF47462C2F20002DA607047E0
:1005A0004FF4C043C4F202034FF03D52DA6070478B
:1005B0004FF4C843C4F202033D229A6070474FF4DF
:1005C000C843C4F202034FF474629A6070474FF458
:1005D000C843C4F202034FF474129A6070474FF498
:1005E000C843C4F202034FF074629A6070474FF43C
:1005F000C843C4F202033D22C2F20002DA6070472F
:100600004FF4C843C4F202034FF47462C2F2000212
:10061000DA6070474FF4C843C4F202030022C2F20A
:100620003D02DA60704700BFCA680B68D0F800C0AE
:100630002DE9F0014F698E69CD690C6A42EA030821
:1006400048EA07073E434B6A35432C4344EA03021A
:100650008C6A42EA04034A6B8C6B48F23F071343EF
:10066000CFF21C0723430CEA07071F4307604469C6
:100670000A6BCB6A24F007041343234343610B69DD
:1006800043604B6883608B68C360BDE8F0017047CE
:100690000023036043608360C3600361436183613F
:1006A000C361036243628362C36203634363836320
:1006B000704700BF036819B923F001030360704756
:1006C00043F0010303607047416070470B060CD58F
:1006D0004369AAB143F08003802943610FD00368C6
:1006E00001F01E01194301607047802907D0002ADC
:1006F000F5D1036801F01E0123EA01010160704792
:1007000023F0800380294361F3D1704770B44FF424
:10071000C04246F20F454FF4C84421F0F023C4F222
:100720000205C4F20204C4F2020223F0C316A84276
:1007300088BF224696B1046804F01E0404EAD1245E
:1007400089004CBF5268126823F0821313EA02003A
:1007500002D0201C18BF012070BC7047446904F00F
:100760008004EDE710B44FF4C84246F20F444FF452
:10077000C043C4F20204C4F20202C4F20203A04263
:100780008CBF1046184611F0005F21F0F02121F0D7
:10079000821114BFC160816010BC704700222DE936
:1007A000F00113460126032703E001330232102B28
:1007B0002CD00D6806FA03F42540A542F5D1D0F8F7
:1007C00000C007FA02F4E44304EA0C0CC0F800C0CD
:1007D00091F804C0D0F800800CFA02FC4CEA080C36
:1007E000C0F800C091F804C00CF1FF3CBCF1010F4F
:1007F0000FD9C5682C40C460CC79C56804FA02F4EE
:1008000001332C430232102BC460D2D1BDE8F00179
:100810007047D0F808C004EA0C0CC0F808C091F882
:1008200005C0D0F808800CFA02FC4CEA080CC0F8AD
:1008300008C0D0F804C02CEA0505456091F806C050
:1008400045680CFA03FC1FFA8CFC4CEA0505456070
:10085000CFE700BF00234FF6FF72026003714371C0
:100860008371C371704700BF036919420CBF002038
:10087000012070470AB9418370470183704700BF68
:10088000CB08083301F0070130B4890050F8235039
:100890000F2404FA01F425EA040440F8234050F838
:1008A000234002FA01F2144340F8234030BC704761
:1008B00008B54FF4A843C4F20003984218D04FF48F
:1008C000B043C4F2000398421ED04FF4B843C4F2C0
:1008D0000003984200D008BD01214FF4000000F051
:1008E00091F94FF400000021BDE8084000F08AB9FA
:1008F00001214FF4001000F085F94FF400100021A1
:10090000BDE8084000F07EB901214FF4800000F0FE
:1009100079F94FF480000021BDE8084000F072B979
:10092000F0B5044685B068460D46A68800F0E8F8A4
:10093000029A4DF68363C4F21B33A3FB021326F025
:100940003F06980C3604360C87B23E43A6802388B7
:1009500023F001031B041B0C238048F2A0612B68C9
:10096000C0F201018B4222D85B00B2FBF3F292B2DB
:1009700001372784032A98BF0422A28323889BB2CD
:1009800043F00103238023886989AA8823F48163C3
:1009900023F002031B040A431B0C13439BB2238066
:1009A0002A89AB8913439BB2238105B0F0BDEE8841
:1009B0004BF6FF718E421DBF03EB830303EB8303F2
:1009C000B2FBF3F203EB43030CBFB2FBF3F242F4CE
:1009D000804292B213051B0D0BB942F001024FF495
:1009E000967344F6D35103FB00F0C1F2620181FB20
:1009F00000318909013142F400422184BDE700BF82
:100A0000002341F28832026083804BF6FF7203813B
:100A100043814FF48043C28083817047038829B9A2
:100A200023F001031B041B0C038070479BB243F0AF
:100A300001030380704700BF038829B923F4807342
:100A40001B041B0C038070479BB243F4807303802C
:100A5000704700BF038829B923F400731B041B0CE3
:100A6000038070479BB243F400730380704700BF5C
:100A70001AB901F0FE010182704741F001010182C3
:100A8000704700BF038829B923F480631B041B0C43
:100A9000038070479BB243F480630380704700BFBC
:100AA000038819B95B045B0C038070476FEA43430A
:100AB0006FEA53439BB20380704700BF01827047C7
:100AC000008AC0B2704700BF82B000230A0F0093B3
:100AD000019301900092009B21F07F4153B1019B53
:100AE00014330193019B1B6819420CBF00200120A5
:100AF00002B07047019B1833090C0193F2E700BF65
:100B000010B44FF46053C4F202039A6802F00C026E
:100B1000042A22D0082A26D04FF41052C0F2F40240
:100B200002604FF46053C4F2020320499C68C4F38E
:100B300003140C5D22FA04F242609C68C4F3822420
:100B40000C5D22FA04F484609B68C3F34233CB5CEF
:100B500022FA03F2C26010BC70474FF49052C0F208
:100B60007A020260DDE75C68596814F4800F5C6803
:100B700015BF4FF490534FF41053C0F27A03C0F2F4
:100B8000F40301F03F01B3FBF1F24FF46053C4F200
:100B90000203C4F388145B68C3F30143013302FB0F
:100BA00004F25B00B2FBF3F20260BAE7000000203F
:100BB0004FF46053C4F202031A6B19B922EA000021
:100BC0001863704710431863704700BF4FF46053B9
:100BD000C4F202031A6C19B922EA000018647047C3
:100BE00010431864704700BF4FF46053C4F202030F
:100BF0005A6C19B922EA00005864704710435864CF
:100C0000704700BF4FF46053C4F202031A6A19B967
:100C100022EA00001862704710431862704700BF54
:100C2000002270B44FF48064C4F201020388C4F25D
:100C30000104904218BFA0429BB214BF00220122BF
:100C400008D04FF48064C4F20004B0F1804F18BFA4
:100C5000A04223D14FF68F754C881D4045EA04030E
:100C60004FF4A0564FF48055C4F20005C4F20006BC
:100C7000B04218BFA8421FBF0D894FF6FF441C4069
:100C800044EA050303804B68C3620B8803850AB1FD
:100C90008B7A03860123838270BC70474FF44065D2
:100CA0004FF40064C4F20005C4F20004A04218BF6F
:100CB000A842D5D1CEE700BF00234FF0FF314160FD
:100CC0000380038143808372704700BF038829B982
:100CD00023F080031B041B0C038070479BB243F07E
:100CE00080030380704700BF038829B923F0010304
:100CF0001B041B0C038070479BB243F0010303806D
:100D0000704700BF038C23F001031B041B0C0384FA
:100D10002DE9F001038C8D8984884F88028BB1F80E
:100D200000C02F4322F07302002523F002034FF48A
:100D3000806612041B04C4F20106C4F20105120C01
:100D40001B0CBFB2A84218BFB042A4B242EA0C02C8
:100D500047EA030316D14FF6F775B1F80EC0B1F8A4
:100D600012800F8A8E881D4045EA0C0C4FF6FB73EB
:100D70004FF6FF4548EA070725400CEA0303BCB2DB
:100D800033432C43848002838A6842630384BDE832
:100D9000F001704700230380438083808360838158
:100DA000C381038243827047038B23F008031B0433
:100DB0001B0C194301837047B0F8443021B95B0420
:100DC0005B0CA0F8443070476FEA43436FEA53432B
:100DD0009BB2A0F84430704783899BB21AB923EACA
:100DE000010181817047194381817047C94389B2EC
:100DF0000182704783899BB21AB923EA010181817C
:100E0000704719438181704770B5038ACA8823F4FB
:100E100040531B041B0C1343038283898A880446B6
:100E200008890D4623F4B0534989024323F00C038B
:100E30001B040A431B0C92B21343A381A38AAA8901
:100E400023F440731B041B0C84B01343A382684635
:100E5000FFF756FE4FF4A0524FF48053C4F2010343
:100E6000C4F201029C4218BF9442A2890CBF039BAA
:100E7000029B12B2002A21DB286803EB830303EBF9
:100E800083038000B3FBF0F148F21F53A089C5F241
:100E9000EB13A3FB0152520900B21601642500288E
:100EA00002FB151213DB12013232A3FB0253C3F310
:100EB000431333439BB2238104B070BD2A6803EB14
:100EC000830303EB83035200B3FBF2F1DCE7D200B0
:100ED0003232A3FB0213C3F342133343EAE700BFEA
:100EE0004FF41652002302600C228380C3800381DA
:100EF00042818381704700BF838929B923F400535D
:100F00001B041B0C838170479BB243F40053838105
:100F1000704700BF838919B95B045B0C83817047FC
:100F20006FEA43436FEA53439BB28381704700BF2C
:100F3000C905C90D818070478088C005C00D704704
:100F400001F01F0310B4C1F342110124A14204FABD
:100F500003F30DD002290DD014302AB9026822EA19
:100F60000303036010BC7047026813430360F9E792
:100F70000C30F2E71030F0E7C1F3421310B401F087
:100F80001F020124012B04FA02F416D0022B0CBF1D
:100F9000028A828A92B2224003880124090A04FA52
:100FA00001F19BB219420CBF00200120002A0CBFA6
:100FB000002000F0010010BC7047828992B22240EC
:100FC000EAE700BF090A012303FA01F1C94389B224
:100FD0000180704770B52A4D2C688CB0002C4BD125
:100FE0006846FFF737FC06A8FFF79AF904200121AD
:100FF000FFF7DEFD10234FF40060C4F202006946E3
:10100000009303238DF804308DF80740FFF7C6FBEB
:1010100001214FF48070FFF7E7FD02A8FFF7A0F968
:101020004FF4803302A80393029404940594FFF7CD
:1010300081F94FF400500126C4F2010006A906947C
:101040008DF81C408DF81D4008940A948DF82C6092
:10105000FFF73EF94FF400502346C4F201000E2181
:101060003246FFF78DF94FF40050C4F201003146CB
:10107000FFF77CF9034B1E6001232B600CB070BDA1
:10108000D4020020FC3D00204FF4005008B5C4F20B
:101090000100FFF7C5F940F2D023C2F2000301229C
:1010A0001A6008BD38B50D4C236805460BB9002001
:1010B00038BD4FF40050C4F201000221FFF7BAF925
:1010C0000028F4D04FF40050C4F20100FFF7AEF94D
:1010D000002328802360012038BD00BFD0020020FB
:1010E00030B448F6396301EB4105941EC3F6E303BF
:1010F0000229C1EBC501D8BF144683FB0153D8BFF9
:10110000013AC917C1EB6301201848F21F54D51CDE
:101110000818C5F2EB1484FB02340430D31732EA0A
:10112000220228BF2A46A3EB641100EBA202C3EB04
:10113000E413521842F29340D218C9F2492080FBBE
:1011400002508018D317C3EBA000C0EBC000101AE8
:1011500030BC704770B40646002922D00078F0B148
:1011600000231846F25CA2F13004E4B2092CA2F18B
:1011700041050DD9052DA2F161049CBFA2F13704F0
:10118000E4B205D9052C9ABFA2F15704E4B20024B9
:101190000133DDB204EB0010A94280B2E2D870BC8A
:1011A00070470846FBE700BF0020C4F20200202180
:1011B0000122FFF75FBB00BF0020C4F20200202124
:1011C0000022FFF757BB00BF00B583B06846FFF7AA
:1011D00041FB01200146FFF7EBFC002020220346E3
:1011E0006946C4F20200009201228DF805308DF8A4
:1011F00004208DF806308DF80730FFF7CFFAFFF79F
:10120000DBFF03B000BD00BF00B583B06846FFF749
:1012100021FB04200121FFF7CBFC4FF400600023E9
:101220004FF40052C4F20200694600928DF8043077
:101230008DF80730FFF7B2FA03B000BD4FF400603D
:1012400008B54FF40051C4F20200FFF70DFBD0F1D6
:10125000010038BF002008BDF0B412490A680346F7
:10126000E2B11148114D066811482D680768114810
:101270009D6004681048114D00682D68D8600020FA
:10128000072C08BF04465D60013F06F164059C61C0
:101290000F245D611F6118621C6008601046F0BC7D
:1012A000704700BF00030020D80200200803002080
:1012B00010030020EC020020DC020020E4020020E9
:1012C000F0B583B068464FF40065FFF7C3FAC4F287
:1012D000020504200121FFF76BFC00244FF400639A
:1012E0006946284600938DF805408DF804408DF836
:1012F0000740FFF753FA6846FFF7ACFA04200121D4
:10130000FFF756FC4FF480570126284669460097A0
:101310008DF805408DF804608DF806408DF8074083
:10132000FFF73CFA284639463246FFF7A3FA03B0E6
:10133000F0BD00BFF8B5A44C2368FF2B56D04FF486
:101340000060C4F202004FF40061FFF78DFA054619
:10135000002833D0FFF728FF23689B4D0120012B85
:1013600033D04AD3022B4DD0984B1A68904200F0EC
:101370008680974E186033689A1F0221122A2960CE
:1013800063D9052B94BF93489348944F06F082FF8E
:10139000934806F07FFF002323603B680F2B00F08B
:1013A000CC81102B6ED0FF2B3AD001333B2B3B600E
:1013B00000F0CE8134D90023236031E0FFF7FCFE3A
:1013C0002368012B2846804DCBD1804B1A6882427E
:1013D00029D01860814BFF221A607D4B002814BF72
:1013E00003200220002220601A60F8BD7D4B1A689D
:1013F000642A19D001321A60F8BD01232B60734BA7
:101400001860F8BD714B1A68904238D0704E186061
:1014100033680322782B2A6012D9704B00221A609D
:1014200000233360F8BDF8BD4FF40060C4F2020041
:101430004FF480510022FFF71DFA00232360F8BD0E
:101440004A2BEDD800232B60EAE7644F0F2B3B6853
:1014500034D8232B00F097813A2B00F085811C2B88
:101460009CD1614A1268D0079FD5604806F012FFF0
:101470005B4806F00FFF002323603B688EE7544B68
:101480001A68B7E75A4A002313605A4A1360564A4B
:101490001360594A1360594A1360594A1360594AF4
:1014A0001360594A1360594A1360594A1360594AE4
:1014B0001360594A136011233B60B1E7A3F1110295
:1014C000292A3FF66BAF01A151F822F0331700082B
:1014D0009D1300089D1300089D1300082D17000898
:1014E00027170008211700081B1700081517000808
:1014F0000F17000809170008F9160008F31600086E
:10150000ED160008E7160008E1160008DB160008D3
:10151000D5160008C5160008BF160008B916000841
:10152000B3160008AF160008AB160008A71600088F
:10153000A11600089B160008951600088F160008D3
:1015400089160008831600087F1600087B1600081D
:1015500069160008571600084516000833160008DB
:1015600021160008B7150008A515000893150008F6
:1015700075150008214A126812F001057FF415AFB5
:10158000264806F087FE164806F084FE25603B6874
:1015900004E72149194A0D681068503501300D6083
:1015A0001060FEE61C49154A0D68106828350130A8
:1015B0000D601060F5E61849104A0D681068143582
:1015C00001300D601060ECE630000020F0020020D9
:1015D0000403002000BF000820BF00082C000020EA
:1015E00038C900080C030020E002002040BF0008BA
:1015F00000030020F802002014030020E80200206D
:10160000FC020020E402002008030020EC0200207D
:10161000DC02002010030020D802002088BF000850
:101620006549664A0D6810680A3501300D60106022
:10163000B7E66149614A0D681068083501300D60F0
:101640001060AEE65C495D4A0D68106804350130F3
:101650000D601060A5E65849584A0D6810680235BB
:1016600001300D6010609CE65349544A0D681068C3
:10167000013501300D60106093E65149D1E75049C2
:10168000D8E74F494D4ADFE74D494C4AE5E74C4919
:101690004A4AEBE74B49494AD6E74A49474ADCE719
:1016A0004849464AE2E7484986E74749B9E7464993
:1016B000C0E74549414AC7E74349404ACDE7424967
:1016C0003E4AD3E7414A126812F001057FF46DAE3D
:1016D0003F4856E73F493D4A6FE73E493B4AA1E74D
:1016E0003C493A4AA7E73B49384AADE73949374AC6
:1016F000B3E73849354AB9E7374A126812F00105AD
:101700007FF453AE35483CE73549334A4CE734491A
:10171000314A52E73249304A84E731492E4A8AE752
:101720002F492D4A90E72E492B4A96E72C492A4A01
:101730009CE72C4A0121116033E62B4B1A6822B139
:101740002A4A0121116000221A6010233B6067E6DB
:10175000274B204A196812689142264922D0204816
:1017600000681A6008605BE6144A1268D2077FF5C9
:101770001CAE214806F08EFD204806F08BFD0022AD
:101780003B682A600AE6114A1268D1077FF50DAE60
:101790000F4806F07FFD194806F07CFD00232B6002
:1017A0003B68FBE50E480C68006801348442D8D1E0
:1017B0000D4C01252560D4E7D8020020E802002066
:1017C00010030020EC020020DC02002014030020A3
:1017D00064BF000808030020E002002040BF0008AA
:1017E000E4020020FC020020F80200200003002098
:1017F00018030020F402002088BF000838C9000840
:10180000034B1A6812B11A68013A1A60704700BF98
:10181000003E0020064B074A1B68012B1EBF064BEB
:101820001B68B0FBF3F010601368002BFCD170470D
:101830001C030020003E002038000020044B054A15
:101840001B6803FB00F010601368002BFCD170478D
:1018500034000020003E0020084B094A1B684FF46A
:101860007A7110F1FF3001FB03F106D311601368A8
:10187000002BFCD110F1FF30F8D27047340000206B
:10188000003E0020012810B423D002282CD01C4B8D
:1018900064221A601B4B0A221A6042F21071032064
:1018A000194B1C684EF21003CEF200034FF46D4248
:1018B000B4FBF1F1CEF2000201395960F02182F857
:1018C000231000229A6007221A60104B186010BC87
:1018D00070470B4B18600B4B44F240214FF47A7267
:1018E0001A60C0F20F01DBE7054B0A221A60054BB4
:1018F00048F2A06164221A60C0F20101D0E700BF83
:101900003800002034000020E80100201C030020E3
:101910002DE9F00140F26C1040F2A81540F24C01A4
:10192000C2F20000C2F20001C2F2000540F2A014AF
:1019300040F2400240F24403C2F20002C2F200034D
:1019400090F8008090F801C087780E7848782D686C
:10195000897882F80080C2F2000482F801C0256014
:1019600097701E7058709970BDE8F001704700BF05
:10197000722009F071B800BF70B5214A82B01160C1
:10198000204A002310608DF804308DF805308DF862
:10199000063000282AD01C481C4A857804784678EE
:1019A00032F8144032F8160032F815208DF8004055
:1019B0004CF6CD45CCF6CC45A5FB0145AD0805EB75
:1019C00085058DF801008DF802204D1B1C46A542AF
:1019D000204601A988BF6946013409F0DDF8042CCE
:1019E000F5D1042009F038F802B070BD0446204655
:1019F00001A9013409F0D0F8042CF8D1F1E700BFB7
:101A0000E4030020400300204C000020ACC3000889
:101A1000D62009F021B800BF70B505460E467224E5
:101A200020462946013409F0B7F8D62CF8D106B97A
:101A300070BDBDE87040FFF7EBBF00BF30B540F2AE
:101A40004402C2F200024CF2AC33C0F6000311783B
:101A50009478557833F8111033F8152033F8143092
:101A600083B08DF80410014601A88DF805208DF88B
:101A70000630FFF7D1FF03B030BD00BF00B583B023
:101A80000023014601A88DF804308DF805308DF84B
:101A90000630FFF7C1FF03B000BD00BF30B51A4BE1
:101AA0001A4D1B688DB0EBB100232A461C46116904
:101AB00011F0020F02F1140205D00CA800EB840112
:101AC000013441F82C3C01330B2BF0D16CB9104A96
:101AD0002346146003EB830305EB83056B6898478B
:101AE0000DB030BD0A4B1B68F4E709F04BFCB0FBAE
:101AF000F4F30CAA03FB140002EB8003044A53F82E
:101B00002C3C1360E6E700BF2004002050000020BA
:101B1000D00300200E2A30B436D81F4B0C789B5CC3
:101B200048F6890213FB04F4C8F68802A2FB0452AB
:101B3000C2F3C70202700C7814B10AB90122027014
:101B40004C7848F6890213FB04F4C8F68802A2FB1D
:101B50000452C2F3C70242704C7814B10AB9012290
:101B600042708C7848F6890213FB04F3C8F68802A9
:101B7000A2FB0342C2F3C70282708B7813B10AB989
:101B80000123837030BC70470B7803704B7843702F
:101B90008B788370F6E700BFA4C4000810B5104B23
:101BA000104C1A68104982B02046FFF7B3FF0F4B64
:101BB0001B689BB10E4B2178A078627833F8111026
:101BC00033F8122033F810308DF8041001A80121E9
:101BD0008DF805208DF80630FFF71EFF02B010BD0E
:101BE000A0010020440000204000002070010020DF
:101BF000ACC300080E4B1B68032B18D8DFE803F0BA
:101C000013100A020B4B00223F2119705A709A7070
:101C1000FFF7C4BF084B012200201A60FFF72EBF58
:101C20000020FFF72BBF054B1868FFF707BF704771
:101C3000EC0300204000002024040020700100205C
:101C40002DE9F00F0C0682B04DD4DFF810C1424CE4
:101C500001276FEA020904EBC10BC2F1040A3D46F9
:101C6000CDF80490ACF10B060021042A1AD8544692
:101C70000BEB070801460A290DD818F8019C49FA10
:101C800004F933B319F0010F05D01CF8019049F0A5
:101C900002090CF80190013C0131B4F1FF3FEAD197
:101CA0000199063163B909180A2909D807EB870891
:101CB00007EB480808EB010401310A293555F9D929
:101CC0000137092F0CF10B0CCED102B0BDE8F00F9B
:101CD000704719F0010F1ABF4FF004090CF801907A
:101CE0000CF80150D7E7B0394C292AD8DFE801F0C9
:101CF0002B29292929292929292929292929292952
:101D0000292929292D29292929292929292929293F
:101D10002929292929292F29292929293129292727
:101D2000292929292D29292929292929292929291F
:101D30002929292929292F2929292929310005215A
:101D400083E7202181E701217FE702217DE703214D
:101D50007BE7042179E700BFACBF0008133E0020F9
:101D60006D2812D848F6A333CBF62E23A3FB00230D
:101D7000DB08DA0741BF03EB830203EB4203C0EB4E
:101D800043000A30043008F007BF704770B52B4B92
:101D90001A6882B006460AB901261E60284A294BF5
:101DA00011785478907833F8111033F8142033F800
:101DB0001030254D8DF8001000248DF801208DF88D
:101DC00002308DF804408DF805408DF806400AE099
:101DD000FFF7C6FF15F8013C013443F001036E2CF8
:101DE00005F8013C15D015F8013B03F00203DBB206
:101DF00020466946002BEBD1204601A9FFF7B0FF32
:101E000015F8013C013423F001036E2C05F8013C68
:101E1000E9D10E4B18680E4B1968FFF7ADFD16B1EE
:101E20000C4B1B6833B1FFF7A3FD0B4B01221A606B
:101E300002B070BD0120FFF701FEF6E7F0030020BD
:101E40004C000020ACC30008083E002040030020E6
:101E5000E4030020EC030020043E002008B5064BFC
:101E60001A6822B1002210461A60FFF78FFF034B59
:101E700001221A6008BD00BF20040020043E00209B
:101E800008B50D4B0D481A680D49FFF743FE0D4B81
:101E90001B68032B03D00C4B1B68990708D40B4B12
:101EA0001B6803B908BD0120BDE80840FFF76EBFFD
:101EB000FFF72EFDF3E700BFA80100204C00002033
:101EC0006C010020EC03002048000020700100207D
:101ED0002DE9F041854B1A6884B03AB984490B6802
:101EE000002B00F0E28004B0BDE8F081814A804917
:101EF0001678DFF818824CF6CD40CCF6CC40A0FB2B
:101F00000650002400091C600C6000F0B380C8F883
:101F100000005578DFF8F8C14CF6CD43CCF6CC4341
:101F2000A3FB05031B0902D1002D40F0BC80CCF8B7
:101F300000309478704F4CF6CD43CCF6CC43A3FBE5
:101F400004231B0902D1002C40F0AB806B4A3B609C
:101F50006B4B00201070507090701E705D709C7004
:101F6000D8F800301C4693B1654A1478A34240F279
:101F7000948014B1002010700124604A5D481578E7
:101F80000078EB18834200F2A08013700124DCF883
:101F900000308BB15A48427893427AD912B100226C
:101FA00042700124554A534855784078EB188342D3
:101FB00000F29080537001243868002861D0504BA3
:101FC0009A78904261D912B100229A7001244B4D47
:101FD000484AAF7896783818B0429CBFC0B2A87013
:101FE00003D9B7424DD0AE703046464992F800C092
:101FF00092F801E06C782F785A781D789B7831F848
:102000001C8031F8177031F81EC031F8122031F8F9
:1020100016E031F8133031F8146031F8104031F81F
:1020200015008DF80A40384D8DF804808DF805C0F4
:102030008DF806E08DF808708DF809608DF80C00B9
:102040008DF80D208DF80E30002406E0012B32D0E3
:10205000032B35D001346E2C09D0635D022BF5D1F2
:10206000204602A90134FFF77BFE6E2CF5D1FFF765
:102070007FFC38E7002E3FF44AAF0123C8F8003058
:1020800047E764BB01230B602DE7121A9A70012405
:102090009DE7D21A4270012484E7E41A14700124E7
:1020A0006BE7012352E7012341E7DFF86080DFF8A7
:1020B00060C0114F54E7204603A9FFF751FEC9E75E
:1020C000204601A9FFF74CFEC4E785421CBF1070F3
:1020D00001245CE785421CBF507001246CE7054A6F
:1020E000064D9678A878064B7FE700BF20040020B5
:1020F000043E00204C000020340400205C0300203B
:1021000020030020ACC30008083E0020C4030020C8
:10211000AC03002070B5154A154B947811785578AA
:1021200033F8111033F8152033F81430114E82B003
:1021300000248DF8001005468DF801208DF802303E
:102140008DF804408DF805408DF80640A35D2B42C4
:10215000204601A918BF69460134FFF701FE6E2C25
:10216000F4D1FFF705FC02B070BD00BF4C000020A9
:10217000ACC30008083E00202DE9F843584B594DE8
:102180001A682AB92E68002E00F09B80BDE8F883FB
:10219000DFF8588100221A602A60C8F80020524CEB
:1021A0004FF0000E7646A4460EEB8E000EEB40007C
:1021B0000B230CEB00095A1E81186718615C11F0A3
:1021C000010F46D00A2A00EB03064BD01CF806602C
:1021D000F60742D421F001013970002A47D0023BB2
:1021E0000126002BE7D10EF1010EBEF10A0FDBD163
:1021F0000120FFF78FFF002E5FD0D8F800300126B6
:10220000012B08BF384CC1D1374F4FF0000EB846F4
:102210000EEB8E000EEB4000002308EB000CC21802
:1022200004EB0209A25C02F00601022926D0013368
:102230000A2BF4D90EF1010E0B37BEF10A0FE7D1CC
:102240000420FFF767FF002EA0D101232B60BDE81B
:10225000F8831346002BAED1C5E713460126002BA9
:10226000A9D1C0E721F0010189F80A10B7E70EF102
:10227000010E0126BEF10A0F96D1B9E743B302F071
:102280000401C9B20029D2D142F004020A2B89F814
:10229000002022D00133C218A25C02F00202D2B2A6
:1022A0004AB10A2B03F1010317D0FA5C02F00202D3
:1022B000D2B2002AF5D10126BAE70123C8F80030CE
:1022C000A2E7DFF82880D8F80030002B98D166E725
:1022D00042F004028CF80020DCE70126AAE700BFE8
:1022E00020040020043E0020083E0020300400208E
:1022F0002DE9F00F6C4B1A6832B96C4A1368002B49
:102300006BD0BDE8F00F704700201860674A684E38
:10231000684B106001213160196033688BB16648E9
:102320000A256C1E0023C25C02F00301012938D08B
:1023300001330B2BF7D10B382546002CF1D134603B
:1023400043E0DFF870A1DAF80010002942D0DFF88E
:102350007CB1DBF80020002A41D0584D58492A684A
:1023600008685849584E02EB820402EB44042418D2
:1023700001320F5D2A6002EB820502EB450527F072
:10238000040728180F5536680C5CB24244F0040567
:1023900008BF44F005040D5404BFCBF800300C54C2
:1023A00013E004EB840004EB40004649C01822F01F
:1023B0000102092C0A5408D005EB850205EB420501
:1023C000EB18CA5C42F00102CA540520BDE8F00FC8
:1023D000FFF7A0BE0123136093E7354E9DE740F25F
:1023E000C031C2F2000140F250330F68324840F26F
:1023F0007431C2F20003C2F20001D3F80090D1F8A8
:10240000008094460A25A0F163066C1ED30749D4C8
:102410000023C25C02F00301022905D001330B2B1B
:10242000F7D14B46002211E0ACB112F0010217D0F7
:1024300005EB850205EB4202D218A846B15C41F0DB
:102440000401B1544FF0010C2746012225460B38F8
:102450008CB19946D9E7F25C42F00502F254F3E7F9
:10246000BCF1000FF0D1F15C41F00401F1544FF0E8
:10247000010C9046E8E740F2C031C2F20001CBF80F
:1024800000C00F6040F25031C2F200010B6040F218
:102490007433C2F20003C3F80080002A95D1CAF851
:1024A000002092E74B46D1E720040020043E0020A4
:1024B00044030020E00300206B3E00207403002052
:1024C00050030020083E0020C0030020FC03002031
:1024D0002DE9F8436B4B1A6832B96B4D2B68002B12
:1024E00000F0A680BDE8F88300201860674C664BBA
:1024F000206018604FEA8008654B08EB0007C0F1C8
:102500000B0600EB400200EB470703EB8202F719D2
:102510001D469946DF191346197841F0040103F866
:10252000011BBB42F8D1C0F1090E431C73454FEAB1
:102530008E0C18D208EB000300EB09070CEB0E0120
:1025400005EB43030B3F0EEB41010A337F18D17AB1
:1025500041F0040102F80B1FD97ABA4241F004019C
:1025600003F80B1FF3D10CEB0E020EEB42025219D3
:102570000346D15C41F00401D1540133B342F8D396
:1025800000284DD0421EC0F10C07BA4210D202EB17
:10259000820102EB41010B185B197E19013B761891
:1025A00013F8011B21F00401B34203F8011CF7D119
:1025B000C0F10A08404528BF4FEA880920D200EB45
:1025C00080034FEA880900EB430309EB08019B18DD
:1025D00002EB050C08EB4101C0F10B065B198C44C2
:1025E00093F800E0991A2EF0040E83F800E011F839
:1025F00006E00B332EF0040E634501F806E0EFD140
:1026000009EB080308EB43031B185B19013B13F8A4
:10261000011B013221F00401BA4203F8011CF6D378
:102620000420FFF777FD236801332360BDE8F883BA
:10263000164C206804287FF65DAF05281CBF144B9C
:1026400003F16E0404D119E0A34203F8010C0ED08B
:1026500013F8012B02F00201C9B242F0040022F08B
:1026600004020029F0D1A34203F8012CF0D1042088
:10267000FFF750FD01232B60BDE8F88304220727F4
:10268000034D84E720040020043E00207003002056
:10269000083E002070B5254A254813681BB9036819
:1026A000002B39D070BD00231360224D224A0360F5
:1026B0002B6013602E6886B9204B03F16E011A78E7
:1026C00022F0040203F8012B8B42F8D10420FFF71B
:1026D00021FD2B6801332B6070BD174A136801334D
:1026E0001360DA07DED5741EA4B26D2C0FD813491F
:1026F0000B5D03F00202D2B22AB10FE00B5D03F0D2
:102700000202D2B252B90134A4B26E2CF6D1012326
:10271000036001362E6070BD064DCBE743F0040325
:1027200004200B55661CFFF7F5FCF2E7200400209F
:10273000043E0020080400202C040020083E002055
:102740002DE9F00F8F4B1A6886B042B98E4B1A688C
:10275000002A00F00D8106B0BDE8F00F704700229E
:102760001A608A4C884B22601A600292DFF820C2FD
:10277000002000EB800200EB42026244002311784B
:10278000013321F004010B2B02F8011BF7D10130BA
:102790000A28EED1029A029B0132C3F1040305928A
:1027A00022600093002000EB0C020023117801331B
:1027B00021F008010B2B02F8011BF7D10B306E281A
:1027C000F1D1009F724CDDF800B07F420197BA460C
:1027D0000027BAF1050F2CBFD1464FF005099DE83F
:1027E00006000023BBF1040F34BFD8464FF00408A5
:1027F0001AE0042934BF0D460425042B404603D9B2
:10280000052A2CBF1546052500EB800600EB460087
:1028100040191CF8005045F008050CF80050013331
:10282000013101320B2B15D0E05C00F00200C0B288
:102830000028F4D0042FDCD9042B05D8042934BF98
:102840000D4604254846DFE7042A8CBF15460525BA
:102850004846D9E701370B340A2F0AF1010A0BF178
:10286000010BB6D1029ADDF808A0DDF814B06FF0C4
:1028700015036FF0090909FB02F903FB02F2534645
:102880000020DB430190049280460393CDF800B012
:10289000039F029807EB080303EB83050AEB8A0208
:1028A0000AEB420203EB4505019B16182D18D219BD
:1028B00003EB0C016644624465445C4600231EE061
:1028C000042B30D8C34509D89B4507D8049FD0199D
:1028D00010F80B7C47F0040700F80B7C11F8010B93
:1028E00000F00807FFB21FB140F0040001F8010C2E
:1028F000013301360132013501340B2B25D002EBB7
:1029000009004078C007E9D5B8F1040FD8D9042BE5
:10291000009811D80928E1D89B45DFD8D07A40F03B
:102920000400D072DAE7C345D8D80A2CD6D8687824
:1029300040F004006870D1E70928CFD80A2C9EBF68
:10294000307B40F004003073C8E7019A009B08F127
:1029500001080B320133B8F10A0F01920AF1010AA2
:10296000009395D1042006B0BDE8F00FFFF7D2BB6D
:10297000064C2068042802907FF6F8AE01221A6007
:10298000E9E600BF20040020043E0020CC03002024
:10299000083E0020F8B59B4C2368002B40F0A28035
:1029A000994B1B68032B11D8DFE803F07242110228
:1029B0002368002B40F0C280944A136833B99449CD
:1029C0000B686D2B40F2C18001231360F8BD2368B2
:1029D000002B00F09D808B498E4B00220A608B49B2
:1029E0001A600A608C4802F10B0500F10B071D60AC
:1029F0000021BF1A8B1A1B187C180DE013F80B6C02
:102A000016F0010F9E5C00F0EC8046F004069E5428
:102A100001339C4200F0EC808D42EFD993F8636063
:102A200006F00206F6B2002E00F0DA809E5CECE7BB
:102A30002368002B76D07349784A00230B607349D2
:102A400013600B605F1C744817601E4603F16E0C28
:102A5000594203F10C0433183A460DE05D7815F045
:102A6000010F5D5C00F0AF8045F0040501325D545C
:102A70000133A24200F0AF800A2AEFD913F80A5CB2
:102A800005F00205EDB2002D00F09C805D5CEBE7E7
:102A90002368002B31D05B4A614B002111605B4AF7
:102AA000196011604C1C5C481C604E42C1F16E07FD
:102AB000331800220CE013F8015C15F0010F5D5C87
:102AC00074D045F0040501325D5401330B2A74D0F3
:102AD0009442F0D99D7A05F00205EDB2002D64D044
:102AE0005D5CEEE708F04EFCC217920F831803F00E
:102AF00003039B1A444A136054E7444A1368002BAB
:102B00007FF464AF464B19680A293FF65DAFC9E709
:102B10003E490B68002B7FF459AF3E4B1A686D2A73
:102B200009D85FE739490B68002B7FF44FAF3B4A68
:102B300013680A2B86D901230B60F8BD314A34494A
:102B400000231360314A0B601360334803F10B021A
:102B50001B180A6003F1160C002113180CEB01047A
:102B60000CE01F789E1A17F0010F354611D0755CE6
:102B7000013345F004059C42755411D06D2AF0D9FB
:102B800013F86E7C07F002079D1AFFB22E46002F45
:102B9000EDD16E5C013326F004069C426E54EDD1FB
:102BA0000B310B326E29D8D126E05D5C25F004058F
:102BB00001325D5401330B2A8AD10B36BE427FF4B9
:102BC00077AF19E05D5C25F0040501325D540133F7
:102BD000A2427FF451AF0B3666457FF43CAF0BE069
:102BE0009E5C26F004069E5401339C427FF414AF91
:102BF0000B316E297FF4FEAE0420BDE8F840FFF7EC
:102C000089BA00BF2004002010040020043E0020E8
:102C10001C04002078030020083E00200C04002043
:102C20006C0300202DE9F04FB54AB64E136885B00D
:102C300033B93368002B00F0978005B0BDE8F08F02
:102C400000231360B04AB14C1360B14AB14D136018
:102C5000B14A336023602B6013602368002B44D19A
:102C6000AE4A11781F2960D951781F2900F2C88017
:102C70003F228DF808308DF809208DF80A30A84BD6
:102C8000A84E1A68A04F03A802A9FEF743FF2968BF
:102C90009DF80C809DF80DC09DF80EE0A24B36F813
:102CA000188036F81CC036F81EE038689F4A83F852
:102CB000008001EB810601EB460108180026194649
:102CC00083F801C083F802E0167056709670FFF723
:102CD00047F823682968964A3868D15495495A1CA0
:102CE000C8542260FEF744FEA7E72A680F2A24D9B9
:102CF000914B03F16E0403E0A34203F8010C0ED0E4
:102D000013F8012B02F00201C9B242F0040022F0D4
:102D100004020029F0D1A34203F8012CF0D10420D1
:102D2000FFF7F8F90123336087E73F228DF8082089
:102D30008DF809308DF80A30A1E7DFF8D4C1724F61
:102D4000DCF80030D7F800809A4279D0724B1B68CB
:102D500002F00109B9F1000F4BD143452ED908F11A
:102D600001033B602A6830E0684C6A4D75E7BBF1AF
:102D70000A0F1AD85B460EEB8E000EEB400043F6AE
:102D80000868C018C2F2000818F8008018F0010F97
:102D9000DDF8008004D0E5E0C85CC00700F1E28007
:102DA00001330B2BF8D1CDF800800EF1010E0B3161
:102DB000BEF10A0F67D11023CCF80030DCF80030E8
:102DC0009A4228D301232A683360092A2ED923681E
:102DD000DFF85C81062B7BD0564E29683A6808F8EC
:102DE0000310052BF25401D801332360FEF7C0FD18
:102DF00023E74345E2D208F1FF333B602A68E4E76A
:102E000092781F2A0AD88DF808308DF809303F23B0
:102E10008DF80A3033E701322A60D6E73F228DF879
:102E200008308DF809208DF80A2028E702EB82008F
:102E30003B683D4902EB4000C018FEF791FFC6E732
:102E400040F2D830C2F200000368984580D112F0F9
:102E5000010900F08F8008F1FF3B9246B8F1000FA6
:102E600002D102F1010AC346BAF1090FA3D80AEB55
:102E70008A0143F608630AEB4101C2F200035918C4
:102E8000D646CDF80080D64562D01EF001033FF44F
:102E900072AF0A230EEB8E000EEB400043F608687B
:102EA000C2F20008C01818F80000DDF80080C00762
:102EB00006D4002B3FF477AF013BC85CC007F8D5C0
:102EC00040F2D830C2F20000CCF800E0036041E7E5
:102ED00098F80030174E092B30D90023013308EB46
:102EE000030218F80300F15C02F8010CF218052B3C
:102EF00002F8011CF2D12368013B23606DE700BF9B
:102F000020040020043E002018040020600300205C
:102F1000B8030020E8030020D80300206C01002043
:102F2000A8010020ACC30008F403002064030020C3
:102F30005403002048030020083E00203278124944
:102F400003EB830003EB40008018FEF709FFC4E7A2
:102F50001EF0010F3FF40BAFBBF1FF3F18BF5B4604
:102F600098D122E740F2D831C2F20001CCF800E05B
:102F70000B60EFE6B8F1090F9CBF08F1010B924618
:102F80007FF672AF6DE700BF640300202DE9F04FBC
:102F9000874B884D1A6885B0002A40F09B802B68CB
:102FA000002B58D1DFF820A2DAF800201D2A55D8CE
:102FB000DFF80CB2DFF818829BF800009BF80110D4
:102FC0009BF802208DF80C008DF80D108DF80E2066
:102FD0009946D8F804400F2C2ED9A4F10F05012DE5
:102FE00064D0A4F11103092B69D9092D5ED904EB32
:102FF000840304EB4303103CA9F1BB070126A51E83
:10300000092C1F4409D9082D45D90136163F6B1CE0
:103010002C460FD0A51E092CF5D89BF8013007F1DE
:103020000B00B3FBF6F303A98DF80D30FEF798FE05
:10303000002CE8D1D8F8044009F101090134B9F1B4
:103040000B0F48F8044FC4D1FEF792FCDAF80030B9
:103050000133CAF8003005B0BDE8F08F564B03F1DC
:103060006E0403E0A34203F8010C0ED013F8012B09
:1030700002F00201C9B242F0040022F00402002969
:10308000F0D1A34203F8012CF0D10420FFF742F85D
:1030900001232B60DFE79BF801303846B3FBF6F3E2
:1030A00003A98DF80D30FEF75BFEAEE705EB85005A
:1030B00005EB400048444149FEF752FE97E705EB17
:1030C000850005EB4000A9F11603C0183C49FEF746
:1030D00047FE8AE73B4ADFF8FC80176800261E603F
:1030E000394B2E603F243A4602A869461E601023E1
:1030F0008DF806308DF800408DF801408DF80540C0
:103100008DF802608DF80460FEF704FD3A4603A8CE
:1031100001A9FEF7FFFC2D4B9DF808709DF809C032
:103120009DF80AE09DF80C409DF80D009DF80E906A
:10313000224933F81770224A33F8144033F81CC080
:1031400033F81EE033F8100033F819300F7046F2F0
:103150006767147081F801C081F802E050709370C5
:103160003446C6F2666711E008F00CF987FB0032BE
:10317000C317C3EBA20303EB8303A0EB430048F8A0
:103180000600013404360B2C3FF409AFE207EBD400
:1031900008F0F8F887FB0032C317C3EBA20303EB78
:1031A0008303A0EB4300053048F80600E9E700BFC1
:1031B00020040020043E0020083E002038040020A7
:1031C000B4030020A8010020B0030020ACC3000815
:1031D0007C03002080030020704700BF074B0120C4
:1031E00003F16E0113F8012B12F0020214BF03F871
:1031F000010C03F8012C8B42F4D17047083E0020EB
:103200002DE9F84F9246814688460AB9BDE8F88F05
:103210000020FEF7BBFD1AF0080F40F095801AF071
:10322000100F40F08D80DFF87CB14146DBF80000E4
:10323000FEF7A2FB524A534B11784CF6CD42CCF626
:10324000CC42A2FB0802920801EBC101C90002EBCB
:10325000420201EB42021AF0040F02EB0301D05CC0
:10326000D4D0494A494F00249460D460146114605A
:1032700054615460148394763B4607F16E05012631
:1032800013F8014B14F0020414BF03F8016C03F8A7
:10329000014CAB42F4D1DBF80030002B62D03C4B48
:1032A0001B68DC0762D5012353709370002301254E
:1032B000CC180133A47814B1042B1555F8D1B9F109
:1032C0000B0F4B7888BFA9F10C099944B9F10B0F8A
:1032D00088BFA9F10C0900EB400009EB80092D4BD8
:1032E00013F8191003EB490329B15B7801205054FE
:1032F0000BB1254AD054284CDFF8ACC004F11B06B2
:10330000002514F8013F9BB105EB0C0315F80C20C8
:1033100098785B7860B102EB820102EB41021818E9
:10332000D219D15C41F00201D15401338342F8D16A
:103330000335B442E5D1194B01221A60BDE8F88F7C
:103340000120FEF79BFB6EE706F01AFDC820FEF792
:1033500075FA134B1B68002B7FF465AF0120FEF755
:103360006DFB60E71AF0100FE5D14FE7B8F1040FDD
:1033700099D9A8F11E08B8F1040F97D893E700BFB8
:10338000BC030020B4C4000824030020083E002031
:1033900048000020C8C600082303002020040020A5
:1033A000EC0300207001002074C6000840F24803BE
:1033B000C2F200031868704738B50B4B0B4D1B6801
:1033C000032B044604D0820702D52B689B0707D540
:1033D000FEF710FC064B2C6001221A60204638BD17
:1033E000FEF796FAF4E700BFEC0300204800002047
:1033F0002004002040F2EC33C2F20003186870474A
:10340000032810B509D8074C2368834203D02060F5
:10341000FEF7F0FB2368184610BD024B1B681846E8
:1034200010BD00BFEC03002040F27813C2F200038D
:10343000186870476328024B88BF64201860704783
:103440007801002040F29C13C2F200031868704714
:103450006228024B88BF0020186070479C01002042
:1034600040F2BC33C2F20003186870470328044BD3
:1034700004D81860034B01221A607047186870471F
:10348000BC03002020040020064B1868022805D940
:1034900000201860044B01221A6070470130186048
:1034A000F8E700BFBC03002020040020054B18688B
:1034B00028B101381860044B01221A6070470320BC
:1034C0001860F8E7BC0300202004002040F21443F9
:1034D000C2F2000318687047074B10B5186000B1BE
:1034E00010BD064B0F241C60FEF7CAFC044B1C6089
:1034F000BDE81040FEF752BB14040020A8010020D4
:10350000A001002040F2A413C2F200031868704723
:10351000024B0A288CBF186818607047A40100206D
:10352000044B1868092802D9002018607047013040
:1035300018607047A4010020044B186810B10138CE
:10354000186070470A201860704700BFA40100206F
:10355000064B1B68012B00D07047054B00223F2112
:1035600019705A709A70FEF78BBC00BFD40300200C
:103570006C01002040F2D433C2F200031868704797
:10358000012810B5034602D9054B186810BD044C3C
:103590002068984203D02360FFF7DAFF206810BD4F
:1035A000D4030020F0B5574B1B68012B83B00446B1
:1035B00041D0022B01D003B0F0BD20B9524B1A68A4
:1035C000002A78D018600020FEF758FA4F4B1B688D
:1035D0003B2B2DD81D2B71D967081E254C4A4D4B0E
:1035E00010785178927833F8100033F8111033F8CE
:1035F0001220454B8DF804001B688DF805108DF8DE
:103600000620002B45D1AF423CBF434E3C4605D37C
:1036100038E0723007F0C0FAAC4233D2306820187C
:103620000134A84201A9F4D33C386328F4D8F0E768
:1036300027463C25D2E70020FEF720FA334B1B68D3
:103640003B2B47D9344B1A683C23A418304AA34279
:1036500098BFC3EB040411782E4B9078557833F85B
:10366000111033F8152033F810308DF80410632C46
:103670008DF805208DF8063004D804F1720001A9F8
:1036800007F08AFA254B1B68002B94D0FEF7C0F98F
:1036900091E7214E002404E0723007F07DFABC422D
:1036A000F0D83368E0180134A84201A9F4D33C38BB
:1036B0006328F4D8F0E701221A6084E7132B7FF621
:1036C0007AAF4AF6AB27CAF6AA27A7FB04377F08CA
:1036D000142583E71D2B0ED8132B7FF66CAF0E4AF3
:1036E0004AF6AB23CAF6AA231268A3FB041402EB22
:1036F00054041423AAE7084B1A681E2302EB54044F
:10370000A4E700BFEC03002024040020780100207F
:1037100044000020ACC300089C0100207001002080
:1037200038B5814B1B680A2B1AD8804A804C126826
:103730007AB9804D2A68C2B97F49804A03EB830376
:1037400001EB83031168986801318142116045D211
:1037500038BD794A03EB830302EB83035B68984728
:10376000744B1B68002BF3D0714C754B1B68012BFD
:103770001FD0744B1B68032B06D02368002BE7D1A6
:10378000BDE8384006F01ABB6F4B70491A68496BA8
:103790000132B2EB411F1A60EFD36D490A68002075
:1037A000013A1860052A3AD8DFE802F059A19A9345
:1037B0008C50684B68491A6849690132B2EB411F65
:1037C0001A60D6D365490A680020013A1860052AB4
:1037D0000CD8DFE802F0625B544B70695B68002133
:1037E000116098472B68002BBED1B1E75C4A136883
:1037F0000133072B00F096805A48136002680B6073
:1038000001320D2A5549026000F083800E2AB0D1A2
:10381000013B08BF06230B6000230360A9E7524A5F
:1038200013680133072B72D05048136002680B6095
:1038300001320D2A4649026060D00E2A9DD1013B1B
:1038400008BF06230B600023036096E7484B9A7875
:10385000002AE4D0013A9A70FEF7A0F98DE7444BB4
:103860005A783E2ADBD801325A70F5E7414B5A7834
:10387000002ABBD0013A5A70FEF702FB79E73D4BB4
:103880009A783E2AB2D801329A70F5E7394B1A7805
:10389000002AABD0013A1A70EEE7364B5A783E2A2E
:1038A000A4D801325A70E7E7324B9A78002A9DD0AB
:1038B000013A9A70E0E72F4B1A783E2A96D80132E7
:1038C0001A70D9E72A4B1A783E2AA8D801321A7002
:1038D000C2E7274B5A78002AA1D0013A5A70BBE7B9
:1038E000234B9A783E2A9AD801329A70B4E7204B3B
:1038F0001A78002A93D0013A1A70ADE70133072BEA
:1039000018BF0B607FF439AF01230B6035E701234B
:103910008AE70133072B18BF0B607FF42AAF01231E
:103920000B6026E7012367E7A401002020040020A4
:1039300070010020043E002050000020F803002009
:10394000D4030020EC030020DC0300202C01002025
:103950007C030020680300207C010020000400207C
:10396000C80300203C00002028040020740100202F
:10397000400000206C010020064B1A783E2A07D830
:1039800003D13F221A70FEF77BBA02321A70FAE7AF
:10399000704700BF6C010020064A137843B1012B29
:1039A00003D100231370FEF76BBA023B1370FAE7E2
:1039B000704700BF6C010020064B5A783E2A07D89A
:1039C00003D13F225A70FEF75BBA02325A70FAE70F
:1039D000704700BF6C010020064A537843B1012BA9
:1039E00003D100235370FEF74BBA023B5370FAE742
:1039F000704700BF6C010020064B9A783E2A07D81A
:103A000003D13F229A70FEF73BBA02329A70FAE76E
:103A1000704700BF6C010020064A937843B1012B28
:103A200003D100239370FEF72BBA023B9370FAE7A1
:103A3000704700BF6C01002040F26C13C2F200031B
:103A40001A7802705A7842709B788370704700BF72
:103A500010B440F26C13047841788278C2F200030B
:103A60003F2C34BF20463F203F2928BF3F213F2A1B
:103A700028BF3F22187059709A7010BCFEF700BA28
:103A800040F24003C2F200031A7802705A78427082
:103A90009B788370704700BF10B440F240030478F5
:103AA00041788278C2F200033F2C34BF20463F2089
:103AB0003F2928BF3F213F2A28BF3F221870597055
:103AC0009A7010BCFEF76AB840F2A813C2F2000365
:103AD000186870470F2803D8034B1860FEF7D0B959
:103AE000014B0F221A60F9E7A8010020034B1A6866
:103AF00002B97047013A1A60FEF7C2B9A801002066
:103B0000044B1A680E2A00D9704701321A60FEF77A
:103B1000B7B900BFA801002040F2A013C2F2000311
:103B2000186870470F2803D8034B1860FEF736B8A3
:103B3000014B0F221A60F9E7A001002030B50125E2
:103B400083B015F0010F0CBF0021392115F0020FD1
:103B50000CBF0022392215F0040F0CBF00233923BB
:103B60008DF804108DF805208DF8063000242046CD
:103B700001A9013407F010F8D62CF8D1204606F040
:103B80006BFF01350320FDF767FE082DD9D100201A
:103B9000FEF7FCF803B030BD284B2DE9F04103F1EE
:103BA0006E01012413F8012B12F0020214BF03F876
:103BB000014C03F8012C8B42F4D1017800293AD052
:103BC00080460746013705260020C6F10502034658
:103BD000FEF736F898F8011059B30A2E18D83D466A
:103BE000344601E00A2C13D8002220461346FEF783
:103BF00027F815F8011F06340029F3D106E000224A
:103C00002046202113460634FEF71AF80A2CF6D96E
:103C10000420FEF77FFA3220FDF710FE013E02D0AD
:103C200017F8011CD0E718F8011F0029CAD1BDE818
:103C3000F0813446EAE7BDE8F08100BF083E00208D
:103C400070B51B4D2B6882B004460BB902B070BD35
:103C50004208184901A807F0E1FB0020FEF796F89A
:103C6000154B04F0010603F16E00012413F8012B3B
:103C700012F0020214BF03F8014C03F8012C834236
:103C8000F4D1002002469DF804100123FDF7D8FF6F
:103C90000022012306209DF80510FDF7D1FF2868BA
:103CA0007100FDF769FE054B01221A60CEE700BFE7
:103CB000700100202CC40008083E002020040020D1
:103CC0002DE9F04FB94B1B68044693B0184613B961
:103CD00013B0BDE8F08F3F268DF834603C260325F5
:103CE0008DF82360162600230CA92A46A4208DF8FF
:103CF00024600F268DF835308DF836308DF825305C
:103D00008DF826308DF82B308DF827508DF82960EE
:103D100000F0AEFB01220DF12101A72000F0A8FB6D
:103D200001220DF12501A82000F0A2FB01220AA921
:103D3000BD2000F09DFBBE2001220DF12A0100F004
:103D400097FBB4F5843F80F0A3809DF821809DF817
:103D500022C09DF825E09DF82610B8F1030F84BF1E
:103D60004FF000088DF82180BCF1030F84BF4FF0A5
:103D7000000C8DF822C0BEF10A0F84BF4FF0000E78
:103D80008DF825E0012902D900218DF826109DF833
:103D900028700F2F02D90F278DF828709DF8296001
:103DA0000F2E71D89DF82A00012802D000208DF82E
:103DB0002A009DF82320642A009203D964258DF8F7
:103DC000235000959DF82430632B02D916238DF8DB
:103DD0002430774C07932568764B01959DF8275042
:103DE0009DF834B002959DF830509DF835A00395AC
:103DF0009DF831509DF8369004959DF8325083F827
:103E000000B005959DF82B5083F801A0069540F26F
:103E1000BC35C2F2000583F80290C5F80080DFF8D7
:103E2000C081029DC8F800C0DFF8B8C1624BCCF871
:103E30000050DFF8B4C1614ACCF800E0DFF8ACE133
:103E40001F60CEF800105E4B0399049D11701E6038
:103E500005995C4B557091701860009A5A4B079DFC
:103E60001A605A4B06991D60594B19600023236054
:103E7000FDF794FEFEF704F8019A2260FFF768FB55
:103E8000FDF7B8FE012023E70F268DF8296089E7AA
:103E9000A92001220DF1260100F0EAFA40F6FF0305
:103EA000C0F201039C427FF650AF01220DF12701C1
:103EB000BC2000F0DDFA0DA92A46D72000F0D8FA80
:103EC00001220DF12901DA2000F0D2FADB200122D3
:103ED0000DF1220100F0CCFAB4F5003FFFF435AF4C
:103EE00001220DF12301DC2000F0C2FADD200122C5
:103EF00009A900F0BDFAFF23C0F202039C427FF63D
:103F000024AF0DF12B010122E02000F0B1FA0FA93E
:103F10000B22E52000F0ACFA0EAE0BA9022240F213
:103F2000251000F0A5FA40F235103146042200F0C9
:103F30009FFA0DF14605274B0DF13B0005E042F0DD
:103F400002021A611433A84212D010F8012FFF2A7E
:103F5000F8D002F01001C9B202F00F029A601A699B
:103F60000029ECD122F002021A611433A842ECD1EC
:103F70009DF82C301848FF2B1EBF184A03F00F0382
:103F800053609DF82D30FF2B1EBF144A03F00F0322
:103F900053610023F25CFF2A1EBF00EB031102F005
:103FA0000F024A600133042BF4D1CEE65C040020FA
:103FB0007001002040000020A80100206C010020BA
:103FC000A001002014040020780100209C010020A2
:103FD00004040020500000202C0100207C0100205F
:103FE000EC03002048000020A4010020D40300209E
:103FF0002DE9F04F854B1B68A3B0002B00F08B80A0
:10400000834B844A93F8008093F801C093F802E050
:10401000814B92F800B01F68804B92F801A01E6897
:104020007F4B92F802901D687E4B8DF819501C68EA
:104030007D4B8DF81A401B688DF820B000937B4BA8
:10404000009C1B688DF81B400193794B019C1B68F9
:104050008DF821A00293774B8DF822901B688DF884
:1040600024800393744B8DF825C01868734B8DF82A
:1040700026E01968724B8DF815701A688DF8166075
:104080008DF81C40029C6F4B8DF81D40039C8DF8F1
:1040900017008DF81E408DF8181000208DF81F2095
:1040A00012ACFF250A2888BF255409D89A681969D7
:1040B00002F00F028907225444BF42F0100222543A
:1040C000013014334028EDD15F4800230AAEFF22AF
:1040D000012B97BF00EB0311F254496801F00F0167
:1040E00098BFF1540133102BF2D1584900230EAD83
:1040F000FF2001EB0312032B97BF5268E85402F034
:104100000F02EA540133102BF3D1A42008A9032293
:1041100000F0C8F918B9002023B0BDE8F08FA7203F
:104120000DF11501012200F0BDF90028F3D0BC20EB
:104130000DF11901012200F0B5F90028EBD0A820FB
:104140000DF11A01012200F0ADF90028E3D0A920F9
:104150000DF11B01012200F0A5F90028DBD0BD20E4
:1041600007A9012200F09EF90028D4D0BE200DF14D
:104170001E01012200F096F90028CCD0D72009A911
:10418000032200F08FF90028C5D0DA200DF11D01BF
:10419000012200F087F90028BDD0DB200DF11601C7
:1041A000012200F07FF90028B5D0DC200DF11701C5
:1041B000012200F077F90028ADD0DD2006A9012208
:1041C00000F070F90028A6D0E0200DF11F010122B7
:1041D00000F068F900289ED0E5202146402200F03A
:1041E00061F9002897D040F225103146102200F0E6
:1041F00059F900288FD0102240F23510294600F0DE
:1042000051F9003018BF012086E700BF5C04002090
:10421000400000206C010020BC030020EC030020C3
:1042200048000020A4010020D4030020A8010020A1
:10423000A001002014040020780100209C0100202F
:1042400004040020500000207C0100202C010020EC
:1042500006F0CEBC2DE9F84381468846174605F0A6
:104260004BFC10B90020BDE8F883552005F0DCFCBC
:104270002E48082105F000FD442005F0D5FC00245F
:1042800043F2144505F09AFC0134AC4298BF002873
:1042900014BF00260126F5D043F214439C4227D8D0
:1042A00005F02AFC0028DDD0552005F0BDFC204C8F
:1042B0001E48082105F0E0FCBE2005F0B5FC0921F0
:1042C000204605F0A3FC05F017FC1A4B1B68222BB7
:1042D00013D0282B11D00923C9F8003094F90130EC
:1042E000DB0FC8F80030237801203B60BDE8F8837D
:1042F00005F002FC3046BDE8F88323796278257822
:10430000C3F34113093302F00704C3F10C00191F72
:1043100045FA00F004FA01F10143D209C9F800306E
:104320000120C8F800203960BDE8F883500400205F
:104330003C0400204C040020F8B5A0F10905032D31
:10434000044602D900263046F8BD05F0C5FC05F04C
:10435000D3FB0028F6D02E4F384605F09BFC3B7867
:104360002C4A13602C4A0121222B0646116001D0F1
:10437000282BE8D105F0C0FB0028E4D0552005F03B
:1043800053FC264F2248082105F076FCBE2005F09C
:104390004BFC0921384605F039FC3B79C3F3411346
:1043A0000933A342CFD005F0A7FB0028CBD055207E
:1043B00005F03AFC0821164805F05EFC4E2005F099
:1043C00033FC7F2005F030FC802005F02DFC6801D7
:1043D00000F0E00005F028FC05F08EFB05F08CFBFA
:1043E0000028B0D0552005F01FFC0948082105F031
:1043F00043FC482005F018FC002405F0DFFB0134E5
:10440000F92C98BF0028F8D005F076FB9BE700BF99
:10441000500400204C040020480400203C040020EC
:104420002DE9F04184B003F03FF8DFF8408000242C
:104430000127650045F0A0050126009728460021C8
:1044400032460DF10F03A419C8F8005003F080F8AC
:1044500030B1082CEDD1044B186804B0BDE8F081F0
:10446000014B30461E60F8E75C0400205804002031
:1044700010B50A4B1C6882B00B4614B9204602B036
:1044800010BD0092064A126801461046012203F050
:104490005FF8D0F1010038BF0020F0E75C04002095
:1044A000580400202DE9F047144B1B6882B01746D2
:1044B00003B3EAB1DFF84CA0114C0646C0EB01098A
:1044C0004FF001080025DAF80000CDF800803146F1
:1044D000012209EB060303F0B9F858B9102023684C
:1044E000002BFCD001382560F9D10136013FEAD11B
:1044F000012000E0002002B0BDE8F0875C0400204D
:10450000783E00205804002070B53E4B1A68824265
:1045100088B0064674D002A81E60FCF79BF904A878
:10452000FCF7DEFC01200146FCF742FB01200146BE
:10453000FCF73EFB20200121FCF756FB0020C4F2D3
:1045400002000B210822FCF79BF900200822C4F28C
:1045500002000C21FCF794F9022300208DF80C30A6
:10456000032304460125C4F2020002A98DF80D3090
:104570004FF4006302938DF80E408DF80F50FCF756
:104580000DF920464FF48053C4F2020002A90293B1
:10459000FCF704F94FF4A050C4F201002946FCF7DF
:1045A000B9FC4FF4A0500C23C4F2010004A9ADF8EB
:1045B0001A300496ADF81440ADF81640ADF8184026
:1045C000ADF81C40FCF720FC4FF4A050C4F20100F1
:1045D0002946FCF791FC4FF4A050C4F2010040F2D0
:1045E00025512A46FCF7ACFC472301A88DF804307E
:1045F0008DF805408DF806408DF80750FBF728FE32
:1046000008B070BD7806002030B40F4A13687F2BC5
:10461000FCD80E490E4D0B685C1C7F2C45F823001E
:1046200098BF0C6001D900230B6072B61368013388
:10463000136062B64FF4A050C4F2010040F227713B
:10464000012230BCFCF77CBC740600207006002000
:104650006804002010B50446007828B1FFF7D4FFA5
:1046600014F8010F0028F9D110BD00BF40F26443D7
:10467000C2F200031868003018BF0120704700BF65
:1046800030B40D4B1A6882B10C490D4D0A68541CA8
:10469000802C55F8225018BF0C6009D072B61A68E9
:1046A000013A1A6062B601220560104630BC7047BC
:1046B00000220A60F2E700BF6404002060040020CA
:1046C0007C060020024A1368002BFCD1704700BF13
:1046D000740600204FF4A05038B5C4F2010040F237
:1046E0002551FCF749FC00282BD14FF4A050C4F20F
:1046F000010040F22771FCF73FFC00B938BD4FF4D0
:10470000A050C4F2010040F22771FCF75BFC234B80
:104710001A68002A38D0224A224C1168481C802886
:1047200008BF002054F8211010601A684FF4A05000
:10473000013AC4F2010089B21A60BDE83840FCF7C2
:10474000F7BB4FF4A050C4F2010040F22551FCF732
:1047500039FC4FF4A050C4F20100FCF7EDFB124B02
:104760001A687F2AC1D81149114D0A68541CC0B279
:104770007F2C45F8220098BF0C6001D900220A6006
:104780001A6801321A60B0E74FF4A050C4F2010079
:1047900040F22771BDE83840FCF7D2BB7406002018
:1047A0006806002068040020640400206C060020D5
:1047B0007C0600202DE9F04383B06846FCF74AF8F8
:1047C00000260120C4F2020601460124FCF7F0F99C
:1047D00000254FF0800930466946CDF800908DF8ED
:1047E00005508DF804408DF806508DF80750FBF702
:1047F000D5FF20462146FCF7DBF94FF04008304654
:104800006946CDF800808DF805508DF804408DF88C
:1048100006508DF80750FBF7C1FF20462146FCF7F4
:10482000C7F910273046694600978DF805508DF876
:1048300004408DF806508DF80750FBF7AFFF304667
:1048400049462246FCF716F8304641462246FCF718
:1048500011F8304639462246FCF70CF803B0BDE8A3
:10486000F08300BFF8B5094D04460F46002601E06D
:104870002B6833B92046FFF703FF0028F8D001204A
:10488000F8BD0136BE422860F4D3F8BD7C3E00205E
:104890002DE9F04F85B0054603F02AFDFFF712FF22
:1048A000FFF7E4FE002843D00024624FDFF888A120
:1048B0000126A346294603A8FFF7D4FFDFF8749129
:1048C0004FF001080346002835D0039B3E600A2BB9
:1048D00007D00D2BEED0FF2CECD80AF804300134B1
:1048E000E8E70AF804B0002C32D103F001FDE1E75B
:1048F000514852491A4606F0DCFD00284CD04E487B
:104900004F49032206F0D5FD00284FD04A484D49B3
:10491000052206F0CEFD002855D14B484B49022216
:1049200006F0C7FD002849D10123C9F80830062048
:1049300005B0BDE8F08F4648019303F0ABFC454855
:1049400003F0A8FC444803F0A5FC019B1846EFE7E0
:104950003F48019303F09EFC374803F09BFC3E4820
:1049600003F098FC34483D49022206F0A2FD38B11C
:1049700031483B49052206F09CFD18B90220D7E7D3
:104980004046D5E72C483749022206F092FD019BAC
:104990000028ADD10320CBE709F13C0032490F22BA
:1049A00006F0A0FDC9F804800420C1E709F11C004D
:1049B0002E491F2206F096FD0520B9E70023C9F80D
:1049C00008300620B4E71C482949052206F071FD8D
:1049D00098B119482749092206F06BFD10B3164813
:1049E0002549042206F065FDA8B113482349092290
:1049F00006F05FFD40B1FF209AE7214812490F22DF
:104A000006F070FD072093E71E481F49FF2206F0BD
:104A100069FD0A208CE71D481D491F2206F062FD32
:104A2000092085E71B4818490F2206F05BFD082086
:104A30007EE700BF7C080020F809002018C70008A6
:104A400024C7000828C70008FD09002030C7000857
:104A5000F8C60008FCC6000804C7000808C700081C
:104A60000CC7000814C70008020A0020FB09002038
:104A700034C700083CC7000848C7000850C70008F2
:104A8000E8090020C8080020010A0020C809002009
:104A9000FC09002088080020F0B583B0074606F026
:104AA00000FD06461A4803F0F5FBBEB13C46F61978
:104AB00004E0184603F0C8FBB4420FD014F8013BE1
:104AC0001449A3F120055E2D68461A46F1D906F077
:104AD000A5FC684603F0DEFBB442EFD10E4803F0BC
:104AE000D9FB03F005FC3846FFF7B4FD0B48FFF790
:104AF000B1FDFFF7E7FD02E0022807D020B10A2050
:104B0000FFF7C6FE0128F7D103B0F0BD0020FBE798
:104B10005CC7000870C7000864C7000838C90008EF
:104B200038B539B10446451814F8010BFFF76CFD90
:104B3000AC42F9D1BDE83840FFF7C4BD40F67C0077
:104B4000C2F20000704700BF10B50020C4F202009E
:104B50008021002282B0FBF78DFE0C4A052114460D
:104B600000201368002BFCD001392060F9D100200F
:104B7000C4F2020080210122FBF77CFE01A8322151
:104B8000FFF770FE0028F9D102B010BD7C3E002076
:104B900008B502460B460748074906F03FFC0548A2
:104BA000FFF77AFF20B1054B002283F83C205A60C2
:104BB00008BD00BFFC0A002078C700087C08002060
:104BC00008B502460B460748074906F027FC05488A
:104BD000FFF762FF20B1054B002283F83C205A60AA
:104BE00008BD00BFFC0A002088C700087C08002020
:104BF00008B5024608B1037823B90748BDE8084064
:104C0000FFF74ABF0549064806F008FC0448BDE81E
:104C10000840FFF741BF00BFB4CD000898C70008A7
:104C2000FC0A002030B54FF4E13083B003F0FAFB0A
:104C3000FFF7C0FD4FF4E130FFF766FC0020C4F23F
:104C4000020010210022FBF715FE1E4C002000225E
:104C5000C4F202008021FBF70DFE05252246002349
:104C600021680029FCD0013D1360F9D1002080218A
:104C70000122C4F20200FBF7FDFD12493222236833
:104C8000002BFCD0013A0D60F9D10020C4F20200E3
:104C900010210122FBF7EEFD03E001A803F006FB63
:104CA00060B901A8FFF7ECFC0028F6D0019803F0EA
:104CB000CBFA01A803F0FAFA0028F2D00198FFF726
:104CC000A3FCEEE77C3E002008B50B4B1A6802B14E
:104CD00008BD01224FF4E1301A6003F0A3FB07483E
:104CE00003F0D8FAFFF766FD4FF4E130FFF70CFC54
:104CF000BDE80840FFF728BF4C0B0020A4C7000800
:104D000010B403781649FBB1002208601446013044
:104D100005E001300E2A14DC10F8013C8BB13D2B6C
:104D200002BF01EBC20300F8014C5860F1D0262B02
:104D3000EFD1013200F8014C41F8320001300E2A67
:104D4000EADD531C0F2B08DC002201EBC3001146E7
:104D50000133815008320F2BFADD10BC704700BFC1
:104D60008C0B0020F8B50A4D0646002455F8343067
:104D7000E70031461846013423B106F080FB18B134
:104D8000102CF3D10348F8BD014BDF197868F8BD4A
:104D90008C0B0020C0C8000808B5FFF7E3FF4CF6F5
:104DA0009C01C0F6000106F06AFBD0F1010038BF9B
:104DB000002008BD00B50B4685B04CF6A4010246A4
:104DC000C0F60001684606F029FB6846FFF7CAFFF7
:104DD00005B000BD10B5044606F063FB014600B9FE
:104DE00010BD2046BDE81040FFF79ABE10B504463E
:104DF0004CF6AC00C0F60000FFF7ECFF4CF6BC0030
:104E0000C0F60000FFF7E6FF4CF6C400C0F6000055
:104E1000FFF7E0FF4CF6D000C0F60000FFF7DAFF26
:104E20004CF6DC00C0F60000FFF7D4FF2046FFF789
:104E3000D1FF4CF6E400C0F60000FFF7CBFF4CF6C4
:104E4000F000C0F60000FFF7C5FF4CF6FC00C0F60E
:104E50000000FFF7BFFF4CF60810C0F60000FFF798
:104E6000B9FF2046FFF7B6FF4CF61010C0F6000061
:104E7000BDE81040FFF7AEBF38B504464CF6181039
:104E8000C0F600000D46FFF7A5FF2046FFF7A2FF82
:104E90004CF62410C0F60000FFF79CFF2846FFF7F1
:104EA00099FF4CF62810C0F60000BDE83840FFF727
:104EB00091BF00BF4CF6C0004CF63C1108B5C0F6DF
:104EC0000000C0F60001FFF7D7FF4CF644104CF687
:104ED0004C11C0F60000C0F60001FFF7CDFF4DF207
:104EE00058104CF65411C0F60000C0F60001FFF750
:104EF000C3FF4CF660104CF66411C0F60000C0F61B
:104F00000001FFF7B9FF4DF2D0204CF66811C0F652
:104F10000000C0F60001FFF7AFFF4CF670104CF632
:104F20007C11C0F60000C0F60001FFF7A5FF4CF6AB
:104F300088104CF69411C0F60000C0F60001FFF78F
:104F40009BFF4CF6A0104CF6A811C0F60000C0F66E
:104F50000001FFF791FF4CF6B010C0F60000BDE86D
:104F60000840FFF737BF00BF054A136801331360DD
:104F7000DB0702D40348FFF72DBF0348FFF72ABF22
:104F8000300C0020CCC90008B4C9000810B5044694
:104F90004CF6D410C0F60000FFF71CFF2046FFF7C8
:104FA00019FF4CF6DC10C0F60000BDE81040FFF71A
:104FB00011BF00BF70B584B00C4605461B491646AC
:104FC00068461A4606F02AFA02A81849089A06F016
:104FD00025FA3CB123782BB12046FFF7FBFE14489D
:104FE000FFF7F8FE1348FFF7F5FE2846FFF7F2FE3D
:104FF0001148FFF7EFFE2846FFF7ECFE0F48FFF7DA
:10500000E9FE3046FFF7E6FE0D48FFF7E3FE68468F
:10501000FFF7E0FE0B48FFF7DDFE02A8FFF7DAFE20
:105020000948FFF7D7FE04B070BD00BFECD40008FC
:1050300084D00008E4C90008FCC9000808CA0008B8
:1050400014CA000824CA000824C9000810B5044680
:105050004CF63020C0F60000FFF7BCFE2046FFF7FC
:10506000B9FE4CF66420C0F60000FFF7B3FE4CF624
:105070007420C0F60000BDE81040FFF7ABBE00BFD3
:1050800070B505460F480E46FFF7A4FE0E48FFF721
:10509000A1FE002E0EDD043D00240C48FFF79AFE11
:1050A00055F8040FFFF796FE01340948FFF792FE0A
:1050B000B442F2D10748FFF78DFE074B00221A6079
:1050C00070BD00BF7CCA0008CCC9000898CA00089F
:1050D000B0CA000890CA0008300C00204CF6C0206E
:1050E000C0F60000FFF776BE38B504464CF6D02077
:1050F000C0F600000D46FFF76DFE2046FFF76AFE82
:105100004CF62410C0F60000FFF764FE2846FFF7B7
:1051100061FE4CF6FC20C0F60000BDE83840FFF709
:1051200059BE00BF08B54CF60C30C0F60000FFF7C2
:1051300051FE4CF61830C0F60000BDE80840FFF7FD
:1051400049BE00BFF0B5044683B01F481E460D4659
:105150001746FFF73FFE2046FFF73CFE1B48FFF7D0
:1051600039FE2046FFF736FE1948FFF733FE002EC2
:1051700024DD043D00240BE01648FFF72BFE55F814
:10518000040FFFF727FE1448FFF724FEB44215D0A2
:105190002246124901A806F041F91148FFF71AFE0C
:1051A00001A8FFF717FE0F48FFF714FEBC4204F1F9
:1051B0000104E1D10C48FFF70DFEDDE70B48FFF7D6
:1051C00009FE03B0F0BD00BF24CB0008FCC90008F5
:1051D00034CB000830CC000864CB0008ECD40008C5
:1051E00048CB000810CA000858CB00083CCB000888
:1051F00070B50E4605460E481446FFF7EBFD3046E7
:10520000FFF7E8FD0B48FFF7E5FD2846FFF7E2FD55
:105210000948FFF7DFFD14B10848FFF7DBFD084838
:10522000FFF7D8FD0748BDE87040FFF7D3BD00BFCA
:10523000D4C9000870CB000894CB0008A8CB0008A4
:1052400030CC0008DCC900082DE9F041069F079D1D
:1052500004461646984611B10B78002B49D12848D0
:10526000FFF7B8FD2046FFF7B5FD2648FFF7B2FD72
:105270002046FFF7AFFD2448FFF7ACFD3046FFF7AF
:10528000A9FD2248FFF7A6FD4046FFF7A3FD2048F1
:10529000FFF7A0FD3846FFF79DFD55B12B7843B1D0
:1052A0001C48FFF797FD2846FFF794FD1A48FFF7C3
:1052B00091FD1A48FFF78EFD2046FFF78BFD184839
:1052C000FFF788FD2046FFF785FD1648FFF782FDB2
:1052D0001548FFF77FFD2046FFF77CFD1348FFF7D9
:1052E00079FD3046FFF776FD1148BDE8F041FFF744
:1052F00071BD0846FFF76EFD0E48FFF76BFDAEE788
:10530000B0CB0008FCC9000808CA0008CCCB0008D4
:10531000D4CB0008DCCB0008ECCB0008F0CB0008B5
:10532000FCCB00080CCC000818CC000828CC0008E6
:1053300034CC000884D000084CF64040C0F6000091
:105340000321FFF7EDBB00BF10B504464CF6D410A7
:10535000C0F60000FFF73EFD4CF644412046C0F683
:105360000001FFF7C1FE4CF67420C0F60000BDE856
:105370001040FFF72FBD00BF70B506464CF6D410A5
:1053800082B0C0F600000D461446FFF723FD4CF630
:10539000C0014CF64C43C0F60001C0F60003304695
:1053A000009301912A462346FFF74EFF4CF67420E6
:1053B000C0F6000002B0BDE87040FFF70BBD00BFB3
:1053C00038B505460C46FFF7CFFD2846FFF7DEFD52
:1053D0002046FFF7DBFD4CF6C000C0F60000FFF7EB
:1053E000D5FD4CF69020C0F60000BDE83840FFF730
:1053F000F1BC00BF10B504464CF65040C0F60000AA
:10540000FFF7E8FC2046FFF7E5FC4CF63430C0F629
:105410000000BDE81040FFF7DDBC00BF10B504463A
:10542000FFF7A2FD2046BDE81040FFF7E3BF00BF35
:105430004CF67040C0F60000FFF7CCBC08B5FFF793
:10544000F7FF4CF69020C0F60000BDE80840FFF7DB
:10545000C1BC00BFF0B583B00E4614461F46089D80
:10546000FFF7DCFF3046FFF791FD4CF6D410C0F695
:105470000000FFF7AFFC4CF6C001C0F600013A4651
:105480002B4620460095FFF795FD4CF6DC10C0F644
:105490000000FFF79FFC2046FFF7D8FD03B0BDE8F2
:1054A000F040FFF7CBBF00BFF8B5069D0E4614468F
:1054B0001F46FFF7B3FF3046FFF768FD2046394629
:1054C0002A46FFF795FE2046FFF7C0FDBDE8F840ED
:1054D000FFF7B4BF2DE9F0410F4614469846069EEB
:1054E000079DFFF79BFF3846FFF750FD4CF6D410A1
:1054F000C0F60000FFF76EFC414632462B462046C0
:10550000FFF720FE4CF6DC10C0F60000FFF762FC4F
:105510002046FFF79BFDBDE8F041FFF78FBF00BFBE
:105520002DE9F04F83B08B4692469946DDF83080E6
:105530000D9F124EFFF772FF1148FFF727FD11482C
:10554000FFF748FC00243D595BF804005AF80410AA
:1055500059F8042058F804308DE86000FFF774FE15
:1055600004340948FFF736FC0C2CECD10748FFF750
:105570006DFD03B0BDE8F04FFFF760BF8CCC0008B5
:105580007CCC000884CC000890CC000838D30008FC
:105590002DE9F04F05460E46C7B0A8482946924669
:1055A00002F030FF33781BB3741C4FF02008002743
:1055B00006E02B2B08BF04F8018C14F8013BBBB1AB
:1055C000252BF6D120460221FBF7C4FDA27804F872
:1055D000010C002A00F04185234603F8012B9A783C
:1055E0001946002AF9D10F7014F8013B002BE7D1BE
:1055F0003146934802F006FF3046FFF781FB28460C
:10560000904905F03CFF002842D028468E4905F01D
:1056100036FF0446002800F0CD8328468B4905F06C
:105620002EFF002800F071842846894905F027FFE5
:105630000446002800F095812846864905F01FFFA2
:10564000002800F06B852846834905F018FF0028E4
:1056500000F0EE872846814905F011FF002800F090
:105660004F8228467E4905F00AFF002800F0048793
:105670007C48FFF7AFFB7C48FFF7ACFB7B48FFF7AC
:10568000A9FB0026FFF758FE304647B0BDE8F08F73
:10569000774C94E803001AAD04F1080685E803008E
:1056A0000FCE3EAF07953D460FC596E80300059720
:1056B00004F1200785E803000FCF25AD04F1340E77
:1056C0002E460FC6BEE80F003F68089504F1480C4F
:1056D0002AAD069537600FC5BCE80F002FAF4834E0
:1056E0003E460FC60FCC0DF1D00844460FC4DCF87F
:1056F0000030DEF800203360236015A914A81CAC2C
:105700000DF1600913AE0DF1580B2A603C9109941C
:10571000CDF8E4903A963B90CDF8F4B002F0C4FF97
:105720000A9002F0C7FF5349C0F30742C0F30723B2
:10573000099805F073FE02F0C3FF4269002A04468F
:1057400032DB0369002B2FDBC16800292CDB80686A
:10575000002829DB6568002D26DBB2F5966F23DC77
:105760000C2B21DC1F291FDC17281DDC3B2D1BDC2B
:1057700002F26C724846404905F050FE22693F49EA
:105780000132304605F04AFEE2683C4914A805F0B3
:1057900045FEA268394915A805F040FE584637492C
:1057A000626805F03BFE0AE000238DF860308DF85A
:1057B0004C308DF850308DF854308DF858303048DA
:1057C000FFF7D0FA0546002801F08A802D4905F040
:1057D00056FE002841F04B802B4C49262B48DFF821
:1057E000C4A0FFF703FBFFF765FB07980221FFF753
:1057F00047FC27480A99FFF7E3FDDAF80030254A0D
:1058000025492648002B18BF1146FFF7D9FDDAF8C5
:105810000030002B41F02580FFF760FC0598062141
:10582000FFF72EFC1E48FFF7F9FD4FF0000A09951F
:105830000594089DDDF818B039E000BF24CE0008BB
:1058400038CE000850CE000878CF0008ECD0000811
:10585000D0D1000854D200088CD3000848D40008E6
:10586000F0D400083CD50008BCC8000854D5000896
:10587000B8C7000854CE000860CE000864CE000807
:105880006CCE000874CE0008A8CC0008C4CE000876
:10589000D0CE000858DD0008F8CC0008D8CE0008AB
:1058A000C0C800085C04002039AB5AF80390754862
:1058B000FFF790FA58F80A4055F80A005BF80A100A
:1058C00057F80A3000944A46FFF774FB0AF1040ABD
:1058D0006D48FFF77FFABAF1140FE5D16B48059CCC
:1058E000099DFFF7B3FBFFF7A9FDFFF7F7FB07984B
:1058F0000221FFF7C5FB6648664A67491E27034633
:105900000097FFF7A7FDFFF7E9FB6148FFF772FD7E
:1059100062486349FFF7E8FB62486349FFF7E4FB2D
:1059200062486349FFF7E0FB62486349FFF7DCFB2D
:10593000FFF77EFD44B16148FFF74CFA2046FFF7C0
:1059400049FA5F48FFF746FA28465A4905F097FD9D
:105950000446002800F0E084FFF7E4FBFFF7ECFCCE
:1059600092E6584B93E803003EAD85E803000595A9
:10597000FDF7ACFD80465448FFF7F4F905460028D2
:1059800001F00282514905F07AFD0646002801F037
:10599000498128464E4905F072FD0646002801F06F
:1059A0001F8028464B4905F06AFD0546002841F056
:1059B000E7814948FFF7F0F910F1000818BF4FF0F0
:1059C0000108CAF800804C2600238DF8BC300A2458
:1059D000FBF75AFB0DF13A00FBF764FB002841F09E
:1059E0000B810A20FBF72AFF013CF3D146AF3F238E
:1059F00027F85C3D02F074FA384982B234A805F009
:105A00000DFD02F073FA354982B239A805F006FDA2
:105A10003348FFF7EBF9FFF74DFA05980221FFF73E
:105A20002FFB30483946FFF7CBFC2F4834A9FFF74E
:105A3000C7FC2E4839A9FFF7C3FC274A2C4B29493C
:105A40002C48CDF80080FFF72FFDFFF747FB2948D2
:105A5000FFF7D0FC1D482849FFF746FB1C482749A3
:105A6000FFF742FBFFF7E4FC002D3FF475AF13484E
:105A7000FFF7B0F92846FFF7ADF91148FFF7AAF98B
:105A80006AE700BFD4C90008DCC9000894CE00084A
:105A9000C0C80008BCCE0008F0CE00087CCE0008CC
:105AA000F8CE000884CE000804CF000874CE0008A9
:105AB00010CF000828CF000834CF000840CF0008DE
:105AC000E0D00008B8C700086CCE0008D8D10008A4
:105AD000E0D10008E8D10008ECD100082CC400088F
:105AE000F4D1000864C9000804D2000808D20008F4
:105AF0000CD2000860C9000824D200083CD200087B
:105B0000914E924D96E8070006F1500320AC84E8D0
:105B100007000FCB3EAF06F10C0E87E80F009EE8A2
:105B2000070025AB08930597089F06F1180387E83F
:105B3000070093E807002AAB0693069F06F12403AB
:105B400087E8070093E807000DF1D008303688E8B1
:105B5000070096E807002B687D4F0DF1E40989E8FE
:105B600007004BB97B4E3B6A39683A69386B86E867
:105B70000E000123F0602B60FDF73CFC0790FDF761
:105B800053FC0A90FDF75EFC0B90FDF70FFC00F054
:105B900002000C90FDF7C0FF0990FDF797FC0D90F7
:105BA0000FA8FDF76DFF6C48FFF7DCF805460028ED
:105BB00000F01B87694905F062FC8346002801F06C
:105BC0008D802846664905F05AFC8346002801F07E
:105BD00005812846634905F052FC8346002801F000
:105BE000C3812846604905F04AFC0646002801F0BA
:105BF000578328465D4905F042FC0646002801F01F
:105C0000F88228465A49072205F053FC0646002828
:105C100001F0E68228465749042205F04AFC064670
:105C2000002801F05A832846534905F028FC002635
:105C3000B34610B9DFF878B153267A6B4F4915A8EF
:105C400005F0ECFB4D490A9A16A805F0E7FB4B4915
:105C50000B9A18A805F0E2FB11AD4849099A10A863
:105C600005F0DCFB0DF1480A44499DF83C2028462C
:105C700005F0D4FB13AF41499DF83D20504605F097
:105C8000CDFB9DF83E203D49384605F0C7FB3C481A
:105C90002F950325CDF8C0A03197FFF7A7F8FFF7A0
:105CA00009F920462946FFF7EBF936483649374AC5
:105CB000009516ABFFF7CEFB009532483449354AC4
:105CC00018ABFFF7C7FB0C9C5CB90D9D002D01F0D4
:105CD00025818DE800032B480899069A2FABFFF722
:105CE0001FFC079F2C4A1B4B26482C490097042475
:105CF0000194FFF7EFFBFFF7F1F921460598284DD6
:105D0000FFF7BEF900242B68DA0700F19A86013408
:105D10001035042CF7D1FFF7E1F91A48FFF76AFBB9
:105D200015482049FFF7E0F9FFF782FBBBF1000FB0
:105D30003FF412AE1C48FFF74DF85846FFF74AF8FB
:105D40001A48FFF747F807E61CC80008100C0020A7
:105D50002C010020180C00206CCE00087CD200081A
:105D60008CD2000854D4000864D4000874D400080D
:105D700084D4000894D40008D8D20008ECD40008D9
:105D80009CD4000888C90008B0D4000868D4000872
:105D9000B8D4000878D4000858D40008D0D400083B
:105DA0003801002080D3000840CF0008E0D0000870
:105DB00004CE0008AB4B93E803000DF1E40908336F
:105DC00089E8030093E807003EAD85E807000595E4
:105DD000FEF7B4FE0546A448AF68FEF7C3FF05F121
:105DE0000C088246002800F0F487A04905F047FB24
:105DF0000646002800F0508650469D4905F03FFBBE
:105E00000646002800F0018750469A4905F037FB06
:105E10000646002800F018875046974905F02FFBEA
:105E2000002800F061852646B24604F06BFD9349D8
:105E3000024634A805F0F2FA9148FEF7D7FFFFF7C3
:105E400039F805980321FFF71BF98E4805F13C014D
:105E5000FFF7B6FA41468C48FFF7B2FA8B48FFF7D6
:105E6000DDFA8B48FFF792F88A48FEF7B3FF4FF050
:105E70000F08894849463A460223FFF763F98749E4
:105E80008748CDF8008005F11C022023FFF792F827
:105E90008448FEF79FFF14238349844A8448009373
:105EA0004023FFF787F88348FEF794FF8248FFF707
:105EB000CDF8FFF7C3FA04F047FD8049804ACDF8DA
:105EC000008003467148FFF7C5FA03237D497E4AE7
:105ED0006E48009334ABFFF7BDFAFFF7FFF86B484D
:105EE000FFF788FA64487949FFF7FEF8FFF7A0FA50
:105EF000002C00F002827648FEF76CFF2046FEF789
:105F000069FF7448FEF766FF26E5734B93E80300CC
:105F10000DF1D00888E803005348FEF723FF04463C
:105F2000002800F0F4846D4905F0A9FA064600281F
:105F300000F0588620466A4905F0A1FA0646002876
:105F400000F0AF862046674905F099FA002840F036
:105F5000DE84654D5726654B1B68002B00F0688575
:105F600004F076FA0DF1E409044662084846434914
:105F700005F054FAE70700F1BC86484605F091FAAF
:105F80005B4B09EB000201469C8818689B7949F835
:105F9000010094809371574B1B68002B00F03F85E4
:105FA00004F0ECFB3EAF04466208384633490597DF
:105FB00005F034FAE40700F1A986059805F071FAB6
:105FC000059C4B4B059F221801469C8818689B79BD
:105FD00078509480937104F02BFA0246002840F028
:105FE0007D8546AF07F85C0D04F018FC02460028DA
:105FF00040F06C8546AC04F8700D06943E48FEF700
:10600000F5FEFEF757FF40460221FFF739F83B48FF
:106010004946FFF7D5F9022439480599FFF7D0F929
:1060200038483949394A00943B46FFF713FA384952
:10603000384A069B33480094FFF70CFAFFF74EF8F6
:106040003048FFF7D7F927483349FFF74DF8FFF7F6
:10605000EFF9002D7FF40BAD7EE421460F70FFF7C2
:10606000C3BA00BF14C800086CCE000884CF000873
:1060700020D0000830D0000840D00008ECD4000840
:10608000A4CF000848D0000854D0000844C9000834
:1060900068D00008D4C9000890CF000870D000086C
:1060A0009CCF000878D000088CD00008C0C8000839
:1060B00064DE0008DCC9000888CF000890D0000822
:1060C00024D000089CD0000834D00008B0D00008CC
:1060D000C0D00008DCD00008B8C70008FCD0000819
:1060E0000CD100081CD10008BCCD0008D41200203F
:1060F00034D10008480400203CD1000854D10008E5
:1061000064D1000858D100086CD1000800D1000803
:1061100094D1000810D10008BCD10008AC4B93E822
:10612000070003F10C0425AE86E8070094E8070099
:106130002AAD03F1180485E8070094E807002FAFA3
:1061400003F1240487E8070094E8070030330DF1D9
:10615000E40989E8070093E8070008963EAE86E860
:10616000070006950596FDF77BF90B90FDF71EF9E4
:106170000546FDF7FFF90C90FDF7A6FC8046FDF7FC
:10618000A5F9944C0D9015A8FDF756FC236805F071
:106190000102C5F3400B0792002B00F075838E4877
:1061A000FEF7E0FD0446002800F00B868B4905F061
:1061B00066F9002800F070832046894905F05FF9F0
:1061C000002840F0AE858748FEF7E6FD002800F085
:1061D0002686012645F002050996CAF80050472692
:1061E0002046814905F04BF90546002800F06A85F4
:1061F00020467E4905F043F9002840F0B0857C4DEB
:10620000DFF870A20A9558260DF1580B42467949DD
:10621000584605F003F9784B76495A690DF1600844
:106220001EA805F0FBF81AAD72499DF854204046AF
:1062300005F0F4F81CAC6F499DF85520284605F090
:10624000EDF89DF856206B49204605F0E7F80A9BCB
:10625000CDF8D0801A6835953694002A40F02B8509
:1062600046AC04F8982D6548FEF7C0FDFEF722FE07
:1062700008980321FEF704FF079D61486149624ABF
:10628000624B0095FFF710F90B9D5D4800950425C2
:106290005F49604A604B0195FFF71CF9099D58481A
:1062A00000955E494F4A5E4BFFF7FEF80D9D002DAD
:1062B00000F0D9840C9D002D00F0E7840223594A98
:1062C00059495A4800932346FFF7C4F8FEF706FFE2
:1062D0004B48FFF78FF856485649FEF705FF5648DA
:1062E0005649FEF701FF41485549FEF7FDFE554866
:1062F0005549FEF7F9FEFFF79BF8BAF1000F3FF49E
:106300002BAB5248FEF766FD5046FEF763FD504842
:10631000FEF760FDFFF720BB4E48FEF75BFDA04691
:106320001EAD20AC42464C49284605F077F8284679
:10633000FEF750FD4948FEF74DFD4046214610222C
:10634000FEF796F800283DD000270CE0E25D2846D5
:1063500005F064F82846FEF73DFD01374048FEF79A
:1063600039FD102F0BD007EB0803B3F5A27F3D4991
:106370003D48EBD90137FEF72DFD102FF3D13848FA
:10638000FEF728FD002320212E2003EB0802B2F5A2
:10639000A27F88BFE15404D8E25C203A5E2A88BF1D
:1063A000E0540133102BF0D1002320468DF89030BB
:1063B00008F11008FEF70EFD2C48FEF70BFDB8F5AE
:1063C000A87FAFD12A48FEF705FDFFF7C5BA00BF89
:1063D0001CC800080C0C00206CCE000860D200081D
:1063E0006CD2000870D20008BCD20008CCD20008E1
:1063F00004040020ECD400087C010020E0D2000856
:10640000D0D20008F4D2000864D20008FCD2000800
:106410001CD30008B0D200087C0B002094C90008EF
:106420002CD30008C0D2000858D3000858D1000867
:106430007CCE0008F8CE000884CE000804CF000807
:1064400070D30008D8D2000880D3000840CF0008DD
:10645000E0D0000858CF000860CF000868CF0008DF
:10646000A4CB000840DC000874CF000838C900083D
:106470006CCF0008F0CD0008B34D0FCD3EAC0594B5
:106480000FC495E80F0084E80F00B048FEF76AFCDF
:10649000044630B1AE49062205F00BF8002800F0A2
:1064A0003A82DFF830B30DF1E409AA48FEF79EFC0A
:1064B00025ACFEF7FFFC05980821FEF7E1FD1AADBB
:1064C00008941CAC4FF0000A079509942AAD20AC43
:1064D000069556462FAF0DF1D0081EAD05940BEB77
:1064E0000A0C48F68904DCF804209B49CDF80CC05E
:1064F000C8F68804A4FB02025209099804F08EFF32
:10650000DDF80CC09449DCF80420A4FB02035B090D
:10651000C3EB0313A2EB8302284604F07FFF8F48EE
:10652000FEF77CFF32468E49079804F077FF32462B
:106530008C49059804F072FF32468B49089804F0A4
:106540006DFF32468949069804F068FF3246884953
:10655000384604F063FF32468649404604F05EFF49
:106560000798FEF713FD5BF80A2083490898C2F3E9
:10657000C012FEF73DFE5BF80A207F490698C2F381
:106580008012FEF735FE32467C49484604F046FF4D
:106590005BF80A207A48C2F3C204FEF71BFC07230B
:1065A000224678494846FEF7CDFD7748FEF712FCB3
:1065B00032467649484604F031FF5BF80A207048BD
:1065C00002F00704FEF706FC224607236D49484601
:1065D000FEF7B8FD6C48FEF7FDFB02246848FEF7A5
:1065E000F9FB6549099A009423463846FEF7E2FC18
:1065F0006548FEF7EFFB6248FEF7ECFB5E4900944E
:106600002A4623464046FEF7D5FC5F48FEF7E2FBEC
:1066100001360598FEF71AFDFEF710FF082E0AF165
:10662000080A7FF45CAFFEF759FD0026FFF794B926
:10663000574F584D97E8070007F13C040DF1D0087B
:1066400088E807000FCC3EAE503705960FC697E896
:106650000F0024682F6834600DF1E40989E80F0009
:10666000002F00F02981DFF870B1FCF74BFF0746DF
:10667000FCF780FF05463548FEF774FB044600280A
:1066800000F0CA83444904F0FAFE0346002800F0F3
:10669000CE822046414904F0F2FE0346002800F075
:1066A0007D8320463E49032204F003FF064600286E
:1066B00000F0758420463B49062204F0FAFE0646A7
:1066C000002800F0C28420463749072204F0F1FE7A
:1066D0000646002800F0A08420463449042204F035
:1066E000E8FE0646002800F062852046304904F0A6
:1066F000C6FE0026B24610B9DFF8E0A053262D48AA
:10670000DFF8D4B0FEF772FB0B24FEF7D3FB404654
:106710000321FEF7B5FC28482849294A294B019452
:1067200000970224FEF7D6FE2749284A284B224824
:1067300001940095FEF7CEFEFEF7D0FC05980521EA
:10674000FEF79EFC002451E07CC800086CCE0008D7
:10675000F8D4000810D5000864CE0008A0C90008CD
:10676000ECD4000824D500082CD5000830D500084A
:1067700034D5000838D50008C0C8000808D500087E
:10678000D4C9000810000020DCC900080CD500089E
:106790001CC80008140C002098D30008A8D30008D7
:1067A000BCD30008C0D30008D8D30008E8D3000841
:1067B000D8D20008F0D3000870C9000808D4000837
:1067C0009CD30008500B002014D40008ACD3000860
:1067D000280C0020A43E00205000002004CE000819
:1067E00001340B2C0BF1140B00F00381DBF810309B
:1067F000D807F5D52246BD491AA804F00FFE224657
:10680000BB491CA804F00AFE2246BA491EA804F09F
:1068100005FE2246B84920A804F000FEDBF8082057
:10682000B64918A804F0FAFDB548FEF7F7FDDBF805
:106830000000FEF7ABFB18A91CA8B24AFEF79CFDAE
:106840001EA8FEF781FDDBF81020AF49C2F340021D
:1068500020A8FEF7CDFC1AA8FEF7F8FBFEF7EEFD28
:10686000BEE7AA480999FEF7ABFDFEF7D5BF28465B
:10687000A74904F004FE00283CD10123CAF80030E7
:106880005026A44CFEF7AABFA34BA44E0FCB86E81C
:106890000F000123236082E4A148FEF77DFA00285F
:1068A00000F05982012645F001050796CAF800500C
:1068B000CDF824B0472693E49A4ADFF8C8B23B46A5
:1068C00053F80B101433DC2B42F8041FF8D1964B0D
:1068D00096491A681B6981E80C0001232B60C4E605
:1068E00006460446FEF77ABFDFF89CA24E26044611
:1068F000FFF79BBA28468E4904F0C1FD002840F0FE
:106900001F83CAF8000050268A4CFEF767BF002696
:106910003546FFF720BBA01D04F03AFA07280446CD
:106920003FF6BFAD01468448FEF744FA834904F0C0
:10693000A6FD002800F05A83DFF850B25BF834302F
:1069400023F080034BF8343021467D48FEF732FABD
:106950007A4904F094FD002800F041835BF834305C
:1069600023F040034BF834300DF1E4092246754919
:10697000484604F053FD4846FEF7F4F904F008FADF
:10698000224671490546484604F048FD4846FEF750
:10699000E9F904F0FDF95BF83430ED0000F0070090
:1069A00023F03F0340EA030205F0380313434BF89A
:1069B000343021466548FEF7FDF904F0E9F9214637
:1069C00005466348FEF7F6F904F0E2F90BEBC40460
:1069D000C5EB051500EB8500606003F023F864E566
:1069E00001F0A6FA5B4DFEF7EFBF06468346FFF7C0
:1069F00024B9FEF773FB48460421FEF741FB564DD0
:106A000000242B68D90700F1C38001341035022C13
:106A1000F7D1FEF763FB3A48FEF7ECFC67E44F4B17
:106A200093E803003EAC059484E80300FFF7D3BA73
:106A30004A4B93E803000DF1E40989E80300FFF7EE
:106A4000AABA224646491AA804F0E8FC224645495B
:106A50001CA804F0E3FC224643491EA804F0DEFC17
:106A600055F8082C254914A804F0D8FC3F48FEF737
:106A7000D5FC55F80C0CFEF789FA14A93C4A1CA861
:106A8000FEF77AFC1EA8FEF75FFC1AA8FEF7DEFAF6
:106A9000FEF7D4FCFFF73BB93648FEF763F904F084
:106AA00077F907463448FEF75DF982463348FEF72A
:106AB00059F90446002F00F0B78104F0F2FC0928D0
:106AC00000F2CC812E4CB246FFF7AFB92AAC20467B
:106AD0000A49069404F0A2FCFFF790BA2FAF38469B
:106AE000064904F09BFCFFF77FBA00BF24D40008DE
:106AF000C8D300082CD40008D0D30008ECD4000878
:106B000070C9000834D40008C0C80008E0CE0008EE
:106B10007CCE0008C8CC0008AC0100207C0B002013
:106B200064D200084C0B00207C010020280C0020BF
:106B300084CE0008E0CC000800D500089CC80008FE
:106B400004D5000808D500080CD50008ACCE000814
:106B50003CD80008D8CD000888010020F8CC0008F7
:106B6000E0D400088CD40008E8D4000888C90008E4
:106B700054D3000890CF00089CCF000864DE0008C2
:106B800000CD000850000020A8CD0008A43E002041
:106B90002246BF4925A804F041FC2246BD492AA847
:106BA00004F03CFC2246BC492FA804F037FC55F801
:106BB000082CBA4916A804F031FCB948FEF72EFC9F
:106BC00055F80C0CFEF7E2F916A9B64A2AA8FEF70A
:106BD000D3FB2FA8FEF7B8FB25A8FEF737FAFEF780
:106BE0002DFC12E7B048FEF7BDF804F0D1F803F031
:106BF00025FC3546FFF7AFB92FAF3846AB49BDF896
:106C00003A2004F00BFCFEF7F5BEA948FEF7AAF8FF
:106C100003F0A0FE002800F0BB803446DFF8E8A2B5
:106C2000FFF703B901F068F9A24DFEF7CDBEA24807
:106C30000493FEF797F804F0ABF8CAF80000049B41
:106C4000074641269A465AE59C48FEF78BF804F021
:106C50009FF803F05DFE002800F0AD803446DFF8B9
:106C6000ACA2FFF7E2B88E48FEF7D8FB9448FEF7D7
:106C70008DF98C4A93485946FEF77EFB9148FEF702
:106C8000E5F9FEF7DBFBFFF715BB059DCDF800909E
:106C90000195834806993A4634ABFEF741FCFFF76D
:106CA0000DBB8948FEF75EF804F072F803F0BCFDF6
:106CB0003546FFF750B920AC2046784904F0AEFBCA
:106CC000FFF7D1BA814B82480A93FEF74BF804F0E4
:106CD0005FF80A9CAA462060FFF796BA7948FEF74B
:106CE00041F804F055F862260990CAF80000FEF752
:106CF000A4BF484604F0D5FB764B09EB0002198887
:106D00009B7829F800109370FFF737B9059804F0C5
:106D1000C8FB704B3A1819889B7839529370FFF76B
:106D20004CB920466C4904F0AAFB002800F04A81C7
:106D300020466A4904F0A3FB002800F0BA812046EF
:106D4000674904F09CFB002800F05981CDF824B07D
:106D50000026FFF745BA25F001050790A6E5204675
:106D6000604904F08CFB002840F00981574D012355
:106D7000CAF800305026DFF898A10A95FFF744BA08
:106D800026462546FEF720BE06460546FEF71CBEF3
:106D900006460446DFF87CA1FFF747B85248049343
:106DA000FDF7E0FF03F0F4FFCAF80000049B05467E
:106DB00046269A46A3E406460446DFF85CA1FFF7A0
:106DC00034B8424BCDF824B0064682460A93FFF70A
:106DD0001BBA064604468246FFF727B84348FDF72C
:106DE000C1FF03F0D5FF8DF83C004148FDF7BAFF25
:106DF00003F0CEFF8DF83D003E48FDF7B3FF03F0F2
:106E0000C7FF8DF83E000F9B1A0CAAF800308AF8D5
:106E100002206326FEF711BF064682466FE425F086
:106E200002050990FFF7D9B93348FDF7DFFF334872
:106E3000FDF7D0FFFEF776F9FEF77EFA4FF4FA7011
:106E4000FAF7FCFC2E4B6F6085F83C7050462146EB
:106E50001F603E46FDF79CFEFEF716BC2648FDF778
:106E6000C5FF2848FDF7B6FFFEF75CF9FEF764FAA8
:106E70004FF4FA70FAF7E2FC214B6E6085F83C6043
:106E8000504621461E60FDF79BFEFEF7FDBB00BF8E
:106E900038D40008E0D3000840D40008ECD400083F
:106EA000D0D2000854D3000800D100082CC4000838
:106EB00024D00008D8CD00089CD3000834D00008A6
:106EC00040D30008A8E1000810D100080404002005
:106ED000C0D2000830D100087CD200088CD2000853
:106EE000ACD200087CCE0008ACD3000898D20008D1
:106EF0009CD20008A4D20008A4CF0008B8CF000894
:106F0000F4110020ECCF000820CD000868CD000867
:106F1000C8CC000844CD000888CD0008C248FEF760
:106F20007DFAC248FEF732F8C14AC24810A9FEF7FE
:106F300023FAC048FEF78AF8FEF780FAFEF7C9BECA
:106F40002846BD4904F09BFA0B90002800F0D18040
:106F50002846BA4904F093FA0446002800F0358127
:106F600000263446FEF73ABCB548FDF7FBFE03F0B9
:106F70000FFF64260790CAF80000FEF75EBE2046A9
:106F8000B04904F07CFA002840F03E81AE4BCAF8CC
:106F900000005026DFF800A30A93FFF735B9E01C84
:106FA00003F0F6FE0A280AD800EB80000BEB800BFA
:106FB000B246DBF80C30CBF80830FFF7A0BBB24686
:106FC000FFF79DBB9B48FDF7CDFE03F0E1FE422697
:106FD0008046CAF80000CDF824B0FFF701B95BF88D
:106FE000343043F040034BF83430BDE4DFF8ACB24A
:106FF0005BF8343043F080034BF83430A4E493481A
:10700000FDF7B0FE03F0C4FE44260B90CAF8000062
:10701000CDF824B0FFF7E4B8E01D03F0B9FE012875
:107020000446CCD802468A492AA804F0F7F92AA8CF
:10703000FDF798FE03F0ACFE0F28C0D8854B03EB9C
:107040000414B2466060FFF75ABBA01D03F0A0FE17
:107050000A288246B3D802467F4920AC1CA804F017
:10706000DDF97E495246204604F0D8F91CA8FDF708
:1070700079FE03F08DFE431E0E2B4FEA8A069CBF5D
:1070800006EB0A030BEB8303564498BF9860204637
:10709000FDF782FE0BEB860B002800F02A81DBF85F
:1070A0001030002643F00203CBF81030B246FFF751
:1070B00026BB6B48FDF756FE03F06AFE8DF85400C0
:1070C0006848FDF74FFE03F063FE8DF855006648F3
:1070D000FDF748FE03F05CFE8DF85600159BCDF8D9
:1070E00024B01A0CAAF800308AF802204326FFF7D1
:1070F00077B85E48FDF736FE03F04AFE03465C486B
:107100000493FDF72FFE03F043FE84465948CDF863
:107110000CC0FDF727FE03F03BFE04465648FDF782
:1071200021FE03F035FE0C905448FDF71BFE03F0E2
:107130002FFE049B0D901A465149484604F06EF903
:10714000DDF80CC04F496246304604F067F922462C
:107150004C4914A804F062F94A490C9A15A804F0A5
:107160005DF948490D9A584604F058F90C9E049B65
:10717000DDF80CC0CAF808600D9ECAF80C40CAF8C9
:1071800004600B9EA3F26C710CF1FF32CAF81C1064
:10719000CAF81020CAF80060204661461A46F9F77E
:1071A0009FFF5426CAF818000B9CFEF717BB201D42
:1071B00003F0EEFD01283FF602AF264B03EB001370
:1071C000B2469A685A60FFF79ABA2F48FDF7CAFD8F
:1071D0001E220146504604F085F97026FEF7FEBADD
:1071E000E81D03F0D5FD0328054664D9B346FEF734
:1071F00024BD2648FDF7B6FD03F0CAFDFCF728F9CB
:10720000B3460B90FEF719BD20460F4C20490A9457
:1072100004F035F91F4B00280CBF9A464FF0000AC6
:1072200008BF5326FEF7F0BF88C9000840D3000806
:1072300054D30008A8E1000890CE0008B8CE00089A
:1072400058D4000884CE000804040020B0D20008FE
:10725000E0D300087C010020C8D30008D0D3000888
:1072600098D200089CD20008A4D20008A0CE000842
:10727000A8CE0008B0CE000854E10008B4CE000843
:1072800060CE000864CE0008BCCE000878D40008A8
:10729000D8D2000804CE0008E0CC0008A43E0020AC
:1072A0001948FDF75FFD03F073FDFCF7C3F8B34623
:1072B0000A90FEF7C2BC024614491CA804F0AEF8BE
:1072C0001CA8FDF74FFD03F063FD0F288ED807EBD8
:1072D0000515B3466860FEF7B0BC281D03F058FDE5
:1072E000032883D807EB0013B3469A685A60FEF769
:1072F000A4BCDBF8103023F002030646CBF81030B4
:107300008246FFF7FCB900BF68D400088CD400089F
:1073100030B585B04FF480446846F9F771FB002220
:10732000200448F2A063C0F201030121ADF804205B
:10733000ADF8082040F4B8404FF480624BF6FF757A
:10734000ADF80650ADF80A20ADF80C400093F9F7FF
:1073500065FB200440F4B8406946F9F7E1FA05B04E
:1073600030BD00BF10B54FF4B844C4F2000420464D
:107370000121F9F76FFB20460121F9F791FB204627
:107380000021F9F78DFB2046F9F792FABDE810408D
:10739000FFF7BEBF70B505460E4643F2010401E09B
:1073A000013C13D04FF4B8402946C4F20000F9F76D
:1073B0008BFB0028F4D04FF4B840C4F200003146F3
:1073C000F9F782FB0028EBD0012070BDFFF7CAFF60
:1073D000204670BD38B5054619B1BDE83840FFF705
:1073E000D9BF43F2010401E0013C0AD04FF4B84098
:1073F000C4F200002946F9F767FB0028F4D0012009
:1074000038BDFFF7AFFF204638BD00BFF8B50746CF
:107410004FF4B840C4F200000E46012115461C4648
:10742000F9F70AFB0120C1F200000021FFF7D2FFAB
:10743000002832D04FF4B840C4F2000034BB012120
:10744000F9F720FB4FF4B844C4F200042046F9B227
:107450000022F9F70DFB0220C1F200000021FFF726
:10746000B9FFB8B18020C1F200000021238BFFF7E3
:10747000B1FFA8B125B1C6F307212046F9F71EFBDD
:107480002046F1B2F9F71AFB0020F8BD0021F9F708
:10749000F9FAD7E76FF00100F8BD4FF0FF30F8BD03
:1074A0006FF00200F8BD00BF30B5284B1C6883B0F8
:1074B0000CB103B030BD012568461D60F9F7CAF96B
:1074C00029464FF40000F9F781FB28462946F9F7D1
:1074D0006FFB04202946F9F76BFB29464FF40000A7
:1074E000F9F790FB21464FF40000F9F78BFB0020E1
:1074F00008210422C4F20200F9F7C2F94FF4006037
:1075000004220921C4F20200F9F7BAF9022300208B
:1075100069468DF804308DF80530C4F202004FF44E
:10752000807300938DF806508DF80740F9F736F90F
:107530004FF400604FF40073C4F2020069460093F8
:10754000F9F72CF9FFF7E4FEB3E700BF340C002095
:107550002DE9F041069D6F1E1E467B427B41804611
:10756000FFF754FF074610B13846BDE8F081802090
:107570000421C1F20000C1F20001FFF70BFF002857
:107580005BD04FF4B844C4F2000420460121F9F75F
:1075900053FA0120C1F200003946FFF71BFF002813
:1075A0004ED020465FFA88F10122F9F761FA0220F5
:1075B000C1F200003946FFF70DFF002843D0238BAE
:1075C0008DB33C4611E040200021C1F20000FFF7DE
:1075D00001FF18B34FF4B840C4F20000F9F770FA95
:1075E0003219AC4202F8010C1DD00134AC42EAD190
:1075F0004FF4B840C4F200000021F9F743FA4FF409
:10760000B840C4F200000121F9F724FA402000211B
:10761000C1F20000FFF7DEFE0028DBD16FF00607A5
:107620003846BDE8F0814FF4B840C4F200000121B3
:10763000F9F728FA3846BDE8F0816FF0030793E7C1
:107640006FF0040790E76FF005078DE770B51C46F3
:107650000023FFF7DBFE064608B1304670BD8020F0
:10766000C1F200003146FFF7B5FE28B3049BD3B149
:10767000049BE51801E0AC4215D04FF4B84014F873
:10768000011BC4F20000F9F719FA80200421C1F2AD
:107690000000C1F20001FFF77DFE0028EBD16FF082
:1076A0000306304670BD4FF4B840C4F2000001211B
:1076B000F9F7D0F9304670BD6FF00206CDE700BF94
:1076C00070B43A4A3A49546A0B689C4207D8956AA2
:1076D000AB4204D2D56B002D4FD0364D13E0D46AA7
:1076E000324DA34208D21268032A15D0052A20D0B1
:1076F00001330B6070BC70472E6BB342F3D2ED6B5D
:10770000002D40D02C4D2E681C1B00FA04F426439B
:107710002E601268032AE9D1102BE9D9142BE7D87F
:10772000264AA3F11105146800FA05F00443146019
:10773000DEE7A3F11402032A16D9A3F11804032CDF
:1077400027D81F4C256800FA02F215432560DA0895
:1077500010BB1C4803F00704855C012606FA04F4FC
:1077600025EA04048454C3E7134AA3F10805146806
:1077700000FA05F52C431460E9E70E4C256840EA51
:1077800045052560AFE70C4C256840EA45052560B6
:10779000A9E72F2BACD8DAE70A4803F00704855C89
:1077A000012606FA04F42C438454A1E7600C00205F
:1077B000480C0020A40C0020C00C0020B80C0020B5
:1077C000BC0C0020380C002000B583B06846F9F7E7
:1077D00041F804200121F9F7EBF94FF40060002390
:1077E0004FF48062C4F20200694600928DF80430C2
:1077F0008DF805308DF806308DF80730F8F7CEFF9C
:1078000003B000BD70B4294A1368002B2BD028495F
:107810000B68022B17D0032B264B26D0264C0E6864
:107820002168264DA0F8011019680670A0F8031011
:107830002E68002119604671216001202960002313
:10784000136070BC70471B4B1D681C68E443E4B2B6
:10785000B4EB152F1BD0184C266848F2EE75AE42DB
:107860001AD00020EBE71846EBE71D681C68E443DC
:10787000E4B2B4EB152FF4D11D680F4CEDB21D60CE
:107880000F4D2E681D6845EA06251D60C7E71D6877
:10789000094CEDB21D60C2E70B250D601D68C5F3F4
:1078A000072525601D68EDB21D60B8E7C80C0020F3
:1078B000400C0020440C0020AC0C0020B00C002038
:1078C000500C00202DE9F0474FF400609E4CC4F2AC
:1078D00002004FF48061F8F7C7FF236893B99B4E0D
:1078E000356895B99A4B002800F0C2801B68002BC0
:1078F00040F00C81974B1A684FF6FE718A4201D80E
:1079000001321A602068BDE8F087934F3A68002A78
:1079100070D0002800F0B280904A11780131C9B2CD
:10792000E929117000F206818D4B8E495A6B096866
:107930008A42E7D1996B0029E4D1DFF868828A494D
:10794000D8F800C00D68AC4500F078818748002762
:1079500007601B68012B00F06481052B00F0798122
:107960000A2B18BF292B03D10068C00700F15581ED
:107970000120022B206040F09C81002A40F002820E
:1079800074480368B3F5E16F80F01682784D794F43
:10799000D5F800903B68DFF8F4A1C1F800C049F0C9
:1079A0000109C5F80090CAF8003002606546724AC5
:1079B0003B6002201060714A1360714B1A68714B72
:1079C0001D60714B1A60236863B10B689C4500F021
:1079D000BA816E4A5F481568664FC8F800300023C8
:1079E0003D6003605A4A002313605C4A33600B60B9
:1079F000137087E7664F3B68002B00F08180584B7F
:107A0000002840F0D1801A68032A00F05581DFF881
:107A10004C81DFF83C915A68D9F8001050488A42EE
:107A20000BD88268914208D898F800C0C268944583
:107A300003D30269944540F2B3815B69484A994295
:107A40000BD39369994208D898F80010D3699942EA
:107A500003D3136A994240F2A9810025356088F862
:107A600000500123C9F80030002D3FF44BAF5BE715
:107A70001A6801321A602068BDE8F087DFF8D090FC
:107A8000DFF8D880D9F80030A3F11F020A2A17D8EE
:107A900098F80020052A13D90A2A11D83D49304800
:107AA000442203F0D1F92F4A002313600122C9F8C0
:107AB000002088F800303B60002D3FF423AF33E70F
:107AC000A3F15E02532A08D898F800202D2A00F26C
:107AD0009F80162A01D93049E1E7A3F13C020F2A21
:107AE00040F28980283B162B00F28F8098F80030F6
:107AF000122B40F28A801F2B00F287802749CEE7A5
:107B0000E8B9134B1A6801321A600DE7204B124A8C
:107B10001D6001231360144A336015601B4A156011
:107B20001F4A1560164A15600E4AFF2111600B4A64
:107B30001370E7E6064933600B601370E2E6074A0C
:107B400001233B601370EFE6C80C00204C0C0020B2
:107B5000C40C0020540C0020A80C00205C0C002059
:107B6000600C0020480C0020C00C0020B40C002049
:107B7000B00C0020C0010020400C0020AC0C002004
:107B8000B80C0020440C0020500C0020A40C002055
:107B9000580C0020F4D50008C0D6000838D60008DC
:107BA000BC0C0020BC0100208C49D3F83490D1F8E3
:107BB00000C0E14500F09180DFF854821A6898F81F
:107BC00000A087480AF1010A5FFA8AFA012A88F8B8
:107BD00000A000F09A80BAF1E90F7FF645AF09F1F5
:107BE000FF32944500F0C4807E4A00233360136066
:107BF00088F8003086E698F800203B2A7FF672AFBE
:107C00004B2A3FF66FAF784949E7002535604AE7D0
:107C1000592A3FF662AF754941E775480023036072
:107C2000D1E60268013A012A88BF2360F5D9714A7A
:107C3000714812680360714B1A60BEE66C480068B8
:107C4000B0F5966FBFF482AE6D48076801370760E4
:107C50007FE60368012BE0D001232360694B1F7886
:107C600058789A7887EA000909F00F0989EA171706
:107C700087EA101002F00F09814501D00020206032
:107C800093F803901F79587982EA09037B40984260
:107C900001D0002323605C4B5C4A1F681068554A82
:107CA00038431860544B126805201860534B1A6013
:107CB00083E6052BD2D0BAE748490A68102A7FF438
:107CC000A6AEDFF82091D9F80020053A072A79D925
:107CD0004F4B306018700546C3E6986B01287FF45F
:107CE0006BAFDFF800915869D9F80010884205D8C9
:107CF0009869814298BF9A637FF6B6AE444A0023E2
:107D00003360C9F800301370FCE5BAF10B0F7FF651
:107D1000ABAEBCF10A0F7FF65EAFDFF8D890C16A58
:107D2000D9F80020ACF10B0A614442EA0A220CF1B6
:107D3000010C0131C9F800200A22C0F834C00163E7
:107D400088F8002065E62B48324F05683A682848D5
:107D5000AA427FF442AE026840F6C90C62459FBF5A
:107D6000294AD2F800C04CF0010CC2F800C034E639
:107D70009B6B002B7FF438AFC1F80090002D3FF4CF
:107D8000C1ADD1E51B4B234F1B6810E60A200F3A0B
:107D90002021186010200F2AD8621963596305D872
:107DA0000120FFF78DFC00233B605AE60020FFF71F
:107DB00087FC00233B6054E6174B164F1A600D4BAF
:107DC0001B68F4E5124A12783B2ADFD94B2ADDD82A
:107DD00000233B6011230B6043E600BF480C0020EA
:107DE000600C0020C40C002004D700087CD60008DA
:107DF000540C0020A40C0020400C0020AC0C0020EF
:107E0000B40C0020380C0020B00C0020BC0C00206A
:107E10005C0C0020C0010020C80C0020F9F734B928
:107E200010B582B004460DF10600F9F73BF978B1C0
:107E3000084B09491B88BDF806200988D21AC2EBF5
:107E40000212CB1A92FBF3F30F2B28BF0F232360F0
:107E500002B010BDCC0C0020CE0C002008B50F4B9A
:107E60001B686BB1FF23C0F2020398420AD80C4B87
:107E700000221A800B4B40F2FF321A80012008BD0D
:107E8000184608BD02220649E120FCF7F1FAE3207A
:107E900004490222FCF7ECFA012008BD5C04002032
:107EA000CC0C0020CE0C002008B50A4B1B680BB987
:107EB000002008BDE12008490222FCF7F3FA00285F
:107EC000F6D00222E3200549FCF7ECFA003018BF97
:107ED000012008BD5C040020CC0C0020CE0C00204A
:107EE00040F6CC43C2F200031888704740F6CE43F8
:107EF000C2F200031888704710B582B0F9F7C4F8D1
:107F00000A240DF10600F9F7CDF840B90A20F9F777
:107F100095FC013CF5D1054C208802B010BD034C06
:107F2000BDF806302380FFF7BFFFF5E7CC0C00203B
:107F300010B582B0F9F7A8F80A240DF10600F9F798
:107F4000B1F840B90A20F9F779FC013CF5D1054CAC
:107F5000208802B010BD034CBDF806302380FFF727
:107F6000A3FFF5E7CE0C0020F9F734B8F0B50746CB
:107F70008DB00A20FCF78CFC092828D00A2813D0E1
:107F8000072803D0002420460DB0F0BDFCF7D6FD35
:107F90000A2201A900F5B67003F0D2FB014638466B
:107FA00002F0EAFC7424EEE7FCF7C8FD00F14C0493
:107FB0002021204603F056FA014610B1002301F8B3
:107FC000013B20463A46FDF7E3FA0446DBE7FCF7BF
:107FD000B5FD01AE00F5A674002502E002340A2DBD
:107FE00012D0237820460221002B7BD06378002B0F
:107FF00078D0F9F7AFF8A37846F8040F0135202BB5
:10800000ECD103340A2DECD1029CA4F141032F2BB7
:10801000B8D801A252F823F0D9800008D98000080E
:1080200033810008D9800008857F0008D9800008C6
:10803000D9800008857F0008857F0008857F0008BB
:10804000857F0008D9800008857F0008ED80000842
:10805000857F0008D9800008857F0008857F00089B
:10806000ED8000080D810008857F0008857F0008ED
:10807000ED800008857F0008857F0008857F000867
:10808000857F0008857F0008857F0008857F0008C0
:10809000857F0008857F0008857F0008D98000085B
:1080A00033810008D9800008857F0008857F00089B
:1080B000857F0008857F0008857F0008857F000890
:1080C000857F0008857F0008857F0008857F000880
:1080D000857F0008F5800008022D7FF453AF039BD5
:1080E0003B6050E7002D3FF44DAF8DE7012D7FF44D
:1080F00049AF48E73846202300F8013B0DF109015C
:108100001E2203F0EFF90023FB773CE7072D7FF4F5
:1081100039AF059BFB60039B03F16402049B7A610A
:10812000013B3B61069BBB60079B7B60089B3B6000
:1081300029E7042D7FF426AF039B3B70049B7B70E3
:10814000059BBB701FE700BF70B53E4B1A688242AB
:1081500088B0064673D002A81E60F8F77BFB04A81F
:10816000F8F7BEFE01200146F8F722FD0120014686
:10817000F8F71EFD4FF400300121F8F727FD00202D
:10818000C4F2020002210722F8F77AFB002007223E
:10819000C4F202000321F8F773FB022300208DF8DC
:1081A0000C30032304460125C4F2020002A98DF815
:1081B0000D30042302938DF80E408DF80F50F8F720
:1081C000EDFA20460823C4F2020002A90293F8F750
:1081D000E5FA4FF48840C4F200002946F8F79AFE09
:1081E0004FF488400C23C4F2000004A9ADF81A3003
:1081F0000496ADF81440ADF81640ADF81840ADF84F
:108200001C40F8F701FE4FF48840C4F200002946F4
:10821000F8F772FE4FF48840C4F2000040F2255196
:108220002A46F8F78DFE262301A88DF804308DF834
:1082300005408DF806408DF80750F8F709F808B0AA
:1082400070BD00BFE80E002030B40F4A13687F2BCA
:10825000FCD80E490E4D0B685C1C7F2C45F82300A2
:1082600098BF0C6001D900230B6072B6136801330C
:10827000136062B64FF48840C4F2000040F22771E8
:10828000012230BCF8F75CBEE40E0020E00E0020B6
:10829000D80C002010B50446007828B1FFF7D4FFB1
:1082A00014F8010F0028F9D110BD00BF30B40D4BF8
:1082B0001A6882B10C490D4D0A68541C802C55F87F
:1082C000225018BF0C6009D072B61A68013A1A60C1
:1082D00062B601220560104630BC704700220A6079
:1082E000F2E700BFD40C0020D00C0020EC0E0020E0
:1082F000024A1368002BFCD1704700BFE40E002037
:108300004FF4884038B5C4F2000040F22551F8F728
:1083100033FE00282BD14FF48840C4F2000040F215
:108320002771F8F729FE00B938BD4FF48840C4F230
:10833000000040F22771F8F745FE234B1A68002A27
:1083400038D0224A224C1168481C802808BF0020DF
:1083500054F8211010601A684FF48840013AC4F2B2
:10836000000089B21A60BDE83840F8F7E1BD4FF46B
:108370008840C4F2000040F22551F8F723FE4FF484
:108380008840C4F20000F8F7D7FD124B1A687F2A24
:10839000C1D81149114D0A68541CC0B27F2C45F850
:1083A000220098BF0C6001D900220A601A680132CD
:1083B0001A60B0E74FF48840C4F2000040F2277121
:1083C000BDE83840F8F7BCBDE40E0020D80E002010
:1083D000D80C0020D40C0020DC0E0020EC0E002075
:1083E00010B541F2EC04C2F2000402460B462046EE
:1083F0004FF4807103F0CEFC2046BDE81040FFF73B
:1084000049BF00BF0FB400B583B004AB53F8040BF1
:1084100019460193FFF7E4FF03B05DF804EB04B0E5
:10842000704700BFFFF790BE10B584B001A8F8F701
:1084300043FC01200146F8F7C9FB0023ADF80C30DE
:10844000ADF80630072301A902934FF0804003F5F1
:108450002D73ADF80430F8F7E3FB01210A464FF025
:108460008040F8F7B9FC01240F2368461C228DF8E0
:1084700000208DF803408DF801308DF80230F7F7B9
:10848000E7FE4FF080402146F8F72EFC04B010BD07
:1084900038B54FF080400121F8F7A8FC6A4B1C6802
:1084A000002C34D0694B1A6843F6982101328A4275
:1084B0001A6000D038BD664C6649674A01202060CA
:1084C0000C6824180C6011680918116014680021E8
:1084D0003C2C1960EED1614B11601A6812181A60B9
:1084E0005F4A10601A683C2AE4D15E4A196013683A
:1084F0001B1813601368182BDCD15B4B11601A68D2
:1085000012181A601A68072AD4D1196038BDFFF70B
:10851000D9F950490B68012B07D9544B1A6840F61A
:10852000A660013282421A6043D0514B1A68013270
:10853000EA2A1A6054D04F4B1A680132962A1A6000
:1085400048D04D4B1A680132962A1A603CD04B4BEA
:108550001A6801320F2A1A6030D03C4B1A6843F671
:108560009820013282421A60A4D1394C3A4A012043
:1085700020600C6824180C601168091811601168DB
:1085800000242D291C6031D01268334B3C2A38D08E
:108590001B681E2B53D03A4B1A68002A8AD01A68DF
:1085A000013A1A601B68002B84D1364B01221A60F5
:1085B00080E71C60344B01221A60B6E7334A012081
:1085C000106000221A60C8E7314A012010600022C2
:1085D0001A60BCE72F4A0120106000221A60B0E741
:1085E0002D4A0120106000221A60A4E72B4B1B4982
:1085F0001C680D68AC421FBF09681960284B1860E1
:10860000C2E7164A00211960136801331360144B46
:108610000120186013683C2BBDD1124B11601A6801
:1086200012181A601A68182AB5D10F4A196013680F
:108630001B1813601368072B08BF1160ABE7194BB9
:1086400001221A60A7E700BF38120020FC110020A9
:10865000F81100204012002034120020481200209F
:108660000C1200202C120020001200201C120020EE
:10867000EC110020101200204C12002008120020E3
:10868000C4010020F011002030120020783E0020AC
:108690007C3E00202812002044120020C801002047
:1086A00018120020141200204DF24870C0F600008D
:1086B000704700BF40F2D013C2F200031868704741
:1086C00041F22C2141F2482241F23423C2F200014E
:1086D000C2F20002C2F2000343F68060C2F2000060
:1086E000096812681B68816042600360704700BFC0
:1086F0002DE9F04F9DB001F04FFF01F0F5FF4FF471
:10870000E130FFF78FFEFFF75FF801F00DFB01F09E
:1087100037FBFFF789FE0120F9F7B4F8F8F754FDAD
:10872000F8F772FD01F0EAFCFBF77AFEF8F786FD38
:10873000002841F0D280C048FFF7ACFDBF48FFF7EA
:10874000A9FDBF48FFF7A6FDBC48FFF7A3FDBD4844
:10875000FFF7A0FDBC48FFF79DFDB848FFF79AFD65
:1087600041F2D420C2F200000368002B01F05C80CB
:10877000B648FFF78FFDB148FFF78CFDB44DFBF70E
:1087800067FD2B68002B01F04680B248FFF782FDA1
:10879000AA48FFF77FFD2B68002B41F07B80AE4C91
:1087A000AE482168FFF72EFE226822F47F0323F4EF
:1087B0007F43EBB940F2FF43C0F201039A4201F25A
:1087C000AA8040F2FF632268C0F201039A4201F2DC
:1087D0009880A348FFF75EFD9848FFF75BFD20688F
:1087E00001F0E2FF206801F0E9FD2068FFF736FBA9
:1087F000FFF7BAFBF8F764FD01F07CF941F238218C
:10880000C2F2000101230B6002F018F841F2382295
:10881000C2F2000200261660FAF7E0FCFAF720FE2A
:1088200041F20423C2F2000341F2242A1860FAF74D
:1088300069FEC2F2000ACAF80000FAF79BFE41F294
:10884000202EC2F2000ECEF80000FAF73FFE41F2F1
:108850003C21C2F200012B68086083B34FF480759D
:1088600023687D4FC0F20205AB4228D07D482946DF
:10887000FFF7C8FD764B3D601B68002B41F07E8002
:108880007948FFF707FD6D48FFF704FD01F0EEFBA7
:10889000002801F06B80FBF7ABFB002801F05E8045
:1088A00002F002F8002801F0518001F0BBF8002826
:1088B00001F01F804FF48073C0F20203236041F285
:1088C0001822C2F2000241F240230120C2F200034A
:1088D00010601C68014602460334FAF77DFC41F241
:1088E0004025C2F2000509A82B689C421ED9FEF75C
:1088F00089FF0028F3D000210A460120FAF76CFC1A
:108900000120F8F7A9FF09A8FEF77CFF0020014627
:108910000246FAF761FC5548FFF7BCFC4748FFF7F1
:10892000B9FC01F0A9FA08B101F0A0FB0020014652
:1089300002468046FAF750FCFCF7C6F9FCF7FEF851
:108940004FF0010ACDF814A0DFF82891484FCDF878
:10895000188000F13C0A834604254446CDF81CA04B
:10896000CDF8108013A8FFF701FB8246002840F0E5
:10897000E381D9F800303BB141F23C22C2F200025F
:108980001368002B40F00381B8F1000F40F0238101
:10899000DBF80030002B40F009863548F8F75CFC26
:1089A000002840F0478141F21820C2F2000003681D
:1089B00073B141F2D421C2F200010B68002B40F0E8
:1089C000FF8541F2182EC2F2000E0023CEF80030CF
:1089D000D9F800306BB141F23C20C2F200000368CC
:1089E0003BB141F23021C2F200010B68002B40F094
:1089F000AB8641F2F012C2F20002136893B1DBF8C9
:108A00000430002B40F0228641F2F016C2F200063C
:108A100040F2C41A0023C2F2000A336040F6D86361
:108A2000CAF8003041F20C2EC2F2000EDEF800301F
:108A3000002B40F052851FE050D7000838C90008CD
:108A400070D7000890D7000848D700089CD70008C6
:108A50005C040020BCD70008D0010020D0D700085B
:108A600088D80008C4D80008E8D80008A8D90008A9
:108A7000803E0020043E002041F21421C2F2000199
:108A80000B68002B00F0368340F2044AC2F2000A61
:108A90008E4ADAF8003000211160002B00F02A83A2
:108AA00041F2482EC2F2000EDEF80020B2FBF3F1D4
:108AB00003FB1123002B40F01D8340F24840C2F21B
:108AC00000000368002B40F0548541F2D42EC2F21E
:108AD000000EDEF80030002B00F0438501F0B8FCFA
:108AE0007B4B7C4A064616F0010F7B484FEA560145
:108AF00018BF1A46FFF786FCFF2E09D03046FBF759
:108B00009FF841F24020C2F200000368063306934A
:108B1000002D40F0038341F24420C2F200000368BC
:108B2000002B40F0188341F2F812C2F200021368E1
:108B3000002B40F0228341F22825C2F200052B6869
:108B4000002B40F02C8301F055F9FF28054600F07A
:108B50003183002101200A46FAF73EFB132D00F273
:108B60006B86DFE815F0C901BC01AA0145021A02B3
:108B70000802E30194025802AE025C0190018301F5
:108B8000760169019D01470132016906C90008A803
:108B9000FFF746F900283FF4F7AE40F2CC13C2F2DB
:108BA0000003089A1968531C8B4203D34B1C9A424A
:108BB0007FF6EAAE4948FFF725FC40F2CC15089B4A
:108BC000C2F2000518462B60FAF784FF0225B8F1BF
:108BD000000F3FF4DDAE41F2F416C2F200064FF092
:108BE00001083368002B7FF4D8AEDBF804304FF077
:108BF0000108002B3FF4D1AE394B3A48C3F800804E
:108C0000FFF748FB3848FFF745FB41F2F01A3749B8
:108C1000079A0BA802F002FCC2F2000A0BA8FAF7AE
:108C2000BBFF3348CAF800800425F8F715FB00287D
:108C30003FF4B9AE012001460022FAF7CDFA41F225
:108C4000D42EC2F2000EDEF80030002B40F0198561
:108C500041F22C20C2F20000BC680368244A9C4206
:108C600000F06685D2F804E0042540F21002B969EC
:108C70003E69D7F800C0F868C2F2000241F2002A4B
:108C800052F821307A69CDF80CC0C2F2000A8DE8A2
:108C90001140CAF80010194641F2482A731C41F2EB
:108CA0002C26C2F20006C2F2000A3460CAF800E0C4
:108CB00041F2342EC2F2000E0E48CEF800C002F28D
:108CC0006C72FFF79FFB32246DE600BF1412002088
:108CD00030D10008C0C8000808DE000810DD000818
:108CE000F41100204CDD000838C9000860DD0008E0
:108CF000803E002068DD0008AC48FFF7CBFAAC48A6
:108D0000FFF7C8FA0126322404960025059E18EACA
:108D1000060F52D1002C3FF425AE013C7FF422AE69
:108D2000204621462246FAF757FA13A8FFF71EF904
:108D3000824600283FF41DAE002101200A46AAF118
:108D4000410AFAF749FABAF1330F00F24182DFE83B
:108D50001AF0A40391038C0376033F0261035603C8
:108D60003F0234023F023F0235033F02CA023F0284
:108D7000B2023F023F02A7024B023F023F022A0318
:108D80001F033F023F023F023F023F023F023F02FA
:108D90003F023F02140305039C023F023F023F02D1
:108DA0003F023F023F023F023F023F023F023F02BB
:108DB00091023F023F023F024202F8F73FFA0028C9
:108DC00040F09C8401260596A4E77A48FFF762FAF2
:108DD0007748FFF75FFA41F23C26C2F2000633689B
:108DE000002B40F0DF840025FAF78AFE3224049538
:108DF00002258BE77048FFF74DFA6D48FFF74AFAF6
:108E000041F23C26C2F200063368002B40F0BB84DE
:108E10000025FAF76BFE32240495022576E76748B1
:108E2000FFF738FA6248FFF735FA0025FAF7B4FD84
:108E300032240495022569E76148FFF72BFA5C4864
:108E4000FFF728FA0025FAF7E7FD322404950225FA
:108E50005CE75C48FFF71EFA5548FFF71BFA00264F
:108E6000FAF7AAFD3224049602254FE75648FFF789
:108E700011FA4F48FFF70EFA0025FAF7ADFD32243C
:108E80000495022542E75148FFF704FA4848FFF7E6
:108E900001FA0026FAF770FD32240496022535E720
:108EA0004B48FFF7F7F94248FFF7F4F90026FAF7C5
:108EB000A3FD32240496022528E74648FFF7EAF985
:108EC0003B48FFF7E7F9FAF7F1FA41F20425C2F25D
:108ED00000050026286032240496042516E73E4843
:108EE000FFF7D8F93248FFF7D5F900240494FBF7CF
:108EF0007FF83224049D09E73848FFF7CBF92C4866
:108F0000FFF7C8F940F2701EC2F2000EDEF8005002
:108F1000D5F1010538BF00250026CEF800503224D7
:108F20000496B5420CBF14250C25EFE62C48FFF73C
:108F3000B1F91F48FFF7AEF941F22C26C2F2000644
:108F4000284B3268002A00F006841A68013A1A6039
:108F500041F2342AC2F2000A0023CAF8003041F27A
:108F6000D42AC2F2000ADAF80060002E73D132244B
:108F700004960425CAE61C48FFF78CF90C48FFF755
:108F800089F9FAF7CDFA41F22426C2F2000600254B
:108F90000495322430600425B8E61448FFF77AF9C6
:108FA0000348FFF777F9FAF7C7FAECE758E000084B
:108FB00038C900083CE0000820E0000858DF00083D
:108FC000E0DF0008BCDF000898DF000878DF000859
:108FD00000E0000878DE000868DE000858DE0008BF
:108FE000F8DE00082C120020D8DE0008B8DE0008E9
:108FF000C448FFF74FF9C448FFF74CF9FAF744FAB1
:1090000041F2042AC2F2000A002504953224CAF86B
:10901000000004257AE6BD48FFF73CF9BA48FFF79F
:1090200039F941F24821C2F20001B94B0A68002A1D
:1090300000F095831A68013A1A6041F2D42AC2F20C
:10904000000A41F23422C2F20002DAF80060002382
:109050001360002E8BD041F22C2A41F2482E41F2AF
:109060003420C2F2000EC2F20000C2F2000A002553
:10907000DAF80010DEF800200368A648B9607A60CC
:109080003B60322401F096F8049504253EE6A248A0
:10909000FFF700F99C48FFF7FDF841F22C2EC2F2D1
:1090A000000E9E4BDEF80020162A00F25E831A683E
:1090B00001321A6041F23420C2F200000023036042
:1090C0004DE79748FFF7E6F88F48FFF7E3F841F2DE
:1090D0004823C2F200031A688D4B3A2A00F24283F9
:1090E0001A6801321A6041F23424C2F200040023EB
:1090F000236034E7049E002E7FF4DFAC069E002E32
:109100003FF406AD41F2402AC2F2000ADAF800301C
:10911000B342FFF4FDAC049E042506968148FFF798
:10912000B9F87948FFF7B6F841F22C2A41F2482EF7
:10913000C2F2000EC2F2000A2A46DAF80000DEF897
:109140000010FAF75DF841F24420C2F20000036813
:10915000002B3FF4E8AC40F27011C2F20001724BF8
:10916000086800221A60FAF7DBFA41F2F812C2F23C
:1091700000021368002B3FF4DEAC6C4B00221A6037
:1091800041F23423C2F2000341F22825C2F2000565
:109190001868FAF707FA2B68002B3FF4D4AC644B3D
:1091A00000221A60F8F7C6F800F024FEFF280546F2
:1091B0007FF4CFAC00250495A8E55E48FFF76AF878
:1091C0005148FFF767F800F057FE002840F0808113
:1091D0003224FFF7CEBB139B40F2C414C3F56E6379
:1091E000C2F200040233236041F2D426C2F2000628
:1091F0003368002B40F0E58241F22C2AC2F2000ACB
:10920000159CDAF800309C4200F0DF82DDF850E077
:10921000042540F21000199B169ADDF84CC0C2F2EA
:10922000000041F22C2650F82310009241F2482A07
:1092300041F20022C2F20002C2F20006C2F2000AAB
:109240000194CDF808E0CDF80CC013603460CAF882
:1092500000E041F2342E189A179B3748C2F2000EF4
:1092600002F26C720133CEF800C03224FFF7CAF864
:10927000FFF77FBB13A8FAF78FFC304813A9FFF75D
:10928000C1F804253224FFF774BB1398FAF7B8F835
:1092900001462B48FFF7B6F804253224FFF769BBD7
:1092A000FAF7A6FE2748FEF7F5FF1748FEF7F2FF8C
:1092B0003224FFF75EBB40F27010C2F20000139B35
:1092C0000268934284D0204A20491360002B204B2F
:1092D000204808BF194614BF0C2514253224FFF777
:1092E00091F8FFF746BB41F2F011C2F200010123F1
:1092F00019480B60FEF7CEFF0348FEF7CBFF322480
:10930000FFF737BB98DE000838C9000828DF0008DF
:1093100048120020803E002010DF00082C120020A0
:1093200040DF000848DE000844120020F811002049
:1093300028120020BCDC000864DC0008F4DC000813
:10934000ACDA0008D4DC00087001002094E00008CA
:10935000A8E0000870DA00089CDC000813A8FAF7FF
:109360009BFBCA489DF84C109DF84D209DF84E304F
:10937000FFF748F83224FFF7FCBA1398FAF7D2FB4C
:10938000C3481399FFF73EF802253224FFF7F1BADC
:10939000C048FEF77FFFC048FEF77CFF3224FAF793
:1093A000CDFBFFF7E6BABD48FEF774FF0124BA48CB
:1093B000FEF770FF04943224FFF7DBBA139B002BF7
:1093C00000F00F8241F23C2AC2F2000AB4480123A5
:1093D000CAF80030FEF75EFFAF48FEF75BFF41F2D0
:1093E0003C21C2F2000140F2CC12C2F20002FF2383
:1093F000086813603224FAF76FF8FFF7BABA1398C7
:10940000F9F7DAFFA7481399FEF7FCFF0425322489
:10941000FFF7AFBA41F22026C2F200061398336874
:1094200098423FF4D5AEFAF7ABF89F4A034601469F
:109430009E4813603224FEF7E5FFFFF79ABA41F227
:109440000421C2F2000113980B6898423FF4C0AEA9
:10945000FAF70CF8964A034601469648136004252D
:10946000FEF7D0FF3224FFF784BA13A8FAF7F0FA18
:10947000914877E741F23C25C2F200052B68002BAA
:1094800040F0BC811398FAF725FB8C481399FEF73E
:10949000B9FF02253224FFF76CBA41F22422C2F24E
:1094A00000021398136898423FF492AEFAF730F82E
:1094B00041F24424824B0146C2F200041960814803
:1094C000002323600425FEF79DFF3224FFF751BAE5
:1094D00000F0CCFD3224FFF74CBA7B4B00221A601F
:1094E00041F2002041F22C22C2F20000C2F200023E
:1094F00041F24825C2F20005016813682A68734DDD
:1095000040F27016C2F20006C3EB0313306802EBA0
:10951000830200F0B3FA002800F0A28041F22C2A66
:1095200041F2482E2968DFF8D0C16948C2F2000A2A
:10953000C2F2000EDAF80020DEF80030D1F1010EA0
:1095400038BF4FF0000E6349C5F800E0BEF1000FD0
:1095500008BF61460CBF14250C25FEF753FFFFF72B
:109560008BBA5D48FEF796FE4B48FEF793FEFFF779
:10957000CFBA41F23821C2F2000101230B6001F0A1
:10958000FDF841F2382A0646544B554A554816F024
:10959000010FC2F2000A18BF1A464FEA5601002313
:1095A000CAF80030FEF72EFFFFF7A6BA4E48FEF7C6
:1095B00071FE3948FEF76EFE4FF00108FFF7EDB976
:1095C000DFF830A1504600F081FE00283FF4F9A9F1
:1095D00041F22C22C2F20002DAF808E013689E453C
:1095E00000F0C680DAF804C0042540F2100AB96918
:1095F000F8687E69C2F2000A41F200225AF821306E
:10960000CDF808C08DE80140C2F20002386841F28E
:10961000482A0390116006F26C7241F22C26C2F2C5
:109620000006C2F2000AC6F800E0CAF800C041F223
:10963000342A19463E683B692C48C2F2000A0133BD
:10964000CAF80060FEF7DEFEFFF7BBB90020014656
:109650000122F9F7C1FD322401F088F9FFF7D4B9EE
:10966000234B4CF6CD451B68CCF6CC45A5FB03053A
:10967000AD0805EB8505AB420CBF04250125FFF7BE
:10968000FBB91C4800F096FDFFF7E2BA44DA000887
:1096900094DB000848DC000838C9000820DB00081B
:1096A000C0DB000820DC000820120020F4DA0008EB
:1096B0000412002088DA000818DA00083CDB0008F1
:1096C00024120020D0DA00080C12002070010020C3
:1096D000C0DD000894E000082CDE000830D100084E
:1096E000C0C80008E0DD00083CDD000894DD00088B
:1096F00048120020803E0020A8E00008A448FEF7A1
:10970000C9FDA448FEF7C6FD41F2F41E4FF0000A61
:10971000C2F2000ECBF804A08BF83CA09E499F48F3
:10972000CEF800A0CDF814A0FBF74AFAFFF7F2BA82
:1097300041F24821C2F20001D2F804E00B689E45D4
:109740007FF492AAFFF791BAFEF768FB944B0022D0
:109750001A60FFF74EB917221A60FFF7F9BB3B22D8
:109760001A606AE400221A60BDE400221A60A1E4D3
:1097700041F24826C2F20006DAF804C033689C457C
:109780007FF432AF31E7874A40F2CC1A0023C2F2AD
:10979000000A18461360FF23CAF80030F9F79CFE50
:1097A000FFF736BB7F4A40F2CC1A0023C2F2000A10
:1097B00018461360FF23CAF80030F9F78DFEFFF753
:1097C00012BB13A800F0F6FC16E541F2482EC2F2D7
:1097D000000EDEF80030DDF850E09E457FF418AD55
:1097E00017E541F23C2EC2F2000E6F48CEF8003071
:1097F000FEF750FD6748FEF74DFDF0E5694A40F27F
:10980000CC160023C2F2000618461360FF23336013
:10981000F9F762FE36E66548654CFEF73BFD5D48AC
:10982000FEF738FDFEF7E4BF6248FEF733FD594806
:10983000FEF730FDFEF7A2BF132D54D80FF2040A35
:109840005AF825F0058F0008EB8E0008C78E000837
:10985000FD8F0008A78F0008838F0008398F00084C
:109860009B90000823900008CF9000082B8E0008E2
:10987000938E0008798E00085F8E0008458E0008E0
:10988000AD8E0008018E0008D78D0008A39800084F
:10989000058D0008002046490422FAF7E9FDFEF78D
:1098A0007EBF41F23C2AC2F2000A40F2CC1EDAF836
:1098B0000030D3F1010338BF0023C2F2000E184676
:1098C000CAF800300025FF23CEF800303224F9F723
:1098D00003FE04950225FFF719BAF7F765FCFBF7BD
:1098E000A1F9FEF728BF0026049632243546FFF77B
:1098F0000DBA3148FEF7CEFC2648FEF7CBFCFEF74A
:10990000D9BF2E48FEF7C6FC2248FEF7C3FC00F084
:1099100063F8FEF75EBF2A48FEF7BCFC1D48FEF761
:10992000B9FC00F079FB2748FEF7B4FC1948FEF7B4
:10993000B1FC2068FAF7C4F92348FEF7ABFC1548E0
:10994000FEF7A8FC00F07EFFFEF73BBF1F48FEF7C6
:10995000A1FC1048FEF79EFCFEF7A7BF1C48FEF7CF
:1099600099FC0C48FEF796FCFEF79ABF1948FEF7E3
:1099700091FC0848FEF78EFCFEF78DBF3046394655
:109980000422FAF78FFD00287EF480AFFEF778BF3F
:10999000C4D9000838C900080CDA000800DA000849
:1099A000301200203C120020F0DB0008B0D8000884
:1099B000D0010020ACD700087CD9000864D800088A
:1099C000F4D7000814D8000840D8000850D900087F
:1099D00030D900080CD9000830B5104B1B6887B08F
:1099E00013B9002007B030BDBF2069461822FAF72E
:1099F0003FFD0028F5D00A486A46002314785178C4
:109A000095781C50C1EB01111C18083305EB81013E
:109A10000332402B6160F1D10120E3E75C040020B8
:109A2000A43E002070B548F6890686B0114C6A46FF
:109A30000023C8F688061819195940681170A6FB4A
:109A400000514909C1EB0115A0EB850008335170A5
:109A500090700332402BEED1074B186838B1BF200D
:109A600018226946FAF71EFD003018BF012006B023
:109A700070BD00BFA43E00205C040020F0B40023B1
:109A80001B4D02E00833402B22D05C5914F0800FAC
:109A900003EB0506F6D076689642F3D1C4F3C2060E
:109AA00004F0070704F0400418B1D4F1010438BFF2
:109AB0000024002CE6D0BE420DD8B14234BF0026AF
:109AC0000126B94288BF0026002EDBD0012000E02D
:109AD0000020F0BC7047B9428CBF00270127B1427B
:109AE00034BF3E4647F00106002ECBD0EEE700BF64
:109AF000A43E0020704700BF70B54FF44064C4F22C
:109B0000020404266420F7F785FE66834FF40C7088
:109B1000F7F780FE284D26831420F7F77BFE0026FA
:109B20004FF496732B60344603E004B92C682B681D
:109B3000ABB14FF440600421C4F20200F6F794FE8A
:109B4000D6F1010338BF0023002C08BF00230028F2
:109B5000EBD0002BEBD02E682B68002BE9D1322004
:109B6000002E18BF002C0CBF0025012515D0F7F7DB
:109B700051FE4FF440600421C4F20200F6F774FE77
:109B800005467820F7F746FE6B1E5842C6EB0404E4
:109B900058411E2C98BF002070BDF7F73BFE4FF4D4
:109BA00040600421C4F20200F6F75EFE7820F7F769
:109BB00031FE284670BD00BF003E002038B54FF48E
:109BC0004064C4F20204042505206583F7F722FEF1
:109BD00025830A20F7F71EFE29462046F6F744FEA5
:109BE00004463220F7F716FE621E5042504138BD3F
:109BF00070B5082401250026FFF7E0FF6B0000B1D7
:109C00002E43013CDDB2F7D1304670BD38B54D1E54
:109C10000446EDB239B101354519FFF7E9FF04F803
:109C2000010BAC42F9D138BD2DE9F0414FF440664B
:109C3000804608250124C4F2020604270AE0052014
:109C4000F7F7E8FD502037836400F7F7E3FD013DA7
:109C5000E4B20ED0502014EA080F7783EFD1F7F763
:109C6000D9FD052037836400F7F7D4FD013DE4B248
:109C7000F0D1BDE8F08100BF38B54D1E0446EDB20D
:109C800039B10135451914F8010BFFF7CDFFAC428E
:109C9000F9D138BD10B50446FFF72EFF024680B952
:109CA000234603F8012B0133627003F8012B03F8FC
:109CB000012B03F8012B03F8012B03F8012B1A7079
:109CC00010BD3320FFF7B0FF20460821FFF79EFFAD
:109CD000FFF712FF012010BD70B5124B1A6882B059
:109CE0000AB102B070BD012468464FF440651C60A3
:109CF000C4F20205F6F7AEFD08202146F6F758FF3C
:109D0000042602232846694600968DF804408DF803
:109D100006408DF807408DF80530F6F73FFD2E839D
:109D2000DFE700BF5012002000B583B06846F6F7A9
:109D300091FD04200121F6F73BFF4FF480724FF4B0
:109D40000060002369460092C4F2020001228DF8EF
:109D500005308DF804208DF806308DF80730F6F7C1
:109D60001DFD4EF27000C0F60000FEF793FA4CF6AF
:109D70003810C0F60000FEF78DFA03B000BD00BF3A
:109D800010B50B4C2368012B10D04FF400604FF43A
:109D900080710122C4F20200F6F76CFD0548FEF75F
:109DA00079FA0548FEF776FA0123236010BD00BF5B
:109DB000D401002084E0000838C9000810B50A4C1E
:109DC000236883B14FF400604FF480710022C4F225
:109DD0000200F6F74FFD0548FEF75CFA0448FEF76F
:109DE00059FA0023236010BDD401002098E0000838
:109DF00038C90008F0B583B06846FDF703FD60B3CD
:109E00001A4A1B4B10681968013010609DF8052034
:109E100031B302F001021749BDF80170BDF803C06B
:109E20001A6000239DF8004018460E4602E00130FB
:109E3000782B12D0CA5C0633A242F8D100EB400264
:109E400006EB4202B2F80150BD42F0D1B2F8032055
:109E5000624503D00130782BECD1FF2003B0F0BD78
:109E600012F00102D7D001221A60F6E75812002042
:109E7000541200205C1200202DE9F04FDFF894818D
:109E80004E4D002783B001263C46C2462846F9F7CE
:109E900083FE2846FEF7FEF94948FEF7FBF96846BF
:109EA000FDF7B0FC04EB440908EB49090AEB070590
:109EB0004846FDF7A7FC0028FAD06A7912F00102A3
:109EC000F6D1D4B399F80010134602E00133A3424F
:109ED00031D018F80200884202F10602F6D103EBF5
:109EE000430C0AEB4C0CB9F80100BCF801E08645C4
:109EF000ECD1B9F803E0BCF803C0F445E6D1FF2B80
:109F000019D00022134602E00133A342D0D018F842
:109F100002C08C4502F10602F6D103EB430C0AEBBA
:109F20004C0CBCF801B08345EED1BCF803C0F4453D
:109F3000EAD1002BBCD1142E37D0731E122B3BD884
:109F4000DFE803F02F2D2B29272523211F1D1B19A7
:109F5000171513110F0A31001A4D01340136063757
:109F600094E7194DF9E7194DF7E7194DF5E7194D44
:109F7000F3E7194DF1E7194DEFE7194DEDE7194DED
:109F8000EBE7194DE9E7194DE7E7194DE5E7194DFD
:109F9000E3E7194DE1E7194DDFE7194DDDE7194D0D
:109FA000DBE7194DD9E7194DD7E71948F9F7F4FD63
:109FB000012003B0BDE8F08F004DCEE7C0E00008FF
:109FC00038C9000888E2000868E2000848E2000892
:109FD0002CE2000810E20008F0E10008D0E10008DF
:109FE000B4E1000898E1000884E1000870E100088D
:109FF0005CE1000848E100082CE1000810E10008DD
:10A00000F4E00008D8E00008D0E00008ACE0000868
:10A01000A4E200085C120020F0B5124B186883B06F
:10A02000E8B10025104F04262C460522304669462B
:10A03000FAF71EFA9DF800C0BDF80110BDF8032024
:10A0400007F805C004EB440307EB4303013405366E
:10A050000635142CA3F80110A3F80320E5D103B0B2
:10A06000F0BD00BF5C0400205C120020F0B5114B75
:10A07000186883B0E0B100250F4F04262C4604EB8E
:10A08000440307EB43037A5DB3F801E0B3F8033010
:10A090008DF800203046052269460134ADF801E014
:10A0A000ADF80330B6180635FAF7FCF9142CE6D1F2
:10A0B00003B0F0BD5C0400205C12002010B582B03B
:10A0C00004460B460092D02000222146FDF740FABC
:10A0D000D0F1010038BF002002B010BD10B582B031
:10A0E00004460B460092D02000222146FDF7AEFA2E
:10A0F000D0F1010038BF002002B010BD30B583B0F0
:10A10000FDF7D2F93F200DF107010122FFF7D6FF3D
:10A11000054620B301240720244B0DEB0001224605
:10A120001C60FFF7CBFF10B39DF80730002B29D13F
:10A1300000200DF107010122FFF7C0FF0446B0B176
:10A140009DF807301A0619D503F07F0300200DF1A2
:10A15000070101228DF80730FFF7C0FF0EE00E2047
:10A160000DF107010122FFF7A9FF044618B90024E9
:10A17000204603B030BD9DF807306BB90C4B01226F
:10A180001A60F5E7072000230DEB000122468DF849
:10A190000730FFF7A3FFCBE70E200DF107010122E7
:10A1A0008DF80750FFF79AFFE8E700BFDC120020A8
:10A1B000D41200202DE9F04F434B1B6889B01BB926
:10A1C000184609B0BDE8F08F836802690193C3683F
:10A1D00041690293466807688069013246F2676305
:10A1E000C6F2666303926439049183FB06B9019950
:10A1F000DDF80CB0019A059083FB078A83FB0BBC4A
:10A2000083FB0118DDF810B00299DDF80CE0D017DF
:10A21000FD1783FB0121029A009183FB0BB3DDF84C
:10A2200010B0C5EBAA05D1174FEAEE724FEAEB7EEC
:10A2300005EB850BC0EBA800F417DDF80080A7EB59
:10A240004B0B019FC4EBA90400EB8009C1EBA801F3
:10A25000A7EB4909029F01EB8108C2EBAC02A7EB17
:10A260004808039F04EB840A02EB820CCEEBA303A5
:10A27000A6EB4A06A7EB4C0C049F06EB041603EB77
:10A28000830E059C8DF81960A7EB4E0E09EB0019A3
:10A2900008EB01180CEB021C0BEB051701340EEB5D
:10A2A000031E002006A907228DF818708DF81A9059
:10A2B0008DF81B408DF81C808DF81DC08DF81EE0B8
:10A2C000FFF70CFF7DE700BFD41200202DE9F04F0F
:10A2D000394B1B688BB004461BB900200BB0BDE89E
:10A2E000F08F002008A90722FFF7E8FE0028F4D02D
:10A2F0009DF825A09DF820709DF826809DF823905C
:10A300009DF82430CDF818904FEA1A1B4FEA171C1D
:10A310000BEB8B0B4FEA1819CDF81CB00CEB8C0C27
:10A320009DF82220CDF800C009EB890908F00F083C
:10A33000DDF81CC005930AF00F0ACDF80890CDF89F
:10A3400004809DF82150DDF81490DDF80480CDF8EC
:10A350000CA011090AEB4C0ADDF808C002F00F024C
:10A3600001EB81012E091B0909F00F0B02EB4101E2
:10A3700008EB4C09069ADDF80080049305F00F0500
:10A3800007F00F0706EB860603EB830305EB460693
:10A3900002F1FF3C07EB48070BEB43030AF1FF35E3
:10A3A00009F1640227606660A160C4F818C0E36028
:10A3B0002561626192E700BFD412002000B50E4B08
:10A3C0001B6883B053B1FF23C0F20203984207D841
:10A3D00000220120094B1A6003B000BD1846FBE7BC
:10A3E0000122DF200DF10701FAF742F89DF807205E
:10A3F0000A2A88BF0022EDE75C040020D812002062
:10A4000000B5094B094A1B68106883B08DF8073006
:10A4100040B1DF2001220DF10701FAF743F80030C7
:10A4200018BF012003B000BDD81200205C0400203A
:10A4300041F2D823C2F200031868704710B541F208
:10A44000D824C2F200042060FFF7DAFF206810BDB4
:10A4500000B50D4B1B6883B0FF200BB903B000BDE6
:10A46000112001A90222FFF729FE0028F6D09DF84D
:10A470000500064B9DF804201B68C0F3400040EA2D
:10A480004200C01AEAE700BFD4120020D812002010
:10A490000649074A074B9A42BEBF51F8040B42F8DF
:10A4A000040BF8E7044880470448004788E40008A4
:10A4B00000000020B402002099A50008DD0100087A
:10A4C0003349344A002301E041F8043B9142FBD375
:10A4D000FEF70EF9FEE7FEE7FEE7FEE7FEE7FEE722
:10A4E000FEE7FEE7FEE7FEE7FEE7FEE7FEE7FEE744
:10A4F000FEE7FEE7FEE7FEE7FEE7FEE7FEE7FEE734
:10A50000FEE7FEE7FEE7FEE7FEE7FEE7FEE7FEE723
:10A51000FEE7FEE7FEE7FEE7FEE7FEE7FEE7FEE713
:10A52000FEE7FEE7FEE7FEE7FEE7FEE7FEE7FEE703
:10A53000FEE7FEE7FEE7FEE7FEE7FEE7FEE7FEE7F3
:10A54000FEE7FEE7FEE7FEE7FEE7FEE7FEE7FEE7E3
:10A55000FEE7FEE7FEE7FEE7FEE7FEE7FEE7FEE7D3
:10A56000FEE7FEE7FEE7FEE7FEE7FEE7FEE7FEE7C3
:10A57000FEE7FEE7FEE7FEE7FEE7FEE7FEE7FEE7B3
:10A58000FEE7FEE7FEE7FEE7FEE7FEE7FEE7000088
:10A59000B4020020E83E00204FF46D42CEF20002EB
:10A5A0004FF46053D2F88810C4F2020341F47001F2
:10A5B000C2F888101968002241F0010119609A6000
:10A5C000186843F2100120F08470C2F2004120F4B8
:10A5D000803018605960196882B021F480211960B8
:10A5E000DA60009201921A6842F480321A6003E045
:10A5F000009AB2F5C06F09D01A6802F400320192D5
:10A60000009A01320092019A002AF1D04FF460536F
:10A61000C4F202031B6813F4003308BF019301D096
:10A6200001230193019B012B00D0FEE74FF46053FF
:10A63000C4F202034FF4E042196CC4F2000241F08C
:10A6400080511964116841F4804111609A6822F0C8
:10A65000F0029A609A6822F460429A609A6842F422
:10A6600080529A601A6822F080721A6019684FF45A
:10A6700060528801C4F20202F8D445F20843C0F2E5
:10A6800041735360136843F08073136011684FF493
:10A6900060538901C4F20203F8D54FF47052C4F23A
:10A6A0000202116841F4407141F002011160126828
:10A6B00002F00702022A00D0FEE79A6822F00302A5
:10A6C0009A609A6842F002029A609A6802F00C025C
:10A6D000082AFAD14FF46D43CEF200034FF0006226
:10A6E0009A6002B0704700BF4FF46053C4F2020397
:10A6F0009A6802F00C02042A14D0082A1CBF4FF4F6
:10A700001052C0F2F40212D04FF46053C4F20203AC
:10A7100018499B68C3F30313CB5C22FA03F2164B70
:10A720001A6070474FF49052C0F27A02ECE7586812
:10A73000596810F4800F586815BF4FF490534FF4C8
:10A740001053C0F27A03C0F2F40301F03F01B3FBEF
:10A75000F1F24FF46053C4F20203C0F388105B6857
:10A76000C3F30143013302FB00F25B00B2FBF3F2DF
:10A77000CAE700BFD8010020E801002000B585B07D
:10A7800001A802A903AAF9F765FD10B9FF2005B0D9
:10A7900000BD029B002BF9D1024B1868039B181ACD
:10A7A000F5E700BFE012002000B50E4B1B6883B038
:10A7B00053B1FF23C0F20203984207D800220120C0
:10A7C000094B1A6003B000BD1846FBE70122DF20E9
:10A7D0000DF10701F9F74CFE9DF807200A2A88BF02
:10A7E0000022EDE75C040020E012002000B5094BD8
:10A7F000094A1B68106883B08DF8073040B1DF202C
:10A8000001220DF10701F9F74DFE003018BF0120BC
:10A8100003B000BDE01200205C04002041F2E02300
:10A82000C2F200031868704710B541F2E024C2F28A
:10A8300000042060FFF7DAFF206810BD0920F9F757
:10A840007BBD00BF00B5144B1B6883B02BB1AA20A1
:10A8500012491022F9F70CFE50B910220F48104986
:10A8600000F040FE0F4B01221A60002003B000BD33
:10A87000BA2001A90222F9F7FBFD0028EDD09DF8CE
:10A8800004109DF80520074B01202D291A60EDD1F9
:10A8900052421A600120E9E75C040020F001002028
:10A8A000B4E20008EC01002000B5134B1B68002B3C
:10A8B00083B01ADB2B228DF804208DF805300F4B66
:10A8C0001B6813B9002003B000BDAA200C49102258
:10A8D000F9F7E8FD0028F5D0BA20022201A9F9F71E
:10A8E000E1FD003018BF0120EDE75B422D228DF81D
:10A8F00004208DF80530E2E7EC0100205C04002024
:10A90000F001002040F2EC13C2F200031868704717
:10A9100010B5014604460A48FDF774FD04F10C0326
:10A92000182B0AD8074B1A68A24204D01C60FFF704
:10A93000BBFF012010BD012010BD002010BD00BFD5
:10A94000C4E20008EC01002040F2F010C2F2000066
:10A95000704700BF014608B540F2F010C2F2000097
:10A9600000F097FDBDE80840FFF79EBF40F2F010F1
:10A97000C2F20000FAF73CB970B5284A48F28013D9
:10A98000126882B0C7F65543CB1802AE4FF461612E
:10A9900001FB023346F8043D0546304600F036FA26
:10A9A0000369DA1E052A04460CD9022B2BD0092B89
:10A9B00010D18369C268D21A182A03DD53B983689B
:10A9C000022B07DC019B304603F56163019300F025
:10A9D0001DFA044663696B6123692B61E36804F126
:10A9E0000C00EB6007C8013102F26C72F6F778FBDD
:10A9F000A861236A2B62A368AB6063686B602368FD
:10AA00002B6002B070BD8369C268D21A182AE1DDDA
:10AA1000002BD7D18368012BD4DCDBE7EC010020CD
:10AA200046F2700048F2200108B5C4F20200C2F2FA
:10AA30000001F5F76BFE60B146F2700048F22001AC
:10AA4000C4F20200C2F20001F5F78CFE014B0022B5
:10AA50001A6008BDE41200202DE9F047DFF834E168
:10AA60000646DEF80030002BFBD1002E00F08A8075
:10AA7000464D4748770007EB060CAC444FF0FF34D7
:10AA800015F802AC631C00EB440104F109098022B3
:10AA900012EA0A0F0CBF4FF027084FF043080133AA
:10AAA00052084B4521F8028FF2D104F1080115F844
:10AAB00003AC00EB410104F11109802212EA0A0FF4
:10AAC0000CBF4FF027084FF04308013352084B45A5
:10AAD00021F8028FF2D104F1100115F801AC00EB5E
:10AAE000410104F11909802212EA0A0F0CBF4FF04C
:10AAF00027084FF04308013352084B4521F8028FD5
:10AB0000F2D1033518346545BAD1002200EB430376
:10AB1000114699520232602AFBD14FF48060012421
:10AB20000021C4F20000CEF80040F6F7DDF846F24E
:10AB300070000021C4F20200F5F7BCFDBB19DB0078
:10AB4000303346F270004FF6F8711940C4F202003B
:10AB5000F5F7BAFD46F2700010212246C4F2020059
:10AB6000F5F7B4FD46F270002146C4F20200F5F795
:10AB7000A1FD4FF48060C4F200002146BDE8F0471B
:10AB8000F6F7B2B8334602483746BEE7EB1200206C
:10AB90006C150020E4120020D52810B409D80C78D8
:10ABA000054A00EB4000131814544A785A708A780A
:10ABB0009A7010BC704700BFE8120020F0B469B171
:10ABC0000A4D01EB410700230478EC54EC18467859
:10ABD000667086780333BB42A670F5D10AB9F0BC23
:10ABE00070470846F0BCFFF737BF00BFE8120020EF
:10ABF0002DE9F041644D9AB0002401A84FF400669D
:10AC0000C4F202062C60F5F725FE04200121F5F7B9
:10AC1000CFFF022703234FF04008304601A98DF8EB
:10AC200009308DF80870CDF804808DF80A408DF851
:10AC30000B40F5F7B3FD3A4606213046A6F81A80D8
:10AC4000F5F71EFE03A8F6F737F806A8F6F7A2F800
:10AC500038460121F5F7BAFF4FF400100121F5F74E
:10AC6000A7FF4FF480606A23C4F2000003A9049395
:10AC7000ADF80C40ADF81440ADF80E40F5F7D0FF3C
:10AC80004FF4806060230126C4F2000006A9ADF8ED
:10AC90001830ADF81A600894ADF82440F6F732F891
:10ACA0004FF48060C4F200000821F6F77DF84FF4FD
:10ACB0008060C4F200003146F6F708F84FF4806077
:10ACC000C4F200003146F6F777F84FF480604FF495
:10ACD00000713246C4F20000F6F78CF80F22684685
:10ACE0008DF800208DF801408DF802408DF803604A
:10ACF000F5F7AEFA0BA8F5F7CBFC46F2700021464B
:10AD0000C4F20200F5F7D6FC46F27000C4F202006D
:10AD1000F5F796FB40F23443C4F200030C934FF472
:10AD2000006312934FF4005313934FF4A2530F9305
:10AD30004FF4806311934FF4403315934FF0206329
:10AD40000B9346F27000114B1494C4F202000BA94D
:10AD50001094CDF838800D93169417961894199482
:10AD60002746F5F761FC8DF82C408DF82D408DF8C5
:10AD70002E402B68002BFCD10BA8D6210122FFF717
:10AD80001DFF1AB0BDE8F081E41200206C15002010
:10AD900000210A2200F046BC08B5074B044613B157
:10ADA0000021AFF30080054B1868836A03B1984710
:10ADB000204601F071F800BF00000000DCE200084E
:10ADC00070B50E4B0E4DED1AAD1000241E4603E07B
:10ADD00056F8242090470134AC42F9D101F05EF8D6
:10ADE000084D094BED1AAD1000241E4603E056F83D
:10ADF000242090470134AC42F9D170BDAC02002050
:10AE0000AC020020B0020020AC02002038B5074B95
:10AE10001C68E36B05461BB9242000F00DF8E063C5
:10AE2000E16B2846BDE8384000F002B8640200201B
:10AE3000002200F0C3B80000024B0146186800F081
:10AE400047BA00BF6402002010B5002302E0CC5CCA
:10AE5000C45401339342FAD110BD8218034601E075
:10AE600003F8011B9342FBD1704700002DE9F74F17
:10AE7000064600F09FFF40F2B1739E42024640F347
:10AE800096806FF4F663F318A6F2B2719B1040F24D
:10AE90006D1505FB0135A6F26D716FF0630391FB33
:10AEA000F3F36FF4C861ED1871184FF4C87391FB98
:10AEB000F3F16D18642196FBF1FC01FB1C6C96FB11
:10AEC000F3F103FB1161D1F10101466006F00306C5
:10AED00038BF002101960346022407261F7A4A2F15
:10AEE00011D15F69019805EB070810B9BCF1000F9B
:10AEF00000D121B13B2FD4BF0027012700E00F462E
:10AF00004744013F3FE0442F02D15F69EF193AE027
:10AF1000019F37B9BCF1000F0CBF89464FF0010902
:10AF200000E089462348D3F80CA04FF0300808FB16
:10AF300009090127A84605E009EB870B01375BF8F3
:10AF400004BCD8445745F7DB08F1040797FBF6FB30
:10AF500006FB1B7B5F691869BAF1010FB8BF4FF0A0
:10AF6000010A0AF1FF3AB7EB0B0748BF073700F1B8
:10AF7000FF3B072000FB0B7759F82A9000E0073FC2
:10AF80004F45FCDA47449869DFF82C8008FB070737
:10AF9000186A013C074443F81C7F9FD1936BD16929
:10AFA0009942ACBF002301231360012000E0002080
:10AFB000BDE8FE8FE0E20008805101002DE9F84372
:10AFC00080460C46174600F0F5FED8F800109B4A64
:10AFD00091FBF2F3064602FB131104E001F5A831E0
:10AFE00001F5C071013B0029F8DB4FF4616091FB72
:10AFF000F0F200FB12113C20A26091FBF0F200FB8A
:10B000001211626021601A1D072192FBF1F001FB11
:10B010001022002AB8BF0732002BA26140F2B2759D
:10B020004FF4C8704FF0640CDFF81C9217DBA907CF
:10B0300004D195FBFCF20CFB125242B995FBF0F1E6
:10B0400000FB1151D1F1010138BF002100E00121C5
:10B0500059F82120934218DB01359B1AE7E7013D9F
:10B06000AA0704D195FBFCF20CFB125242B995FBE6
:10B07000F0F100FB1151D1F1010138BF002100E0D6
:10B08000012159F821209B18E9D4A5F26C72626164
:10B090006B4AE3614FF0300909FB0129002222616C
:10B0A00002E001319B1A2161216959F82120934264
:10B0B000F7DA0133E360002F40F0BA8000F0A6FC1D
:10B0C000604B1B681BB373689D4205D13168D8F88B
:10B0D0000030F26931B90CE02846FFF7C7FE0028BE
:10B0E000F4D110E093420CDBB26B934209DA0123F6
:10B0F0000BE09342FBDAB26B9342ACBF0023012317
:10B1000003E0002301E04FF0FF33236200E02762F9
:10B11000236A2568012B0CBFF36B336A4FF461601F
:10B1200093FBF0F200FB12333C2093FBF0F100FBA9
:10B1300011336068411AA0686160EB1A821A3B2BD8
:10B140002360A26003DD013161603C3B04E0002B21
:10B1500003DA013961603C33236063683B2B03DD14
:10B160000132A2603C3B04E0002B03DA013AA2600A
:10B170003C336360A368172B1FDDE2690132E26193
:10B18000A2690132062AC8BF0022A261E268183B08
:10B190000132A3602369E26059F823108A4244DD3A
:10B1A0000133521A0C2BE26023613ED16269002305
:10B1B000013223616261E36137E0002B35DAE26935
:10B1C000013AE261A269013A48BF0622A261E2683F
:10B1D0001833013AE260A3603ABB2369013B01D412
:10B1E00023611EE00B23236163695A1E12F0030FD3
:10B1F000626103F26B7305D1642293FBF2F102FBEF
:10B20000113252B94FF4C87293FBF2F102FB1133C1
:10B21000D3F1010338BF002300E0012303F5B67327
:10B22000E361236959F82330E36000F0F0FB01E0AB
:10B23000002323622046BDE8F88300BF805101004F
:10B24000E0E20008F43D002040E3000830B50029AA
:10B250003BD051F8042C0B1F1C49002AB8BF9B1887
:10B260000A6812B95A600B6030BD93420CD219685B
:10B270005818904203D15A588918426819605A6088
:10B28000124A136030BD0A46516809B19942FAD991
:10B29000146815199D420AD11B68E318D01888421A
:10B2A000136012D108681B1813604B680CE002D9B8
:10B2B0000C23036030BD18681C188C4203D10C6845
:10B2C0004968001918605960536030BDF03D002096
:10B2D000F8B5CD1C25F0030508350C2D38BF0C251D
:10B2E000002D064645DB8D4200D242E0234B1B6811
:10B2F0001C4612E02268521B0DD40B2A02D9226090
:10B30000A4181EE0A34203D163681C4A136021E025
:10B3100062685A601EE023466468002CEAD123E08C
:10B320003046214600F06AF838602946304600F081
:10B3300065F8431C01461CD0C41C24F0030484425D
:10B3400001D1256006E03046611A00F057F801305F
:10B35000F7D10EE004F10B00231D20F00700C31A03
:10B360000AD05A42E250F8BD054F3B68002BDCD1B1
:10B37000D6E70C2333600020F8BD00BFF03D00206D
:10B38000EC3D00201A4B10B51C68A36BD3B91820F4
:10B39000FFF752FD43F20E33A06303804AF6CD332C
:10B3A000438041F2342383804EF26D63C3804DF6B7
:10B3B000EC630381052343810B2383810122002356
:10B3C000C0E90423A46B0B49206962690A4B41431D
:10B3D00003FB0212A0FB03015118012200231218E3
:10B3E00043EB0103C4E9042323F0004010BD00BF78
:10B3F000640200202DF451582D7F954C38B5064C31
:10B40000002305460846236000F02CFD431C02D1B2
:10B41000236803B12B6038BDE43E00200EB400B5B4
:10B420009CB04FF40271ADF814106FF000411DABE9
:10B43000049107914FF6FF71ADF81610084953F8C3
:10B44000042B029006900868019302A900F0E6F927
:10B45000029B00221A701CB05DF804EB03B0704729
:10B4600064020020C9B2034610F8012B12B18A42CF
:10B47000F9D102E0002918BF00231846704710F8E0
:10B48000012B11F8013B012A28BF9A42F7D0D01AAC
:10B490007047034611F8012B03F8012B002AF9D15C
:10B4A0007047034613F8012B002AFBD1181A013804
:10B4B000704770B5A2B108E0012A03D128781B7843
:10B4C000C01A70BD013A002CF8D00B460546002A80
:10B4D000F4D010F8016B1C780131B442ECD0EDE7E8
:10B4E000104670BD30B50139034609E011F8015F1F
:10B4F00003F8015B013A1C4615B99B18002205E0D0
:10B500001C46002AF2D1F8E704F8012B9C42FBD13B
:10B5100030BD00002DE9F74F01904148D0F8009070
:10B520000846044614F8015B09EB050620467778C7
:10B5300007F00807FFB2002FF3D12D2D03D114F827
:10B54000015B012704E02B2D04BF244614F8015BA6
:10B55000002B5ED0102B08D158E02078782801D03D
:10B5600058284ED1657810230234002F0CBF6FF09D
:10B5700000404FF00040B0FBF3FA002603FB1A082E
:10B58000304609EB050C9CF801C00CF0040B5FFA87
:10B590008BFBBBF1000F01D0303D0BE01CF0030C26
:10B5A0001BD0BCF1010F14BF4FF0570C4FF0370CFC
:10B5B000CCEB05059D4210DAB6F1FF3F0AD05045AD
:10B5C00006D801D1454503DC03FB0050012601E00C
:10B5D0004FF0FF3614F8015BD3E7731C0AD1002F3C
:10B5E00001990CBF6FF000404FF0004022230B6028
:10B5F00022B912E007B140427AB106B1611E116072
:10B600000BE03025002BB0D10823AEE7302DACD1B4
:10B61000A3E7302DA1D00A23A7E7BDE8FE8F00BF26
:10B620006802002030B51346044A05460C461068EF
:10B6300029462246BDE83040FFF76CBF6402002077
:10B640002DE9F74F01903D48D0F800900846044698
:10B6500014F8015B09EB05062046777807F0080728
:10B66000FFB2002FF3D12D2D03D114F8015B012778
:10B6700004E02B2D04BF244614F8015B002B57D0A7
:10B68000102B08D151E02078782801D0582847D1D4
:10B690006578102302344FF0FF3ABAFBF3FA03FB4C
:10B6A0000AF000266FEA0008304609EB050C9CF80A
:10B6B00001C00CF0040B5FFA8BFBBBF1000F01D053
:10B6C000303D0BE01CF0030C1BD0BCF1010F14BF8C
:10B6D0004FF0570C4FF0370CCCEB05059D4210DABC
:10B6E000B6F1FF3F0AD0504506D801D1454503DCED
:10B6F00003FB0050012601E04FF0FF3614F8015B18
:10B70000D3E7731C05D1019922230B60304622B97F
:10B7100012E007B140427AB106B1611E11600BE040
:10B720003025002BB7D10823B5E7302DB3D1AAE7D8
:10B73000302DA8D00A23AEE7BDE8FE8F68020020B6
:10B7400030B51346044A05460C4610682946224681
:10B75000BDE83040FFF774BF640200202DE9F047D8
:10B760008D68AB4281460C4692461F463FD38A897C
:10B7700012F4906F39D0266809696369C1EB060835
:10B7800003265E43022508F1010302F4806296FB62
:10B79000F5F6DB1912B29E4238BF1E4682B1314621
:10B7A000FFF796FD054600B913E021694246FFF711
:10B7B0004BFBA38923F4906343F08003A3810CE047
:10B7C000324600F022FB054638B948462169FFF7AA
:10B7D0003DFD0C23C9F8003018E025616661454441
:10B7E000C8EB06062560A6603D46AF4200D23D4646
:10B7F0002A462068514600F0EFFAA3685B1BA3605D
:10B8000023685D1925600020BDE8F087A38943F017
:10B810004003A3814FF0FF30BDE8F0872DE9F04FE2
:10B820009DB0064603938B8903F080031BB20D463F
:10B83000144663B10B6953B94021FFF749FD2860F5
:10B84000286110B90C233360D0E040236B610023E2
:10B85000099320238DF82930DFF89C81DFF89C9133
:10B8600030238DF82A3023469A4613F8012B1AB953
:10B87000BAEB040B0FD002E0252AF5D1F8E73046E9
:10B88000294622465B46FFF769FF013000F0A7809A
:10B89000099B5B4409939AF80030002B00F09F80CD
:10B8A00000234FF0FF3204930793059206938DF81F
:10B8B00053301A930AF1010A4FF0010B05E0C8EB6F
:10B8C00000000BFA00F00343049354464A482178E1
:10B8D000052200F073FA0AF1010A049B0028EED158
:10B8E000D90602D520228DF853201A0702D52B2223
:10B8F0008DF8532022782A2A03D0079B21460A205C
:10B9000010E0039A111D12680391002A01DB0792CF
:10B9100004E0524243F0020307920493013408E02A
:10B9200000FB03230C4601312278303A092AF7D96B
:10B93000079323782E2B19D163782A2B09D1039BE7
:10B940001A1D1B6803920234002BB8BF4FF0FF335F
:10B950000BE0611C00230A2001E000FB03230C46DE
:10B9600001312278303A092AF7D905932348217802
:10B97000032200F023FA40B14023C9EB000003FA90
:10B9800000F0049B03430493013414F8011B1C488A
:10B990008DF82810062200F011FA88B1194B33B93E
:10B9A000039B073323F007030833039313E003AB30
:10B9B0000093304604A92A46134BAFF3008007E0FA
:10B9C00003AB0093304604A92A460F4B00F092F8CF
:10B9D000431C074603D0099BDB19099343E7AB8956
:10B9E00003F040031BB20BB9099801E04FF0FF30A0
:10B9F0001DB0BDE8F08F00BF48E300084EE300082B
:10BA000052E30008000000005DB70008704770476F
:10BA10002DE9F04715461F468A680B69DDF820803E
:10BA20009A42A8BF13462B6091F8432006460C4665
:10BA30000AB101332B602368990602D52B680233C3
:10BA40002B60236813F0060916D094F8433022685F
:10BA5000003318BF0123920616D41EE0012330469E
:10BA600039465246C047013003D14FF0FF30BDE8A0
:10BA7000F08709F1010901E004F1190AE1682B6876
:10BA8000CB1A9945EADBE0E7E218302182F843104F
:10BA900094F84510023382F844103046394604F1D8
:10BAA0004302C0470130E0D023682A68E16803F010
:10BAB0000603042B08BFC2EB01052369A2680CBF73
:10BAC00025EAE57500259A42C4BFC3EB0203ED18D1
:10BAD0004FF000091A3408E0012330463946224667
:10BAE000C0470130C1D009F10109A945F4DB0020AC
:10BAF000BDE8F0872DE9FF470E7E0C9D6E2E914626
:10BB000080460C469A4601F1430200F0AF800FD800
:10BB1000632E1DD006D8002E00F0C080582E40F0B5
:10BB2000D0804FE0642E1CD0692E40F0CA8018E00F
:10BB3000732E00F0B78005D86F2E2BD0702E40F0FA
:10BB4000C08043E0752E25D0782E40F0BA8041E0C9
:10BB50002B681A1D1B682A6001F1420781F84230E8
:10BB6000B3E021682B6811F0800F02D0191D296005
:10BB700008E011F0400F03F10401296002D0B3F98D
:10BB8000005000E01D68002D45DA2D236D4284F839
:10BB9000433040E021682B6811F0800F02D0191D5E
:10BBA000296007E011F0400F03F10401296001D082
:10BBB0001D8800E01D68237E5F486F2B14BF0A2399
:10BBC000082324E081F845605B4807E00B6843F0F8
:10BBD00020030B607823594884F8453021682B688E
:10BBE00011F0800F03F104062E6000D003E04F0631
:10BBF00001D51D8800E01D68CE0744BF41F020013B
:10BC000021601DB9236823F0200323601023002145
:10BC100084F8431001E048480A236668002EA660B5
:10BC200003DB216821F00401216005B96EB104F144
:10BC30004201B5FBF3F603FB16550F46455D01F8CF
:10BC400001593546002EF4D100E01746082B0AD1E1
:10BC50002368DB0707D561682369994203DC302339
:10BC600007F8013C013FD21B226133E009682B68D1
:10BC700011F0800F05D0191D2960196863690B60E8
:10BC80000CE011F0400F03F10401296003D01968A2
:10BC900063690B8002E061691B68196000232361FE
:10BCA000174617E02B681A1D2A601F683846FFF7F1
:10BCB000F8FB63682061984288BF23612369636051
:10BCC00005E004F1420784F8426001232361002368
:10BCD00084F84330CDF800A04046214603AA4B46E5
:10BCE000FFF796FE013002D14FF0FF3021E04046D1
:10BCF00049463A462369D0470130F5D02368980772
:10BD00000ED4E068039B9842B8BF184611E00123A7
:10BD1000404649463246D0470130E5D0013502E081
:10BD2000002504F11906E168039BCB1A9D42EEDB66
:10BD3000E7E704B0BDE8F08759E300086AE30008CC
:10BD400030B5141E9BB0054604DA8B2303604FF018
:10BD5000FF301DE04FF40272ADF80C200091049109
:10BD600001D0611E00E021464FF6FF72029105915D
:10BD7000ADF80E2028461A4669461E9BFFF74EFD79
:10BD8000431C01DA8B232B6014B1009B00221A7034
:10BD90001BB030BD73B50093054B06460D461446E7
:10BDA000186831462A462346FFF7CAFF7CBD00BF0C
:10BDB00064020020004870476C02002010B5C9B230
:10BDC0000346821803E0047801338C4203D0934287
:10BDD0001846F8D1002010BD814210B511D28C1840
:10BDE000A0420ED253428118E418CB1801E0A15CA6
:10BDF000995412F1FF32FAD210BDCC5CC454013315
:10BE000000E000239342F8D110BDF8B50646154670
:10BE10000C4621B91146BDE8F840FFF759BA1AB9E6
:10BE2000FFF714FA2C4612E000F013F8A8420ED2E5
:10BE300030462946FFF74CFA074638B121462A46D4
:10BE4000FFF702F830462146FFF700FA3C4620464D
:10BE5000F8BD51F8040C002802DA04390B58C01858
:10BE600004387047094A136863B118186946884254
:10BE700098BF106004D9064B0C221A604FF0FF33B4
:10BE800018467047034B1360EFE700BFF83D0020F2
:10BE9000E43E0020E83E0020FEE700BFF8B500BF0A
:10BEA000F8BC08BC9E467047F8B500BFF8BC08BC9B
:10BEB0009E46704765617374657220646174653A6B
:10BEC00020253034642D253032642D253032640D28
:10BED0000A000000536F00004D6F0000446900002D
:10BEE0004D690000446F000046720000536100007D
:10BEF0005375000054750000576500005468000039
:10BF00004443463737204572726F723A204869675A
:10BF1000682070756C7365203C3D20350000000082
:10BF20004443463737204572726F723A204869673A
:10BF3000682070756C7365203E3D2032350000002E
:10BF40004443463737204572726F723A20706172EF
:10BF500069747920503120696E636F727265637401
:10BF6000000000004443463737204572726F723A32
:10BF70002070617269747920503220696E636F722B
:10BF800072656374000000004443463737204572F1
:10BF9000726F723A2070617269747920503320692F
:10BFA0006E636F7272656374000000000000000031
:10BFB0000000000006090906000000000A040A0A41
:10BFC0001F110000110E1111110E000012090909B4
:10BFD00009060000040A0A0A090A0000000000001D
:10BFE0000000000000000000000000000000000051
:10BFF0000000000000000000000000000000000041
:10C000000000000000000000000000000000000030
:10C010000000000000000000000000000000000020
:10C020000000000000000000000000000000000010
:10C030000000000000000000000000000000000000
:10C0400000000000000000000000000000000000F0
:10C0500000000000000000000000000000000000E0
:10C0600000000000000000000000000000000000D0
:10C0700000000000000000000000000000000000C0
:10C0800000000000000000000000000000000000B0
:10C0900000000000000000000000000000000000A0
:10C0A0000000000000000000000000000000000090
:10C0B0000000000004040404000400000A0A000058
:10C0C0000000000000051F0A1F140000040E0C04ED
:10C0D000060E040009150E0E15120000040A0C15B8
:10C0E000120D000004040000000000000304080812
:10C0F000080403001804020202041800040A040AD7
:10C1000000000000000000040E0400000000000019
:10C11000000404080000000E000000000000000001
:10C1200000040000010202040408080006090909CD
:10C1300009060000040C0404040E00000C020204B2
:10C14000080E00000C020C02020C000002060A0F8E
:10C15000020200000E080C02020C000006080E0984
:10C16000090600000F010204040400000609060984
:10C170000906000006090907010600000000040086
:10C180000004000000000400000404080001020C88
:10C190000201000000000F000F000000000804036F
:10C1A000040800000E010204000400000609131533
:10C1B00017100F0000040A0A1F110000000E0A0CDD
:10C1C0000A0E00000007080808070000000E090911
:10C1D000090E0000000E080E080E0000000E080EEA
:10C1E000080800000007080B090700000009090FF4
:10C1F00009090000000E0404040E0000000E0202F3
:10C20000020C000000090A0C0A09000000080808D6
:10C21000080F000000111B151511000000090D0B7F
:10C2200009090000000E1111110E0000000E090E88
:10C2300008080000000E1111110E0201000C0A0C7A
:10C240000A09000000060804020C0000001F040494
:10C250000404000000090909090600000009090991
:10C2600006060000001115150A0A000000110A0454
:10C270000A11000000110A0404040000000F010666
:10C28000080F000006040404040406001008080453
:10C29000040202000C04040404040C00040A0A1141
:10C2A000110000000000000000001F000804000052
:10C2B0000000000000000C020E0F000008080E092C
:10C2C000090E0000000006080806000002020E1217
:10C2D000120E00000000040E0806000003040F0404
:10C2E00004040000000007090F010E0008080A0DF1
:10C2F0000909000004000C040404000002000E02FE
:10C3000002020C0008080A0C0A0900000C040404CC
:10C31000040400000000151F1515000000000A0DA0
:10C3200009090000000006090906000000000E09C6
:10C33000090E080000000E12120E020000000A0C86
:10C34000080800000000060C020C000000040F04A6
:10C3500004020000000009090B05000000000909A3
:10C3600006060000000015150E0A00000000090670
:10C37000060900000000090906061C0000000E0660
:10C38000080E00000204040804040200040404046B
:10C390000404040008040402040408000000000D62
:10C3A0001200000000040A0A0A0E0000000001004A
:10C3B0000100020002000300030004000400050065
:10C3C000050006000700080009000B000D000E0024
:10C3D000100012001400170019001C001F0021009B
:10C3E000240028002B002E003200360039003D00CA
:10C3F000420046004A004F00540059005E006300AE
:10C4000069006E0074007A00800086008C00930042
:10C410009900A000A700AE00B600BD00C500CD0089
:10C42000D500DD00E500EE00F600FF0025750000F8
:10C430004E6F6E65000000005261696E626F77009A
:10C440004661646500000000526F6C6C00000000E3
:10C450004578706C6F64650052616E646F6D0000AA
:10C46000536E616B6500000054656C65747970658E
:10C470000000000043756265000000004D617472A9
:10C480006978000044726F70000000005371756598
:10C49000657A65004E6F726D616C0000436C6F636E
:10C4A0006B320000080809090A0A0B0B0C0C0D0D71
:10C4B0000E0E0F000000000000000100030A000043
:10C4C0000100040A00000100080A00000101040B39
:10C4D0000C000101030B0C0001010C000000010124
:10C4E000030A0C000101040A0C000101080B000002
:10C4F0000101040B00000101030B0000000000001B
:10C5000000000100030A00000100040A000001010C
:10C51000080000000101040B0C000101030B0C00DA
:10C5200001010C0000000101030A0C000101040AD2
:10C530000C000101090000000101040B00000101D1
:10C54000030B00000000000000000100030A0000CF
:10C550000100040A00000100080A00000100050AA9
:10C5600000000101030B0C0001010C00000001019F
:10C57000030A0C000101050B00000101080B00007B
:10C580000101040B00000101030B0000000000008A
:10C5900000000100030A00000100040A000001017C
:10C5A000080000000100050A00000101030B0C0057
:10C5B00001010C0000000101030A0C000101050B40
:10C5C00000000101090000000101040B000001014D
:10C5D000030B000045534B4953544C46DC4E460078
:10C5E0005A45484E5A57414E5A49470044524549C8
:10C5F0005649455254454C0054474E414348564FC6
:10C60000524A4D0048414C42515A57D64C46500070
:10C610005A5745494E53494542454E004B445245B1
:10C6200049524846DC4E4600454C464E45554E560E
:10C630004945520057414348545A45484E525300C9
:10C64000425345434853464D55485200574553536E
:10C65000490000004F53534900000000524845492B
:10C660004E2D525548520000534348574142454EC3
:10C6700000000000000000000002000303000704A7
:10C68000010004010407020004020404020407027A
:10C69000000B03020403060304000404050505005F
:10C6A0000405020305020405050606010406070445
:10C6B0000700030703040707040801040805040929
:10C6C00001050908030000000D1A0F1A0E1A121AAC
:10C6D000161A131A191A111A171A151A181A141ADF
:10C6E0000D0010000E0012001600130019001100BA
:10C6F00017001500180014002800000054696D652B
:10C700006F757400290D0A004F4B00004552524FBF
:10C71000520000002D20000049504144445245532E
:10C7200053200000415020004D4F444520000000A0
:10C730006170000054494D45200000004649524DAB
:10C740005741524520000000434D442000000000A6
:10C750004854545020474554200000002D2D3E20C1
:10C76000000000003C30643E3C30613E0D0A000099
:10C770003C253032783E0000636170202225732210
:10C780002C22257322000000617020222573222CA8
:10C79000222573220000000074696D652022257334
:10C7A0002200000045535038323636204C4F474760
:10C7B00045520D0A0000000064D500086CD5000841
:10C7C00074D500087CD5000880D5000884D5000801
:10C7D00088D500088CD50008A0CE0008A8CE000897
:10C7E000B0CE000854E10008B4CE0008C0C800086C
:10C7F000C0C80008C0C80008C0C80008C0C80008F9
:10C80000040000000200000002000000020000001E
:10C810000200000094D50008A0D5000864D50008E7
:10C820006CD500088CD5000898D200089CD200086E
:10C83000A4D2000800D20008A4D50008A8D500089A
:10C8400054D3000854D3000854D30008ACD50008D2
:10C85000ACD50008ACD5000864D50008B0D50008F8
:10C8600044CC0008C0D500088CD5000864D5000869
:10C87000B0D5000844CC00088CD50008CCD5000801
:10C88000D4D50008DCD50008E0D50008E8D50008BC
:10C89000ECD5000804D200088CD5000861637469E7
:10C8A000766500002573256400000000485454504C
:10C8B0002F312E3020323030204F4B000D0A0D0A20
:10C8C000000000003C68746D6C3E0D0A0000000022
:10C8D0003C686561643E0D0A000000003C746974A8
:10C8E0006C653E003C2F7469746C653E0D0A000057
:10C8F0003C2F686561643E0D0A0000003C626F6475
:10C90000793E0D0A000000003C48313E0D0A00004F
:10C910003C2F48313E0D0A003C6120687265663D3F
:10C92000222F0000223E00003C2F613E266E6273E3
:10C93000703B266E6273703B0D0A00004D61696E9C
:10C94000000000006E6574776F726B004E6574773F
:10C950006F726B0054656D706572617475726500FD
:10C960006C6472004C445200446973706C617900CD
:10C97000616E696D6174696F6E730000416E696DFF
:10C980006174696F6E730000616D62696C696768DC
:10C9900074000000416D62696C6967687400000092
:10C9A00074696D657273000054696D65727300007F
:10C9B0003C503E003C7472206267636F6C6F723D46
:10C9C000236630663066303E0D0A00003C74723ECD
:10C9D0000D0A00003C74643E000000003C2F7464AB
:10C9E0003E0000003C696E70757420747970653D7E
:10C9F0002274657874222069643D220022206E61D1
:10CA00006D653D2200000000222076616C75653D59
:10CA10002200000022206D61786C656E6774683DAD
:10CA200022000000222073697A653D220000000088
:10CA30003C74643E3C627574746F6E2074797065EA
:10CA40003D227375626D697422206E616D653D22B1
:10CA5000616374696F6E222076616C75653D227327
:10CA600061766500223E5365743C2F627574746F65
:10CA70006E3E00003C2F74643E0D0A003C746162FF
:10CA80006C6520626F726465723D303E0D0A000075
:10CA90003C2F74723E0D0A003C74683E3C666F6E1B
:10CAA0007420636F6C6F723D626C75653E000000B0
:10CAB0003C2F666F6E743E3C2F74683E0D0A00007A
:10CAC0003C2F7461626C653E3C503E0D0A000000D4
:10CAD0003C627574746F6E20747970653D22737555
:10CAE000626D697422206E616D653D2261637469B7
:10CAF0006F6E222076616C75653D22003C2F627559
:10CB000074746F6E3E266E6273703B003C2F626FD2
:10CB100064793E0D0A0000003C2F68746D6C3E0D78
:10CB20000A0000003C73656C6563742069643D22F3
:10CB300000000000223E0D0A000000003C2F73653B
:10CB40006C6563743E0D0A003C6F7074696F6E20F3
:10CB500076616C75653D22002073656C6563746554
:10CB6000640000003C2F6F7074696F6E3E0D0A0008
:10CB7000266E6273703B3C696E70757420747970B8
:10CB8000653D22636865636B626F7822206E616D1C
:10CB9000653D2200222076616C75653D22616374DB
:10CBA0006976652220000000636865636B65640038
:10CBB0003C696E70757420747970653D2272616E87
:10CBC0006765222069643D220000000022206D6913
:10CBD0006E3D220022206D61783D22002220737478
:10CBE000796C653D2277696474683A0070783B001F
:10CBF00022206F6E696E7075743D22005F6F7574D0
:10CC00007075742E76616C75653D00002E76616CD2
:10CC10007565223E000000003C6F757470757420CD
:10CC20006E616D653D2200005F6F757470757422D2
:10CC30003E0000003C2F6F75747075743E0000005C
:10CC40002E0D0A0044656661756C74003135000074
:10CC50003C666F726D206D6574686F643D22474558
:10CC6000542220616374696F6E3D222F0000000022
:10CC70003C2F666F726D3E0D0A000000436F6C6FB3
:10CC8000727300003C74643E0D0A000036340000EC
:10CC9000266E6273703B266E6273703B266E627303
:10CCA000703B0D0A000000004C6561726E696E6792
:10CCB0002049522072656D6F746520636F6E7472C7
:10CCC0006F6C2E2E2E000000537769746368696EB6
:10CCD0006720706F776572206F6E2E2E2E00000019
:10CCE000537769746368696E6720706F7765722027
:10CCF0006F66662E2E2E00006F66666C696E65008C
:10CD00004D696E696D756D206C656E677468206F16
:10CD100066206B65792069732031302100000000A6
:10CD200054696D65736572766572207375636365AA
:10CD3000737366756C6C79206368616E6765642EC9
:10CD40000000000053657474696E67206F66206E82
:10CD500065772074696D65736572766572206661AA
:10CD6000696C65642E00000054696D657A6F6E65AC
:10CD7000207375636365737366756C6C7920636883
:10CD8000616E6765642E000053657474696E672078
:10CD90006F66206E65772074696D657A6F6E6520A9
:10CDA0006661696C65642E0047657474696E6720FE
:10CDB0006E65742074696D650000000044697370CD
:10CDC0006C6179696E672074656D706572617475E8
:10CDD00072652E2E2E00000053746F726564206DF4
:10CDE000696E696D756D2076616C75650000000077
:10CDF00054657374696E6720646973706C61792E11
:10CE00002E2E0000536176696E6720736574746915
:10CE10006E6773207065726D616E656E746C792ECD
:10CE20002E2E00006874747020706174683A202798
:10CE30002573270D0A0000006874747020706172F9
:10CE4000616D65746572733A20272573270D0A009A
:10CE50002F000000253032642E253032640000009F
:10CE60002534640025303264000000006163746979
:10CE70006F6E00006C6561726E697200706F77652D
:10CE8000726F6E00706F7765726F666600000000EB
:10CE9000736176656461746574696D650000000096
:10CEA00079656172000000006D6F6E7468000000AB
:10CEB000646179006D696E00736176657469636B96
:10CEC00065720000576F7264436C6F636B00000003
:10CED00056657273696F6E00454550524F4D0000A4
:10CEE000454550524F4D2056657273696F6E000074
:10CEF0005469636B65720000506F776572204F6EE6
:10CF000000000000506F776572204F6666000000D9
:10CF10004C6561726E2049522072656D6F74652098
:10CF2000636F6E74726F6C00656570726F6D64759F
:10CF30006D700000454550524F4D2064756D700076
:10CF40003C503E0D0A3C666F6E7420636F6C6F72CE
:10CF50003D677265656E3E003C5052453E000000E4
:10CF60002530347800000000202000003C2F505273
:10CF7000453E0000202020002F6E6574776F726B95
:10CF80000000000073617665776C616E0000000040
:10CF9000776C616E6D6F6465000000007373696487
:10CFA00000000000576F7264436C6F636B204E6526
:10CFB00074776F726B0000003C423E436F6E6E658B
:10CFC0006374696E6720746F2041636365737320B7
:10CFD000506F696E742C2074727920616761696E7C
:10CFE000206C617465722E3C2F423E003C423E53E1
:10CFF000746174696E672061732041636365737344
:10D0000020506F696E742C20747279206167616999
:10D010006E206C617465722E3C2F423E0000000051
:10D020007361766574696D6573657276657200000B
:10D030007361766574696D657A6F6E6500000000D6
:10D040006E657474696D6500495020616464726531
:10D050007373000045535038323636206669726D5E
:10D060007761726500000000574C414E00000000DF
:10D070005353494400000000266E6273703B266ED5
:10D080006273703B266E6273703B00004B657900E3
:10D0900054696D65207365727665720054696D65BB
:10D0A000207A6F6E652028474D54202B2900000000
:10D0B000476574206E65742074696D65000000001A
:10D0C0003C503E0D0A3C666F6E7420636F6C6F724D
:10D0D0003D7265643E3C423E000000003C2F423EF3
:10D0E0003C2F666F6E743E0D0A0000002F74656D54
:10D0F0007065726174757265000000007361766519
:10D1000074636F72727274630000000073617665FD
:10D1100074636F7272647331387878006469737005
:10D120006C617974656D706572617475726500000B
:10D130002E350000266465673B430000576F72641C
:10D14000436C6F636B2054656D70657261747572AA
:10D15000650000005254432074656D7065726174FF
:10D1600075726500445331387878000054656D70ED
:10D1700020636F7272656374696F6E20525443202E
:10D1800028756E697473206F6620302E35B0432980
:10D190000000000054656D7020636F7272656374E7
:10D1A000696F6E204453313878782028756E697421
:10D1B00073206F6620302E35B043290044697370A8
:10D1C0006C61792074656D7065726174757265004B
:10D1D0002F6C6472000000006C64726D696E000058
:10D1E0006C64726D61780000736176656175746F4F
:10D1F00000000000576F7264436C6F636B204C44F7
:10D20000520000004D696E004D6178004175746FE9
:10D210006D61746963206272696768746E657373A7
:10D2200000000000536574206173206D696E696DA4
:10D23000756D2076616C7565000000005365742083
:10D240006173206D6178696D756D2076616C7565AF
:10D25000000000002F646973706C617900000000A9
:10D2600073617665697469730000000073617665A7
:10D2700073796E63616D62690000000073617665A9
:10D280006272696768746E657373000073617665B6
:10D29000636F6C6F7273000072656400677265651E
:10D2A0006E000000626C75650000000073617665B9
:10D2B000646973706C61796D6F6465007361766524
:10D2C00074696E74657276616C00000074657374C5
:10D2D000646973706C61790073617665616C6C0070
:10D2E000576F7264436C6F636B20446973706C6139
:10D2F0007900000045532049535400005065726D79
:10D30000616E656E7420646973706C6179206F66FC
:10D310002022455320495354220000004469737071
:10D320006C6179204D6F64650000000055736520C5
:10D33000646973706C617920636F6C6F7273000045
:10D340004272696768746E6573732028312D3135B8
:10D35000290000003000000054656D70206469737E
:10D36000706C617920696E74657276616C00000082
:10D370005465737420646973706C617900000000F7
:10D380005361766520616C6C000000002F616E694E
:10D390006D6174696F6E730073617665616E696D3E
:10D3A0006174696F6E00000073617665636F6C6F06
:10D3B00072616E696D6174696F6E0000646566000C
:10D3C00073617665616E0000737025640000000073
:10D3D00066617625640000007361766563616E00A6
:10D3E00063737025640000006364656600000000DC
:10D3F000576F7264436C6F636B20416E696D61742B
:10D40000696F6E7300000000416E696D6174696F31
:10D410006E000000436F6C6F7220416E696D617425
:10D42000696F6E00616E256400000000646566250A
:10D43000640000003100000063616E25640000009C
:10D4400063646566256400002F616D62696C6967BD
:10D450006874000073617665616D62696D6F646503
:10D460000000000073617665616D62696C656473CC
:10D470000000000073617665616D62696F666673B6
:10D48000657400007361766561616E00617370257B
:10D49000640000006164656600000000576F7264FC
:10D4A000436C6F636B20416D62696C6967687400DF
:10D4B000234C4544730000004F6666736574206F0B
:10D4C00066207365636F6E64203D203000000000AD
:10D4D000416D62696C69676874204D6F6465000016
:10D4E00061616E256400000061646566256400006A
:10D4F0002F74696D657273007361766569640000ED
:10D50000610000006F00000066256400742564005F
:10D51000576F7264436C6F636B2054696D657273EF
:10D5200000000000696425640000000061256400BB
:10D530006F256400682564006D25640048545450CC
:10D540002F312E3020343034204E6F7420466F75CA
:10D550006E640000343034204E6F7420466F756E58
:10D56000640D0A004E616D650000000056616C7527
:10D570006500000059595959000000004D4D000048
:10D5800044440000686800006D6D000041637469E8
:10D590006F6E0000574C414E20436C69656E7400FD
:10D5A00041500000470000004200000036330000F8
:10D5B000446563656C65726174696F6E000000009C
:10D5C0004661766F7572697465000000536C6F7404
:10D5D0000000000041637469766500004F6E000032
:10D5E00046726F6D00000000546F0000486F757246
:10D5F00000000000010000000F0000001500000006
:10D60000070000000B000000070000000B000000F6
:10D61000070000000B0000000F00000014000000D5
:10D62000000000000F0000001400000000000000D7
:10D6300001000000000000000500000002000000E2
:10D640000B0000000C0000001A00000002000000A7
:10D650000B000000020000000B00000000000000B2
:10D66000100000001C000000280000003000000036
:10D6700001000000010000000000000002000000A6
:10D68000050000000C000000110000002200000056
:10D69000050000000C000000050000000C00000068
:10D6A000000000001000000010000000200000003A
:10D6B0002000000001000000010000000000000048
:10D6C00002000000050000000C0000001100000036
:10D6D00022000000050000000C0000000500000012
:10D6E0000C0000000000000000000000000000002E
:10D6F0000000000000000000010000000100000028
:10D700000000000003000000050000000C00000005
:10D710000F0000001E000000050000000C000000CB
:10D72000040000000B0000000000000010000000DA
:10D730001500000025000000250000000100000089
:10D740000100000000000000322E302E36000000E4
:10D750000D0A57656C636F6D6520746F20576F728B
:10D7600064436C6F636B204C6F67676572210000C8
:10D770002D2D2D2D2D2D2D2D2D2D2D2D2D2D2D2DD9
:10D780002D2D2D2D2D2D2D2D2D2D2D2D000000007D
:10D7900056657273696F6E3A2000000072746320E0
:10D7A0006973206F6E6C696E65000000727463208F
:10D7B0006973206F66666C696E65000065657072DE
:10D7C0006F6D206973206F6E6C696E6500000000DC
:10D7D00063757272656E7420656570726F6D207608
:10D7E000657273696F6E3A203078253038780D0A8B
:10D7F0000000000072656164696E672069722063D1
:10D800006F6465732066726F6D20656570726F6DF1
:10D810000000000072656164696E6720646973705E
:10D820006C617920636F6E66696775726174696F88
:10D830006E2066726F6D20656570726F6D000000FE
:10D8400072656164696E672074696D65736572766F
:10D85000657220646174612066726F6D2065657009
:10D86000726F6D0072656164696E67206E696768CA
:10D87000742074696D6572732066726F6D206565C2
:10D8800070726F6D0000000072656164696E6720E0
:10D8900074656D7020636F6E666967757261746917
:10D8A0006F6E2066726F6D20656570726F6D00001F
:10D8B000656570726F6D206973206F66666C696E46
:10D8C000650000007570646174696E67204545509D
:10D8D000524F4D20746F2076657273696F6E2030E1
:10D8E00078253038780D0A0077726974696E672080
:10D8F00076657273696F6E20746F20454550524F84
:10D900004D206661696C656400000000777269747F
:10D91000696E6720495220636F64657320746F20BD
:10D92000454550524F4D206661696C6564000000AA
:10D9300077726974696E6720636F6E6669672074B9
:10D940006F20454550524F4D206661696C656400FB
:10D9500077726974696E672074696D657365727634
:10D960006572206461746120746F20454550524F88
:10D970004D206661696C656400000000777269740F
:10D98000696E67206E696768742074696D652064CC
:10D9900061746120746F20454550524F4D2066617F
:10D9A000696C65640000000063616C6C696E6720DF
:10D9B0004952206C6561726E2066756E6374696F82
:10D9C0006E0000007573657220627574746F6E204E
:10D9D000707265737365643A20636F6E666967750C
:10D9E00072696E6720657370383236362061732035
:10D9F00061636365737320706F696E74000000006B
:10DA0000776F7264636C6F636B0000003132333484
:10DA10003536373839300000636F6D6D616E643AAA
:10DA20002073657420646973706C617920636F6C16
:10DA30006F727320746F2025642025642025640D87
:10DA40000A000000636F6D6D616E643A2073657447
:10DA500020616D62696C6967687420636F6C6F72B6
:10DA60007320746F2025642025642025640D0A002E
:10DA7000636F6D6D616E643A2073657420706F77AB
:10DA80006572202573000000636F6D6D616E643AEE
:10DA90002073657420646973706C6179206D6F64A4
:10DAA0006520746F2025640D0A000000636F6D6DA2
:10DAB000616E643A2073657420616D62696C696798
:10DAC0006874206D6F646520746F2025640D0A00F2
:10DAD000636F6D6D616E643A2073657420616E6969
:10DAE0006D6174696F6E206D6F646520746F2025A1
:10DAF000640D0A00636F6D6D616E643A2073657426
:10DB000020636F6C6F7220616E696D6174696F6EF6
:10DB1000206D6F646520746F2025640D0A0000007D
:10DB2000636F6D6D616E643A2073686F7720746502
:10DB30006D7065726174757265000000636F6D6D64
:10DB4000616E643A2073657420646973706C6179E6
:10DB5000206272696768746E65737320746F202524
:10DB6000642C2064697361626C65206175746D6FEB
:10DB70006D61746963206272696768746E6573733E
:10DB800020636F6E74726F6C20706572204C44520B
:10DB90000D0A0000636F6D6D616E643A20736574E9
:10DBA00020616D62696C6967687420627269676878
:10DBB000746E65737320746F2025640D0A00000075
:10DBC000636F6D6D616E643A20656E61626C652095
:10DBD0006175746F6D6174696320627269676874DE
:10DBE0006E65737320636F6E74726F6C000000005B
:10DBF000636F6D6D616E643A2064697361626C6518
:10DC0000206175746F6D6174696320627269676801
:10DC1000746E65737320636F6E74726F6C000000B6
:10DC2000636F6D6D616E643A20736574206469730F
:10DC3000706C617920666C61677320746F20307836
:10DC40002530327800000000636F6D6D616E643ABC
:10DC500020737461727420646973706C61792074CC
:10DC600065737400636F6D6D616E643A20736574E3
:10DC70002074696D6520746F202573202534642D10
:10DC8000253032642D2530326420253032643A2527
:10DC90003032643A253032640D0A0000636F6D6DD6
:10DCA000616E643A207374617274206E65742074BE
:10DCB000696D65207265717565737400636F6D6D54
:10DCC000616E643A206C6561726E20495220636F08
:10DCD00064657300636F6D6D616E643A2073617685
:10DCE0006520646973706C61792073657474696E02
:10DCF00067730000636F6D6D616E643A20707269C6
:10DD00006E74207469636B65723A2027257327004F
:10DD10006C64723A206F6C64206272696768746E1A
:10DD200065733A202564206E6577206272696768A2
:10DD3000746E6573733A2025640D0A00657370383C
:10DD4000323636206E6F772075700000657370383C
:10DD5000323636206E6F77206F6E6C696E6500000C
:10DD6000202049502025730064636637373A202508
:10DD700073202534642D253032642D253032642003
:10DD8000253032643A253032643A253032640D0A47
:10DD90000000000072656164207274633A2025738C
:10DDA000202534642D253032642D25303264202521
:10DDB0003032643A253032643A253032640D0A003C
:10DDC000466F756E642054696D65723A2025732024
:10DDD000617420253032643A253032640D0A000027
:10DDE000676F742074656D706572617475726520FB
:10DDF00066726F6D20445331387878783A20256404
:10DE000025730D0A00000000676F742074656D7043
:10DE1000657261747572652066726F6D205254432D
:10DE20003A20256425730D0A000000006E6F2074EF
:10DE3000656D706572617475726520617661696C7B
:10DE400061626C6500000000757064617465206437
:10DE50006973706C6179000049524D503A20504FFF
:10DE6000574552206B65790049524D503A204F4B2F
:10DE7000206B65790000000049524D503A206465DE
:10DE80006372656D656E7420646973706C6179206E
:10DE90006D6F64650000000049524D503A20696E74
:10DEA0006372656D656E7420646973706C6179204E
:10DEB0006D6F64650000000049524D503A20646562
:10DEC0006372656D656E7420616E696D6174696FF2
:10DED0006E206D6F6465000049524D503A20696EA6
:10DEE0006372656D656E7420616E696D6174696FD2
:10DEF0006E206D6F6465000049524D503A20646594
:10DF00006372656D656E7420686F75720000000045
:10DF100049524D503A20696E6372656D656E74208A
:10DF2000686F75720000000049524D503A206465D8
:10DF30006372656D656E74206D696E757465000041
:10DF400049524D503A20696E6372656D656E74205A
:10DF50006D696E757465000049524D503A206465D4
:10DF60006372656D656E74207265642062726967A4
:10DF700068746E657373000049524D503A20696EA3
:10DF80006372656D656E7420726564206272696784
:10DF900068746E657373000049524D503A20646591
:10DFA0006372656D656E7420677265656E2062725E
:10DFB000696768746E6573730000000049524D50C4
:10DFC0003A20696E6372656D656E7420677265656F
:10DFD0006E206272696768746E657373000000007A
:10DFE00049524D503A2064656372656D656E7420C8
:10DFF000626C7565206272696768746E6573730020
:10E0000049524D503A20696E6372656D656E742099
:10E01000626C7565206272696768746E65737300FF
:10E0200049524D503A2064656372656D656E742087
:10E030006272696768746E657373000049524D506F
:10E040003A20696E6372656D656E742062726967ED
:10E0500068746E657373000049524D503A206765CD
:10E06000742074656D70657261747572650000006E
:10E07000706F7765725F696E697428292063616CBF
:10E080006C656400737769746368696E6720706F8C
:10E09000776572206F6E0000737769746368696ECC
:10E0A0006720706F776572206F6666002020676555
:10E0B000742074656D70657261747572650000001E
:10E0C0002020706F776572206F66662F6F6E00007C
:10E0D00020206F6B00000000202064656372656D76
:10E0E000656E7420646973706C6179206D6F64650E
:10E0F000000000002020696E6372656D656E7420FB
:10E10000646973706C6179206D6F64650000000054
:10E11000202064656372656D656E7420616E696D43
:10E120006174696F6E206D6F646500002020696EF8
:10E130006372656D656E7420616E696D6174696F7F
:10E140006E206D6F64650000202064656372656DEC
:10E15000656E7420686F7572000000002020696E83
:10E160006372656D656E7420686F757200000000E3
:10E17000202064656372656D656E74206D696E75CF
:10E18000746500002020696E6372656D656E742091
:10E190006D696E7574650000202064656372656D3D
:10E1A000656E7420726564206272696768746E655A
:10E1B000737300002020696E6372656D656E742054
:10E1C000726564206272696768746E6573730000BB
:10E1D000202064656372656D656E74206772656585
:10E1E0006E206272696768746E6573730000000068
:10E1F0002020696E6372656D656E74206772656557
:10E200006E206272696768746E6573730000000047
:10E21000202064656372656D656E7420626C75653F
:10E22000206272696768746E657373002020696E7E
:10E230006372656D656E7420626C756520627269CB
:10E240006768746E65737300202064656372656D22
:10E25000656E7420676C6F62616C206272696768BA
:10E26000746E6573730000002020696E6372656DC3
:10E27000656E7420676C6F62616C2062726967689A
:10E28000746E6573730000002020746F67676C659F
:10E29000206175746F206272696768746E6573734C
:10E2A0000000000020205468616E6B20796F75219A
:10E2B000000000003139322E35332E3130332E310B
:10E2C000303300004E65772074696D657A6F6E6536
:10E2D0003A2025640D0A00004300000004020020DB
:10E2E0001F0000001C0000001F0000001E000000B6
:10E2F0001F0000001E0000001F0000001F000000A3
:10E300001E0000001F0000001E0000001F00000093
:10E310001F0000001D0000001F0000001E00000084
:10E320001F0000001E0000001F0000001F00000072
:10E330001E0000001F0000001E0000001F00000063
:10E340006D0100006E010000232D302B2000686C51
:10E350004C00656667454647003031323334353608
:10E360003738394142434445460030313233343541
:10E3700036373839616263646566000020202020EA
:10E380002020202020282828282820202020202065
:10E390002020202020202020202020208810101045
:10E3A000101010101010101010101010040404049D
:10E3B0000404040404041010101010101041414112
:10E3C000414141010101010101010101010101017D
:10E3D0000101010101010110101010101042424210
:10E3E000424242020202020202020202020202024D
:10E3F00002020202020202101010102000000000AF
:10E40000000000000000000000000000000000000C
:10E4100000000000000000000000000000000000FC
:10E4200000000000000000000000000000000000EC
:10E4300000000000000000000000000000000000DC
:10E4400000000000000000000000000000000000CC
:10E4500000000000000000000000000000000000BC
:10E4600000000000000000000000000000000000AC
:10E47000000000000000000000000000000000009C
:08E480005C1DFF7F010000009C
:10E488000000000001020304010203040607080952
:10E49800F0BE0008D8BE0008F4BE0008F8BE0008A8
:10E4A800FCBE0008E8BE0008ECBE0008FF00000043
:10E4B800FF000000E8030000010000000500000064
:10E4C80020000000200000000300000020000000E1
:10E4D80030C400085D1E00080200000002000000B1
:10E4E8000000000040C40008D11E0008040000001D
:10E4F800040000000300000048C400089529000833
:10E5080002000000020000000300000050C40008E0
:10E51800412700080200000002000000030000007C
:10E5280058C400089D1A00080200000002000000FC
:10E538000000000060C40008252C0008020000004C
:10E54800020000000300000068C4000895260008C7
:10E5580004000000040000000300000074C4000868
:10E56800D12400080200000002000000030000009F
:10E578007CC400088D2F0008020000000200000083
:10E588000300000084C40008F12200080200000013
:10E5980002000000030000008CC400087921000874
:10E5A80004000000040000000300000094C40008F8
:10E5B800000000000000000000000000C8CE0008B5
:10E5C8000000000000000000000000009CC40008DB
:10E5D80000000000000000000000000038C400082F
:10E5E80004000000040000000100000020000000FA
:10E5F80001000000050000003C00000030C40008D5
:10E6080001000000010000000000000038C40008FC
:10E6180004000000040000000100000016000000D3
:10E628000F000000010000000F0000004CC60008A9
:10E6380054C600085CC6000868C60008FFFF000052
:10E64800FFFF0000D80E0000FF000000FF000000E0
:10E65800FFFFFFFFFF0000000000000000000000B7
:10E668000102030406070809007A030A01000000F2
:10E678003139322E35332E3130332E3130330000DC
:10E688000000000000000000000000000000000082
:10E698000000000000000000000000000000000072
:10E6A80000000000D8E200080000000000000000A0
:10E6B8000000000000000000000000000000000052
:10E6C8000000000000000000000000000000000042
:10E6D8000000000000000000000000000000000032
:10E6E80000000000040200207BE300080100000095
:10E6F800000000004A0000000000000000000000C8
:10E708000000000000000000000000000000000001
:10E718004A000000000000000000000000000000A7
:10E72800000000000000000000000000AD0100082B
:04E73800890100084B
:0400000508000000EF
:00000001FF
